:020000040800F2
:10000000F0AD00209D010008093A0108892401088B
:100010002D3701088D35000849D401080000000083
:10002000000000000000000000000000216701083F
:10003000B56C00080000000001430108457101088B
:10004000B7010008B7010008B7010008B7010008B0
:10005000B7010008B7010008B96C0008B701000833
:10006000B7010008C56C0008D16C0008B701000892
:100070001567000825670008B7010008B7010008E8
:10008000B7010008B7010008B7010008B701000870
:1000900091350008A1350008B7010008DD6C0008A3
:1000A00039720108B7010008B7010008B70100085C
:1000B000B7010008B7010008B7010008B701000840
:1000C000B7010008B7010008B7010008B701000830
:1000D000B70100085DA20108B7010008B7010008D8
:1000E000B7010008B7010008B7010008B701000810
:1000F000B7010008B7010008B7010008356700081C
:10010000B7010008B7010008B7010008B7010008EF
:10011000B7010008B7010008B701000849720108DB
:10012000B7010008456700085567000865670008C3
:10013000B7010008B7010008B7010008B7010008BF
:10014000B1350008C1350008B7010008793A010847
:1001500075670008856700089567000879A201089F
:10016000B7010008B7010008B7010008B70100088F
:10017000B7010008B7010008B7010008000000003F
:10018000B7010008B7010008DFF80CD000F0C4FB8D
:100190000048004795D70108F0AD00200648804789
:1001A00006480047FEE7FEE7FEE7FEE7FEE7FEE75C
:1001B000FEE7FEE7FEE7FEE7197201088901000885
:1001C0002DE9F05F0546002092469B46884606468C
:1001D000814640241BE0284641464746224600F01F
:1001E0002DFA53465A46C01A914110D3114618466B
:1001F000224600F014FA2D1A67EB01084F462246FA
:100200000120002100F00BFA17EB00094E41201EDF
:10021000A4F10104DFDC484631462A464346BDE8E6
:10022000F09F00000649074A0868504343F239022C
:10023000104408604008704701490860704700009A
:10024000000000206D4EC64140EA01039B0703D029
:1002500009E008C9121F08C0042AFAD203E011F805
:10026000013B00F8013B521EF9D27047D2B201E0C7
:1002700000F8012B491EFBD270470022F6E710B5AB
:1002800013460A4604461946FFF7F0FF204610BD04
:1002900010B5044604E00B7800F8013B03B1491C9B
:1002A000521EF8D2204610BD421C10F8011B002936
:1002B000FBD1801A704710B5002200E0521C835C0D
:1002C0008C5CA34201D1002BF8D1D8B2E1B2401A24
:1002D00010BD034611F8012B00F8012B002AF9D1BB
:1002E0001846704730B505460020034600E05B1C09
:1002F000934205D2EC5CC85C201A01D1002CF6D1E7
:1003000030BD2DE9FE4F804681EA0300C00F0C4648
:10031000009021F0004123F00045B8EB0200A94114
:1003200005D24046214690461C460B46024623F025
:100330000040104347D0270DC7F30A00C3F30A510A
:100340000290401A019040286BDAC3F3130040F486
:10035000801B0098924620B10023D2EB030A63EB86
:100360000B0B01985946C0F14002504600F057F976
:1003700006460D4650465946019A00F06FF910EBBB
:1003800008006141002487EA115284EAE7731A43A6
:1003900040D0009A62B3019A012A4FEA075215DC55
:1003A000001B61EB02014FF0004202EA0752CDE967
:1003B0000042001C41F5801132462B4600F0A6F9A0
:1003C00003B0BDE8F08F40462146F9E7001B61EB22
:1003D0000201001C41F5801300185B412018A2F5B2
:1003E000001747EB030140EAD570B6196D4111E0E3
:1003F0006D084FEA360645EAC0754FEA0752001B02
:1004000061EB0201001C41F5801149084FEA300000
:100410000019514132462B4603B0BDE8F04F00F0C1
:1004200066B90098012240000023D0EB020263EB82
:10043000E073009821464FEAE074B8EB000061EBEE
:100440000401E9E783F000435BE781F0004158E7EE
:100450002DE9FE4F81EA030404F0004421F000413D
:1004600000944FF0000B23F0004350EA01045ED0EB
:1004700052EA03045BD0C3F30A54C1F30A552C4477
:10048000A4F2F3340194A0FB0254C1F3130141F42C
:100490008011C3F3130343F4801301FB024400FBF8
:1004A000034E840A970A44EA815447EA8357A4FB1F
:1004B000076802958D0A05FB07854FEA932C04FB1C
:1004C0000C542705029D4FEA065847EA1637B5EB4C
:1004D00008056EEB070C870E920E47EA811742EA79
:1004E0008312A7FB0201B6EB0B0164EB00042B0D9A
:1004F00043EA0C335E1844EB1C50DA465146E7FBE6
:100500000201C5F313044FEA0B3343EA14534FEAD5
:100510000432019C43EA0603A4F10C040294009CFB
:10052000CDE900B400F0F2F803B0BDE8F08F002090
:100530000146F9E70EB5C10F80EAE0700844CA072A
:10054000002140F233438DE80E000A460B4600F0CE
:10055000DDF803B000BD70B5C1F30A5201F00045EB
:100560000024C1F3130140F2FF3341F480119A4299
:1005700001DA002070BD40F233439A42A2F23342C6
:1005800003DC524200F05AF800E090402C43F1D0D6
:10059000404270BD00F0004230F000400AD0C10D72
:1005A00001F56071C0F3160042EA0151C20840072C
:1005B0001143704700200146704701F0004330B4FA
:1005C00021F0004150EA010206D00A0DA2F5607246
:1005D000C1F31301002A02DC30BC00207047440F35
:1005E00044EAC104C100E01830BC00EBC25000F086
:1005F00047B830B50B46014600202022012409E00F
:1006000021FA02F59D4205D303FA02F5491B04FACB
:1006100002F52844151EA2F10102F1DC30BD202AAA
:1006200004DB203A00FA02F1002070479140C2F149
:10063000200320FA03F3194390407047202A04DB7B
:10064000203A21FA02F00021704721FA02F3D0404B
:10065000C2F120029140084319467047202A06DB68
:10066000CB17203A41FA02F043EAE07306E041FA80
:1006700002F3D040C2F1200291400843194670476E
:100680000029A8BF7047401C490008BF20F00100A6
:10069000704710B4B0FA80FC00FA0CF050EA010484
:1006A00004BF10BC704749B1CCF1200421FA04F416
:1006B00011FA0CF118BF012121430843A3EB0C01EF
:1006C000CB1D4FEA00614FEA102042BF002010BC52
:1006D000704700EBC35010440029A4BF10BC704702
:1006E000401C490008BF20F0010010BC704710B545
:1006F000141E73F1000408DA401C41F10001921845
:100700005B411A4301D120F0010010BD2DE9F04DED
:1007100092469B4611B1B1FA81F202E0B0FA80F242
:1007200020329046FFF77BFF04460F4640EA0A005E
:1007300041EA0B0153465A46084313D0114653EA87
:10074000010019D0C8F140025046FFF777FF054677
:100750000E46504659464246FFF761FF084305D012
:10076000012004E020463946BDE8F08D0020054315
:1007700046EAE0762C4337430A986305E40AA0EB87
:1007800008000022FD0A44EA47540A3002D500203E
:100790000146E9E7010510196941DDE9084500193D
:1007A0006941BDE8F04DA2E72DE9F04D81EA03046F
:1007B00004F0004B21F0004514464FF0000A23F0EE
:1007C000004150EA050220D054EA01021DD0C5F3D1
:1007D0000A570246C5F31303C1F31300C1F30A56C7
:1007E00040F4801543F48013A7EB0608101BD6468F
:1007F00008F2FD3873EB050002D308F1010801E0AF
:1008000092185B41B8F1000F03DA00200146BDE801
:10081000F08D00204FF48011064684460EE0171B31
:1008200073EB050705D3121B63EB050306434CEA84
:10083000010C49084FEA300092185B4150EA010769
:10084000EDD152EA030012D082EA040083EA0501E6
:10085000084305D0101BAB4106D20122002306E05D
:1008600000224FF0004302E06FF0010253101AEB38
:1008700006004CEB085110EB0A0041EB0B01BDE800
:10088000F04DFFF734BFC1F30A52C1F3130140F238
:10089000FF3341F480119A4202DA0020014670478A
:1008A00040F233439A42A2F2334202DC5242FFF753
:1008B000C5BEFFF7B4BE000030B5041E71F10004E0
:1008C00004DB4FF00044404264EB0101141E73F15D
:1008D000000405DB1C464FF00043524263EB040367
:1008E0008B4208BF824230BD30B5041E71F1000456
:1008F00004DB4FF00044404264EB0101141E73F12D
:10090000000405DB1C464FF00043524263EB040336
:10091000994208BF904230BD064C074D06E0E068A2
:1009200040F0010394E8070098471034AC42F6D336
:10093000FFF72EFC285E0208485E02080EB540F262
:10094000334102910021CDE900110A460B46FFF721
:10095000DDFE03B000BD70B58C1810F8015B15F01A
:10096000070301D110F8013B2A1106D110F8012B21
:1009700003E010F8016B01F8016B5B1EF9D12B0746
:1009800005D40023521E0DD401F8013BFAE710F8FC
:10099000013BCB1A921C03E013F8015B01F8015BE9
:1009A000521EF9D5A142D8D3002070BD80B582B0C7
:1009B000019042F20030C4F20100009000994868B2
:1009C00020F440304860019842680099486810431C
:1009D000486001980168486820F480704860019878
:1009E00001680269486840EA02204860019801688D
:1009F000486820F040704860019801688268486843
:100A00001043486001980168886820F4006088609D
:100A100001980168C2688868104388600198806AFC
:100A20000121C0F60071884219D0FFE701980168E2
:100A3000886820F07060886001980168826A886820
:100A40001043886001980168886820F040508860F1
:100A500001980168C26A8868104388600CE00198B8
:100A60000168886820F07060886001980168886873
:100A700020F040508860FFE701980168886820F006
:100A8000020088600198027E0168886840EA42009E
:100A90008860019890F8200060B3FFE70198406AF1
:100AA00030B1FFE70198406A082801D8FFE708E065
:100AB00045F24E00C0F6020040F2A6711CF0C4FDE3
:100AC000FFE701980168486840F4006048600198B9
:100AD0000168486820F46040486001980168426AF3
:100AE0004EF20000CFF6FF7000EB42324868104330
:100AF000486006E001980168486820F4006048609A
:100B0000FFE701980168C86A20F47000C862019884
:100B10000168C2690020CFF6F07000EB0252C86A8B
:100B20001043C86201980168886820F400708860EA
:100B3000019890F830200168886840EA4220886077
:100B400001980168886820F48060886001980168D5
:100B50004269886840EA8220886002B080BD000057
:100B600080B58AB008900791089820B9FFE7FF2068
:100B70008DF827009BE0079820B9FFE7FF208DF84C
:100B8000270094E0079890ED000A90ED013A90ED6F
:100B9000021A90ED032A20EE030A21EE021A30EE2B
:100BA000010A30EE000A8DED060A079890ED010A61
:100BB00090ED021A20EE000A21EE011A30EE010A31
:100BC00030EE001AB7EE000A8DED010A30EE410A50
:100BD0008DED050A9DED060ADDED050A21F06CFE9E
:100BE0009DED011A089880ED010A079890ED000A22
:100BF00090ED013A90ED024A90ED032A20EE040AAE
:100C000022EE032A30EE420A30EE000A8DED040A8D
:100C10009DED040AB0EEC00AB4EE410AF1EE10FAFE
:100C20000ADBFFE7DDED040A9FED230A1CF020FD3F
:100C3000089880ED020A07E09DED040A21F03AFBD6
:100C4000089880ED020AFFE7079890ED000A90ED02
:100C5000011A90ED022A90ED033A20EE030A21EEEC
:100C6000021A30EE010A30EE000A8DED030A0798F1
:100C700090ED020A90ED031A20EE000A21EE011A0F
:100C800030EE010A30EE001AB7EE000A30EE410AEB
:100C90008DED020A9DED030ADDED020A21F00CFE46
:100CA000089880ED000A00208DF82700FFE79DF9E5
:100CB00027000AB080BD00BFDB0FC93F80B58CB0F4
:100CC0000A9009918DED080A0A9820B9FFE7FF20E4
:100CD0008DF82F0029E19DED081AB7EE000A80EE8D
:100CE000010A0A9880ED040A0A994FF07E500860C4
:100CF0000A99002048600A9988600A99C860099892
:100D0000002800F00E81FFE7099801680091406813
:100D1000FFF740FC0246009801920A46019942EC16
:100D2000101B8DED020BFFF735FC9DED020B41EC26
:100D3000110B21F0C1FC8DED040B9DF8170080F024
:100D400080008DF8170004980599FFF736FC07908E
:100D5000099890ED000AB5EE400AF1EE10FA2BD199
:100D6000FFE7099890ED010AB5EE400AF1EE10FA9E
:100D700022D1FFE7099890ED020AB5EE400AF1EEA4
:100D800010FA19D1FFE70A9940F2C560C3F64D7019
:100D900008600A9944F62D20C3F60D4048600A9970
:100DA0004AF25640CBF6393088600A9944F2AD7069
:100DB000C3F61970C860B3E09DED070A9FED5D1A98
:100DC000B4EE410AF1EE10FA08DBFFE79DED070AE9
:100DD000B5EE400AF1EE10FA19DDFFE70A9945F683
:100DE0006E10C3F67F7008600A9945F20C30C3F6A6
:100DF000B01048600A9948F6AB00CBF6BB3088606B
:100E00000A9949F28550C3F69750C86087E09DED76
:100E1000070A9FED491AB4EE410AF1EE10FA0ADB17
:100E2000FFE79DED070A9FED431AB4EE410AF1EE8C
:100E300010FA19DDFFE70A9940F2C560C3F64D705C
:100E400008600A9944F62D20C3F60D4048600A99BF
:100E50004AF25640CBF6393088600A9944F2AD70B8
:100E6000C3F61970C86059E09DED070A9FED331A6B
:100E7000B4EE410AF1EE10FA0ADBFFE79DED070A36
:100E80009FED2D1AB4EE410AF1EE10FA19DDFFE7DD
:100E90000A9940F2C560C3F64D7008600A9944F69D
:100EA0002D20C3F60D4048600A994AF25640CBF611
:100EB000393088600A9944F2AD70C3F61970C86081
:100EC0002BE09DED070A9FED1D1AB4EE410AF1EEED
:100ED00010FA08DBFFE79DED070AB5EE400AF1EED8
:100EE00010FA19DDFFE70A9940F2C560C3F64D70AC
:100EF00008600A9944F62D20C3F60D4048600A990F
:100F00004AF25640CBF6393088600A9944F2AD7007
:100F1000C3F61970C860FFE7FFE7FFE7FFE7FFE7E9
:100F2000FFE700208DF82F00FFE79DF92F000CB0A0
:100F300080BD00BFDB0FC93FDB0F49400000B4425A
:100F400081B000900099002088604860086001B07E
:100F50007047000080B52DED048BB2B030902F911A
:100F60002E922D93309828B9FFE7FF208DF8C70007
:100F700000F0F7BD2F9828B9FFE7FF208DF8C700D4
:100F800000F0EFBD2E9828B9FFE7FF208DF8C700CD
:100F900000F0E7BD40F28411C2F200014EF69E70EF
:100FA000C3F6275008602D9848B9FFE730982F996D
:100FB0002E9A00F0DDFD8DF8C70000F0D2BD2D980F
:100FC000006809902D98406808902D9880680790D7
:100FD0009DED090AB5EE400AF1EE10FA19D1FFE7CE
:100FE0009DED080AB5EE400AF1EE10FA11D1FFE7C7
:100FF0009DED070AB5EE400AF1EE10FA09D1FFE7C0
:1010000030982F992E9A00F0B3FD8DF8C70000F0AC
:10101000A8BD2F98006806902F98406805902F98DB
:10102000806804902E98006803902E984068029083
:101030002E988068019030989DED033A90ED010A5A
:1010400090ED022A90ED031A20EE430A9DED023A3C
:1010500022EE032A30EE420A9DED012A21EE021A09
:1010600030EE410AB6EE001A20EE010A8DED270A95
:1010700030989DED034A90ED000A90ED023A90ED14
:10108000032A20EE040A9DED014A23EE043A30EED5
:10109000030A9DED023A22EE032A30EE420A20EEC8
:1010A000010A8DED260A30989DED024A90ED000A66
:1010B00090ED013A90ED032A20EE040A9DED014ADD
:1010C00023EE043A30EE430A9DED033A22EE032A62
:1010D00030EE020A20EE010A8DED250A30989DEDD2
:1010E000014A90ED000A90ED013A90ED022A20EEBF
:1010F000040A9DED024A23EE043A30EE030A9DED08
:10110000033A22EE032A30EE420A20EE010A8DED68
:10111000240A9DED060AB5EE400AF1EE10FA11D14F
:10112000FFE79DED050AB5EE400AF1EE10FA09D190
:10113000FFE79DED040AB5EE400AF1EE10FA00F06B
:101140009984FFE79DED060A20EE000A9DED051A41
:1011500021EE011A30EE010A9DED041A21EE011A6A
:1011600030EE010A11F016FA8DED2C0A9DED2C1AC5
:101170009DED060A20EE010A8DED060A9DED2C1A62
:101180009DED050A20EE010A8DED050A9DED2C1A54
:101190009DED040A20EE010A8DED040A9DED090A79
:1011A00020EE000A9DED081A21EE011A30EE010A28
:1011B0009DED071A21EE011A30EE010A11F0EAF94D
:1011C0008DED2C0A9DED2C1A9DED090A20EE010AE9
:1011D0008DED090A9DED2C1A9DED080A20EE010AFD
:1011E0008DED080A9DED2C1A9DED070A20EE010AEF
:1011F0008DED070A309890ED000A30EE000A9DED63
:10120000091A20EE010A8DED210A309890ED000AAE
:1012100030EE000A9DED081A20EE010A8DED200A3D
:10122000309890ED000A30EE000A9DED071A20EE8E
:10123000010A8DED1F0A309890ED010A30EE000A88
:101240009DED091A20EE010A8DED1E0A309890EDF1
:10125000000A30EE000A8DED190A309890ED010A6F
:1012600030EE000A8DED180A309890ED020A30EE4B
:10127000000A8DED170A309890ED030A30EE000A4F
:101280008DED160A309890ED000A90ED021A30EEBE
:10129000000A20EE010A8DED150A309890ED020A41
:1012A00090ED031A30EE000A20EE010A8DED140ACB
:1012B000309890ED000A20EE000A8DED130A309868
:1012C00090ED000A90ED011A20EE010A8DED120A50
:1012D000309890ED000A90ED021A20EE010A8DED93
:1012E000110A309890ED000A90ED031A20EE010AE1
:1012F0008DED100A309890ED010A20EE000A8DED78
:101300000F0A309890ED010A90ED021A20EE010AC2
:101310008DED0E0A309890ED010A90ED031A20EE43
:10132000010A8DED0D0A309890ED020A20EE000AB8
:101330008DED0C0A309890ED020A90ED031A20EE24
:10134000010A8DED0B0A309890ED030A20EE000A99
:101350008DED0A0A9DED091A9DED130A21EE000A92
:101360009DED202A309890ED025A90ED033A22EE3E
:10137000032A30EE420A9DED1F2A22EE052A30EEA6
:10138000020A9DED0F2A21EE022A30EE020A9DED9F
:10139000182A9DED084A22EE044A24EE054A30EE52
:1013A000040A9DED074A22EE042A22EE032A30EEBB
:1013B000020A9DED0C2A21EE022A30EE420A9DED32
:1013C0000A2A21EE021A30EE410A8DED230A9DED24
:1013D000210A309890ED015A90ED024A90ED033ABF
:1013E00020EE030A9DED081A9DED132A21EE022A34
:1013F00030EE020A9DED1F2A22EE052A30EE420A47
:101400009DED1E2A22EE042A30EE020A9DED0F2ADF
:1014100021EE022A30EE420A9DED0C2A21EE022A2C
:1014200030EE020A9DED172A9DED074A22EE042AAE
:1014300022EE032A30EE020A9DED0A2A21EE021A5C
:1014400030EE410A8DED220A9DED230A20EE000ABE
:101450009DED221A21EE011A30EE010A11F09AF8E0
:10146000B7EE006A86EE000A8DED1D0A9DED210A99
:10147000309890ED012A90ED021A90ED033A20EE9B
:10148000011A9DED200A20EE020A30EE412A9DED60
:10149000071A9DED130A21EE000A30EE022A9DED97
:1014A0001E0A20EE030A30EE020A9DED0F2A21EEFD
:1014B000022A30EE420A9DED172A9DED084A22EEDF
:1014C000042A22EE032A30EE020A9DED0C2A21EEB8
:1014D000022A30EE420A9DED0A2A21EE021A30EE6F
:1014E000010A8DED1C0A9DED1D0A30EE000A8DEDFE
:1014F0001B0A9DED1C0A30EE000A8DED1A0A9DEDC7
:10150000170ADDED0D0A30EEA02A9DED151A31EE19
:10151000422A9DED061A31EE021A20EE010A9DEDD7
:10152000181ADDED123A33EEA32A9DED143A32EE8D
:10153000032A9DED053A32EE432A21EE021A70EE9F
:10154000014A9DED1C3A309890ED011A90ED020A87
:10155000D0ED032A63EE001A9DED1D2A9DED0C7A55
:10156000B6EE004A8DED004A77EE445A9DED0A5AD8
:1015700035EE255A62EE055A9DED115A75EE606AF8
:1015800063EE266A75EEA66ADDED095A75EEA65A77
:1015900061EEA51A71EEA41A62EE222A23EE011A58
:1015A00031EE621ADDED0E2ADDED104A72EEE42A0C
:1015B00062EE222ADDED0B4A73EEA43A63EE233A83
:1015C00072EEA32ADDED083A72EEE32A21EE221A2A
:1015D00031EE211A22EE000A35EE205A22EE052ABB
:1015E0009DED0F5A34EE455A35EE475A23EE053A33
:1015F00032EE032A9DED073A32EE432A20EE020A2C
:1016000030EE010A8DED2B0A9DED160ADDED0D2A57
:1016100032EEA21A9DED152A31EE421A9DED062AF0
:1016200031EE421A20EE010A9DED191ADDED126A23
:1016300036EEA62A9DED143A32EE032A9DED053AC8
:1016400032EE432A21EE021A30EE011A3098D0ED24
:10165000005AD0ED014AD0ED023A90ED032AB1EEE6
:10166000000A24EE803A9DED0F7A37EE075A75EEA8
:10167000461ADDED0C0A30EEA05A75EE211A9DEDEA
:10168000045A35EE215A23EE053A31EE031A9DED48
:101690001C5A65EE027A9DED1D3A74EE601A9DEDBE
:1016A0000A8A71EEC81A23EE218ADDED111A32EE94
:1016B000E19A25EE099A38EE098A9DED099A38EEED
:1016C000498A67EE887A31EE271A63EE233A65EE8F
:1016D000255A73EEA53ADDED0E5ADDED107A75EE62
:1016E000E75A63EE255ADDED0B7A76EEA76A65EED2
:1016F000266A75EEA65ADDED086A75EEE65A63EEC7
:10170000A53A31EE231A23EE022ADDED1A3A63EEF2
:10171000A43A32EE632A71EEA21A23EE213A34EE95
:10172000477A37EE607A25EE075A33EE053A9DED9B
:10173000075A33EE453A22EE032A31EE021A8DEDB6
:101740002A1A9DED191ADDED0D0A30EEA03A9DED35
:10175000152A32EE433A9DED062A32EE032A21EE97
:10176000021A9DED162ADDED124A34EEA43A9DEDE3
:10177000145A33EE053A9DED055A33EE453A22EE02
:10178000032A31EE022A309890ED001AD0ED011AAA
:10179000D0ED022AD0ED033A22EE800A9DED0F5AD9
:1017A00035EE053A33EE467A9DED0C6A36EE063A92
:1017B00033EE077A9DED043A33EE073A20EE030A42
:1017C00070EE025A9DED1B0A20EE620A9DED1C3A56
:1017D00023EE012A30EE420A9DED1D2A34EE467AB0
:1017E000DDED0A6A37EE667A62EE076A9DED117AE0
:1017F00070EEC77A63EE277A76EEA76ADDED097A96
:1018000076EEE76A20EE260A30EE250A62EE211A0D
:1018100063EE233A71EEA31ADDED0E3ADDED105AB8
:1018200073EEE53A62EE233ADDED0B5A74EEA54A0B
:1018300063EE244A73EEA43ADDED084A73EEE43A0F
:1018400061EEA31A30EE210A22EE011ADDED1A1A1A
:1018500061EEA21A31EE611A37EE207A22EE072AE3
:1018600034EE455A35EE465A23EE053A32EE032A57
:101870009DED073A32EE432A21EE021A30EE010ABC
:101880008DED290A9DED180A9DED0D7A37EE071AA8
:101890009DED152A31EE421A9DED062A31EE421ACF
:1018A00020EE010A9DED171ADDED122A32EEA22A72
:1018B0009DED143A32EE032A9DED053A32EE432AAD
:1018C00021EE021A70EE013A9DED1B1A3098D0ED10
:1018D000001A90ED010AD0ED020A90ED032A21EEE4
:1018E000022A9DED1C3A23EE001A31EE421A9DEDBC
:1018F0001D2A9DED0C5A34EE456ADDED0A4A36EE9E
:10190000646A62EE064A9DED116A77EE465A63EE0E
:10191000255A74EEA54ADDED095A74EEE54A21EE2A
:10192000241A31EE231A62EE211A63EE200A70EEB9
:10193000E10ADDED0E1ADDED103A71EEE31A62EE0A
:10194000211ADDED0B3A72EEA32A63EE222A71EE24
:10195000A21ADDED082A71EEE21A60EEA10A31EE5C
:10196000201A22EE000A36EE076A22EE062A9DEDC4
:101970000F6A34EE464A34EE454A23EE043A32EE1C
:10198000032A9DED073A32EE432A20EE020A30EE9A
:10199000010A8DED280A9DED2B0A20EE000A9DED2F
:1019A0002A1A21EE011A30EE010A9DED291A21EEC4
:1019B000011A30EE010A9DED281A21EE011A30EECF
:1019C000010A10F0E7FD8DED2C0A9DED2C1A9DED1E
:1019D0002B0A20EE010A8DED2B0A9DED2C1A9DEDB0
:1019E0002A0A20EE010A8DED2A0A9DED2C1A9DEDA2
:1019F000290A20EE010A8DED290A9DED2C1A9DED94
:101A0000280A20EE010A8DED280A40F28410C2F265
:101A1000000090ED000A9DED2B1A20EE011A9DEDBD
:101A2000270A30EE410A8DED270A90ED000A9DED60
:101A30002A1A20EE011A9DED260A30EE410A8DED9C
:101A4000260A90ED000A9DED291A20EE011A9DED5F
:101A5000250A30EE410A8DED250A90ED000A9DED34
:101A6000281A20EE011A9DED240A30EE410A8DED70
:101A7000240AFFE79DED271A309890ED000A90EDBB
:101A8000042A21EE021A30EE010A80ED000A9DEDD3
:101A9000261A309890ED010A90ED042A21EE021AE0
:101AA00030EE010A80ED010A9DED251A309890ED87
:101AB000020A90ED042A21EE021A30EE010A80EDAE
:101AC000020A9DED241A309890ED030A90ED042A45
:101AD00021EE021A30EE010A80ED030A309890EDF3
:101AE000000A90ED013A90ED022A90ED031A20EEE3
:101AF000000A23EE033A30EE030A22EE022A30EE09
:101B0000020A21EE011A30EE010A10F043FD8DEDBC
:101B10002C0A9DED2C1A309890ED000A20EE010A57
:101B200080ED000A9DED2C1A309890ED010A20EE10
:101B3000010A80ED010A9DED2C1A309890ED020A01
:101B400020EE010A80ED020A9DED2C1A309890EDEE
:101B5000030A20EE010A80ED030A00208DF8C70079
:101B6000FFE79DF9C70032B0BDEC048B80BD0000DB
:101B700080B5A0B01E901D911C921E9820B9FFE761
:101B8000FF208DF87F00D3E21D9820B9FFE7FF20EA
:101B90008DF87F00CCE21C9820B9FFE7FF208DF87C
:101BA0007F00C5E240F28411C2F2000142F6023029
:101BB000C3F6075008601D9800681B901D98406888
:101BC0001A901D98806819901C98006818901C98AD
:101BD000406817901C98806816901E989DED183AE2
:101BE00090ED010A90ED022A90ED031A20EE430ACF
:101BF0009DED173A22EE032A30EE420A9DED162A99
:101C000021EE021A30EE410AB6EE001A20EE010A69
:101C10008DED100A1E989DED184A90ED000A90ED8A
:101C2000023A90ED032A20EE040A9DED164A23EEB7
:101C3000043A30EE030A9DED173A22EE032A30EE05
:101C4000420A20EE010A8DED0F0A1E989DED174AFB
:101C500090ED000A90ED013A90ED032A20EE040A7F
:101C60009DED164A23EE043A30EE430A9DED183AF4
:101C700022EE032A30EE020A20EE010A8DED0E0A52
:101C80001E989DED164A90ED000A90ED013A90EDF8
:101C9000022A20EE040A9DED174A23EE043A30EEA4
:101CA000030A9DED183A22EE032A30EE420A20EE96
:101CB000010A8DED0D0A9DED1B0AB5EE400AF1EE0D
:101CC00010FA11D1FFE79DED1A0AB5EE400AF1EEC8
:101CD00010FA09D1FFE79DED190AB5EE400AF1EEC1
:101CE00010FA00F0AE81FFE79DED1B0A20EE000A1E
:101CF0009DED1A1A21EE011A30EE010A9DED191A16
:101D000021EE011A30EE010A10F044FC8DED150AA7
:101D10009DED151A9DED1B0A20EE010A8DED1B0AA3
:101D20009DED151A9DED1A0A20EE010A8DED1A0A95
:101D30009DED151A9DED190A20EE010A8DED190A87
:101D40001E9890ED000A30EE000A8DED0C0A1E98E8
:101D500090ED010A30EE000A8DED0B0A1E9890ED11
:101D6000020A30EE000A8DED0A0A1E9890ED030A71
:101D700030EE000A8DED090A1E9890ED000AB1EED2
:101D8000003A20EE030A8DED080A1E9890ED010A34
:101D900020EE030A8DED070A1E9890ED020A20EE50
:101DA000030A8DED060A1E9890ED010AB2EE001AA4
:101DB00020EE010A8DED050A1E9890ED020A20EE34
:101DC000010A8DED040A1E9890ED000A20EE000A2B
:101DD0008DED030A1E9890ED010A20EE000A8DEDAC
:101DE000020A1E9890ED020A20EE000A8DED010A0B
:101DF0001E9890ED030A20EE000A8DED000A9DED7D
:101E0000081A9DED010A21EE000A9DED0A2A9DEDBA
:101E10001B4A22EE042A30EE020A9DED022A21EE30
:101E2000021A30EE010A9DED0B1A9DED1A2A21EEE1
:101E3000021A30EE410A8DED140A9DED071A9DED50
:101E4000000A21EE000A9DED092A9DED1B4A22EEB3
:101E5000042A30EE420A9DED032A22EE032A1E9840
:101E600090ED014A22EE042A30EE020A9DED0C2A82
:101E70009DED1A4A22EE042A30EE420A30EE410A63
:101E80009DED052A9DED024A22EE044A30EE040A39
:101E90009DED014A22EE042A30EE020A9DED192A38
:101EA00021EE021A30EE010A8DED130A9DED030AB0
:101EB00020EE030A1E9890ED021A20EE010A9DED15
:101EC0000C1A9DED1B2A21EE021A30EE010A9DED3F
:101ED000061A9DED002A21EE022A30EE020A9DED3F
:101EE000092A9DED1A4A22EE042A30EE420A30EE0B
:101EF000410A9DED042A9DED024A22EE044A30EE8D
:101F0000040A9DED014A22EE042A30EE020A9DEDFC
:101F1000192A21EE021A30EE010A8DED120A9DED0A
:101F2000020A20EE030A1E9890ED032A20EE020A10
:101F30009DED0B1A9DED1B4A21EE041A30EE410A6D
:101F40009DED011A21EE031A21EE021A30EE010A6C
:101F50009DED0A1A9DED1A2A21EE021A30EE410A71
:101F60008DED110A9DED140A20EE000A9DED131A65
:101F700021EE011A30EE010A9DED121A21EE011A2E
:101F800030EE010A9DED111A21EE011A30EE010A20
:101F900010F000FB8DED150A9DED151A9DED140A4C
:101FA00020EE010A8DED140A9DED151A9DED130A20
:101FB00020EE010A8DED130A9DED151A9DED120A12
:101FC00020EE010A8DED120A9DED151A9DED110A04
:101FD00020EE010A8DED110A40F28410C2F20000D9
:101FE00090ED000A9DED141A20EE011A9DED100AE5
:101FF00030EE410A8DED100A90ED000A9DED131AA6
:1020000020EE011A9DED0F0A30EE410A8DED0F0A08
:1020100090ED000A9DED121A20EE011A9DED0E0AB8
:1020200030EE410A8DED0E0A90ED000A9DED111A79
:1020300020EE011A9DED0D0A30EE410A8DED0D0ADC
:10204000FFE79DED101A1E9890ED000A90ED042A0E
:1020500021EE021A30EE010A80ED000A9DED0F1A02
:102060001E9890ED010A90ED042A21EE021A30EE3E
:10207000010A80ED010A9DED0E1A1E9890ED020AEC
:1020800090ED042A21EE021A30EE010A80ED020AD8
:102090009DED0D1A1E9890ED030A90ED042A21EE95
:1020A000021A30EE010A80ED030A1E9890ED000A34
:1020B00090ED013A90ED022A90ED031A20EE000A0D
:1020C00023EE033A30EE030A22EE022A30EE020A31
:1020D00021EE011A30EE010A10F05CFA8DED150ABE
:1020E0009DED151A1E9890ED000A20EE010A80ED74
:1020F000000A9DED151A1E9890ED010A20EE010AC6
:1021000080ED010A9DED151A1E9890ED020A20EE51
:10211000010A80ED020A9DED151A1E9890ED030A42
:1021200020EE010A80ED030A00208DF87F00FFE712
:102130009DF97F0020B080BD84B00290019102988B
:1021400020B9FFE7FE208DF80F001CE0019820B9B0
:10215000FFE7FE208DF80F0015E0029900200090A7
:10216000C1F81B00886148610861C86088604860E8
:102170000199886148610861C860886048600860AA
:102180008DF80F00FFE79DF90F0004B070470000C5
:1021900080B582B00090009820B9FFE7FE208DF84E
:1021A00007002AE042F29C30C2F200000078C0072B
:1021B00020B1FFE7FD208DF807001EE01BF004FFB3
:1021C00042F6AC71C2F20001086020B9FFE7FE20C0
:1021D0008DF8070011E042F27D42C0F600020220B5
:1021E000032101F037F942F29C31C2F200010120D3
:1021F000087000208DF80700FFE79DF9070002B086
:1022000080BD000080B582B0019000910199C4208A
:1022100081F826000199DDF800C0DCF80000DCF848
:102220000420DCF80830DCF80CC0C1F833C0C1F879
:102230002F30C1F82B20C1F827000199002081F828
:102240003700019890F84A00012808D1FFE701996A
:1022500091F8370040F0010081F837001DE0019847
:1022600090F84A00022808D1FFE7019991F8370059
:1022700040F0020081F837000EE0019890F84A0023
:10228000032808D1FFE7019991F8370040F00400D6
:1022900081F83700FFE7FFE7FFE7019827302121AA
:1022A0004FF6FF7202F0EEF90199A1F84800002004
:1022B00002B080BD80B582B0019000910199A82044
:1022C000C8770198203004214FF6FF7202F0DAF946
:1022D00001998884002002B080BD000080B584B0E0
:1022E00002900191029804301B2102F0E7F908B92D
:1022F000FFE724E0029880680199486002984068EE
:10230000019908600298C068019988600298007C71
:10231000C0F3C000019908760298D0F81100019925
:10232000C8600298D0F81500019908610298D0F8A9
:1023300019000199486100208DF80F000AE041F270
:102340008811C2F20001086801300860FF208DF892
:102350000F00FFE79DF90F0004B080BD80B582B08B
:102360000090022001F016F8009904311B220FF0B2
:102370002DFF20B9FFE700208DF8070003E0FF20C4
:102380008DF80700FFE79DF9070002B080BD00004F
:1023900080B584B002908DF807109DF80700C00743
:1023A00090B1FFE7022000F0F5FF02991F312B22C8
:1023B0000FF09CFF20B9FFE700208DF80F0015E01B
:1023C000FF208DF80F0011E0022000F0E3FF0299DA
:1023D000263124220FF08AFF20B9FFE700208DF874
:1023E0000F0003E0FF208DF80F00FFE79DF90F00BD
:1023F00004B080BD80B54FF48040012100221BF065
:1024000055FDA0F58040B0FA80F0400980BD000085
:1024100084B08DED030ACDED020A9DED030A9DED1A
:10242000021AB1EE411AB4EE410AF1EE10FA07DADF
:10243000FFE79DED020AB1EE400A8DED010A18E0BA
:102440009DED030A9DED021AB4EE410AF1EE10FA79
:1024500005DDFFE79DED020A8DED000A04E09DED2C
:10246000030A8DED000AFFE79DED000A8DED010ADC
:10247000FFE79DED010A04B07047000080B542F609
:10248000AC70C2F2000000684FF480411BF0BCFC4D
:1024900080BD000080B542F69C70C2F2000000686A
:1024A00002211BF0B1FC80BD80B582B040F6BC12A9
:1024B000C2F20002002001901221132300F06EFAF4
:1024C000019802B080BD000080B5082001214FF0C6
:1024D000FF321BF0EBFC80BD81B000909FED010A44
:1024E00001B070470000C84380B542F69C70C2F24C
:1024F0000000006801211BF087FC80BD82B00190C4
:10250000019890ED000A00209FED141AB4EE410AE4
:10251000F1EE10FA00901BDAFFE7019890ED010A46
:1025200000209FED0E1AB4EE410AF1EE10FA009071
:102530000EDAFFE7019890ED020A9FED081A0020DD
:10254000B4EE410AF1EE10FAB8BF01200090FFE7A7
:10255000009800F0010002B0704700BF8FC2F53C48
:1025600080B540F6BC10C2F20000C21D012002215D
:10257000062300F013FA002080BD000080B504207F
:1025800001214FF0FF321BF091FC80BD80B58CB073
:102590000A9009910A9820B9FFE7FE208DF82F00D4
:1025A000B5E0099820B9FFE7FE208DF82F00AEE0D6
:1025B00042F29830C2F200000078C00720B1FFE775
:1025C000FD208DF82F00A2E01BF0FEFC42F69C716E
:1025D000C2F20001086020B9FFE7FE208DF82F004D
:1025E00095E009980A99C861002008907E21B622DA
:1025F000069200F087FA069A0120142100F082FA70
:102600001E20079000F01CFB0799089800F00CFAB8
:102610000899084600F008FA1E2804D0FFE7FC20BD
:102620008DF82F0073E00120002100F0FDF90F2844
:1026300004D0FFE7FC208DF82F0068E01020039005
:1026400000F0A6FB2020049000F0A2FB42F6251229
:10265000C0F6000201210291084600F079FE0398BD
:1026600042F29541C0F6000100F006FC049842F2E7
:10267000E941C0F6000100F0FFFB00200590402179
:10268000AA2200F03FFA029A0598412100F03AFA96
:1026900005985321082200F035FA059858210422A4
:1026A000019200F02FFA019A05987D2100F02AFA94
:1026B000322000F0C5FA029A0F21104600F022FAEB
:1026C00002980399032200F01DFA0298059A162138
:1026D00000F018FA029A1821104600F013FA029836
:1026E0001521802200F00EFA0A2000F0A9FA0299C2
:1026F000039842F29832C2F20002117000F082FB9D
:10270000049800F07FFB05988DF82F00FFE79DF9F6
:102710002F000CB080BD000084B00290029820B958
:10272000FFE7FE208DF80F006AE040F6BC11C2F210
:102730000001B1F80100ADF80600B1F80300ADF8F2
:102740000400B1F80500ADF80200BDF9060000EE86
:10275000100AB8EEC00A029880ED000ABDF9040024
:1027600000EE100AB8EEC00A029880ED010ABDF929
:10277000020000EE100AB8EEC00A029880ED020ACC
:10278000029890ED000A9FED201A80EE010A80ED7C
:10279000000A029890ED010A80EE010A80ED010A1C
:1027A000029890ED020A80EE010A80ED020A487C50
:1027B000897CC00040EA5110ADF80000BDF900006E
:1027C000B0F5806F07DBFFE7BDF80000A0F5006003
:1027D000ADF80000FFE7BDF9000000EE100AB8EE0A
:1027E000C00AB4EE001A20EE010AB3EE071A30EE6A
:1027F000010A029880ED060A00208DF80F00FFE71D
:102800009DF90F0004B0704700A0AA4584B0029063
:10281000029820B9FFE7FE208DF80F007AE040F61D
:10282000BC10C2F20000B0F80710ADF80610B0F806
:102830000910ADF80410B0F80B00ADF80200BDF9B6
:10284000060000EE100AB8EEC00A029880ED030AF6
:10285000BDF9040000EE100AB8EEC00A029880ED3F
:10286000040ABDF9020000EE100AB8EEC00A029890
:1028700080ED050A029890ED030A9FED281A80EE7C
:10288000010A80ED030A029890ED040A80EE010A25
:1028900080ED040A029890ED050A80EE010A80EDB1
:1028A000050A029890ED030A9FED1D1A20EE010A19
:1028B00080ED030A029890ED040A20EE010A80EDF3
:1028C000040A029890ED050A20EE010A80ED050A3F
:1028D0000298C16991ED001A90ED030A30EE410AA9
:1028E00080ED030A0298C16991ED011A90ED040A86
:1028F00030EE410A80ED040A0298C16991ED021A96
:1029000090ED050A30EE410A80ED050AFE208DF8B3
:102910000F00FFE79DF90F0004B070476F120342EC
:1029200035FA8E3C80B50020C4F20200102108F078
:10293000F9FC80B9FFE70020C4F202001021012257
:1029400008F01AFD42F69C70C2F2000000680821EF
:102950001BF05AFAFFE740F20040C4F202000121E6
:1029600008F0E0FC88B9FFE740F20040C4F2020042
:102970000122114608F000FD42F69C70C2F20000F0
:10298000006804211BF040FAFFE780BD80B50320FA
:1029900001214FF0FF321BF089FA80BD80B586B06F
:1029A0008DF817008DF8161004928DF80F300498EA
:1029B00008B9FFE736E09DF817000146029120B103
:1029C000FFE70298012808D010E00020C4F20200BE
:1029D0001021002208F0D0FC08E040F20040C4F2D0
:1029E00002000121002208F0C7FCFFE79DF8160055
:1029F00040F0800040F6CF11C2F200010091087053
:102A00000120019000F084FC0099019A14230BF03E
:102A1000F1FE019800F07CFC04999DF80F200BF06A
:102A2000ABFDFFE706B080BD80B586B08DF816001F
:102A30008DF81510012000F003F99DF816000146ED
:102A4000049120B1FFE70498012808D010E000208D
:102A5000C4F202001021002208F08EFC08E040F2CF
:102A60000040C4F202000121002208F085FCFFE7CB
:102A70009DF8150040F0800040F6CF11C2F2000131
:102A8000019108700120009000F042FC009A019929
:102A9000142302930BF0AEFE009800F039FC01996C
:102AA000029B02220BF050FC9DF816000146039198
:102AB00020B1FFE7039801280FD01EE00020C4F2E8
:102AC00002001021012208F057FC40F6CF10C2F29C
:102AD000000040788DF817000FE040F20040C4F28B
:102AE00002000122114608F047FC40F6CF10C2F266
:102AF000000000788DF81700FFE79DF8170006B07A
:102B000080BD000080B584B08DF80F008DF80E10E8
:102B10008DF80D209DF80E0000F07F0040F6CF11DB
:102B2000C2F2000108709DF80D004870012000F00D
:102B300087F89DF80F000146029120B1FFE7029847
:102B4000012808D010E00020C4F202001021002269
:102B500008F012FC08E040F20040C4F2020001213B
:102B6000002208F009FCFFE7012000F0D1FB40F64D
:102B7000CF11C2F20001022214230BF03BFE9DF89C
:102B80000F000146019120B1FFE70198012808D00C
:102B900010E00020C4F202001021012208F0ECFB3A
:102BA00008E040F20040C4F202000122114608F0A1
:102BB000E3FBFFE704B080BD83B08DF807009DF80C
:102BC00007000146009150B1FFE7009801280CD1A1
:102BD000FFE741F22470C2F20000029008E041F2E7
:102BE000FC60C2F20000029002E000200290FFE7C9
:102BF000029803B07047000082B08DF806008DF88F
:102C000005100092009820B9FFE7FE208DF807001C
:102C100011E000989DF8061040F2F823C2F200037C
:102C2000342211FB02319DF8052041F822000020DA
:102C30008DF80700FFE79DF9070002B0704700001C
:102C400080B586B004901AF067FE01464FF47A70A2
:102C5000B0FBF1F0039004980399B0FBF1F00290FF
:102C60001AF01CFE0146481C019198B1FFE701983B
:102C7000022820D3FFE7019802280FD0FFE7019830
:102C80000338022806D3FFE701986FF0004188421D
:102C900015D1FFE7FF208DF8170014E0029818B156
:102CA000FFE70298009002E001200090FFE7009803
:102CB0001AF0AEFD03E0049807F0C8FDFFE700201E
:102CC0008DF81700FFE79DF9170006B080BD0000E2
:102CD00080B588B007900798E0B1FFE707980B2808
:102CE00018D8FFE707980490002002900220069071
:102CF0000120059007F00AFFFFE7322004F0A4FA54
:102D000008B1FFE7F9E702A801A907F0C1FD07F044
:102D10006FFEFFE708B080BD80B584B003900291DC
:102D2000019202980399019AFDF78EFA04B080BDD2
:102D300080B584B003900291019207F0E7FEFFE7AF
:102D40000198C0B1FFE7FFE7322004F07DFA08B137
:102D5000FFE7F9E70399029802780023184607F085
:102D600051FE0398013003900298013002900198BF
:102D700001380190E4E707F03BFE04B080BD00009D
:102D800080B582B0019001981CF004FF02B080BDB4
:102D900080B582B0ADF80400BDF8040001380146EA
:102DA00000911F2822D80099DFE801F01820202088
:102DB0002020201C20202020202020102020202027
:102DC0002020202020202020202020140A2008F06D
:102DD000FBFE0FE0172008F0F7FE0BE0062008F0DE
:102DE000F3FE07E0092008F0EFFE03E0FF208DF876
:102DF000070003E000208DF80700FFE79DF90700BA
:102E000002B080BD80B582B0ADF80400BDF804000A
:102E10000138014600911F2822D80099DFE801F00F
:102E2000182020202020201C2020202020202010BE
:102E3000202020202020202020202020202020149E
:102E40000A2008F0D9FE0FE0172008F0D5FE0BE0AD
:102E5000062008F0D1FE07E0092008F0CDFE03E0CF
:102E6000FF208DF8070003E000208DF80700FFE742
:102E70009DF9070002B080BD83B0ADF80800019154
:102E8000019820B9FFE7FE208DF80B0025E0002017
:102E90008DF80300FFE79DF803000F2819DCFFE71A
:102EA000BDF808009DF80310C840C00750B1FFE707
:102EB00001989DF8032040F27C31C2F2000141F8F4
:102EC000220006E0FFE79DF8030001308DF80300C3
:102ED000E1E700208DF80B00FFE79DF90B0003B040
:102EE0007047000080B588B008200490012005904C
:102EF00000200690079041F2B460C2F2000004A9DD
:102F000004F058FE18B1FFE703F0EEFEFFE741F2D0
:102F1000B460C2F20000019005F086FA0198052124
:102F200005F0ECF9019804F0A5FF03909DED030A6C
:102F3000B8EE400A40F2EC20C2F2000090ED001A18
:102F400020EE010A9FED041A20EE010A8DED020A1F
:102F50009DED020A08B080BD5D74214180B588B046
:102F6000102004900120059000200690079041F267
:102F70006C60C2F2000004A904F01CFE18B1FFE767
:102F800003F0B2FEFFE741F26C60C2F20000019074
:102F900005F04AFA0198052105F0B0F9019804F00E
:102FA00069FF03909DED030AB8EE400A40F2EC2061
:102FB000C2F2000090ED001A20EE010A8DED020A27
:102FC0009DED020A9FED061A30EE010A9FED051AEB
:102FD00020EE010AB3EE091A30EE010A08B080BDF6
:102FE0005C8F42BF0000C84380B588B006AA039238
:102FF000024603988DF81E208DF81D1080ED000A02
:1030000090ED000AB7EE001AB4EE410AF1EE10FAA4
:1030100004DDFFE7FF208DF81F0097E0039890ED97
:10302000000A9FED4C1A20EE010ABDEEC00A10EE18
:10303000100AADF812009DF81E0001460291F0B191
:10304000FFE70298012804D0FFE7029802280BD07E
:1030500020E0BDF8120042F2B811C2F20001096886
:10306000C8630820059015E0BDF8120042F2B811BF
:10307000C2F2000109688863042005900AE0BDF8E7
:10308000120042F2B811C2F2000109684863002040
:103090000590FFE79DF81D000146019140B1FFE753
:1030A0000198012814D0FFE70198022820D049E0B8
:1030B000059942F2B810C2F200000DF0CBFF059A5C
:1030C00042F2B031C2F2000108681043086039E0F2
:1030D000059942F2B810C2F200000EF09DF9059A6F
:1030E00042F2B031C2F2000108689043086029E062
:1030F00042F2B030C2F2000000680599084210D0D8
:10310000FFE7059942F2B810C2F200000EF084F910
:10311000059A42F2B031C2F200010868904308609B
:103120000FE0059942F2B810C2F200000DF092FFD4
:10313000059A42F2B031C2F20001086810430860FB
:10314000FFE7FFE700208DF81F00FFE79DF91F0054
:1031500008B080BD00FF7F4780B582B00190019824
:103160001CF0F4F902B080BD80B586B004A90291CC
:10317000014602988DF8161080ED000A90ED000AC5
:10318000B7EE001AB4EE410AF1EE10FA04DDFFE7E3
:10319000FF208DF817006AE0029890ED000AB5EE66
:1031A000400AF1EE10FA03DAFFE700200490FFE78F
:1031B0009DF816000146019120B1FFE70198012812
:1031C00015D029E0029890ED000A42F2E000C2F228
:1031D0000000006890ED0B1AB8EE411A20EE010ACB
:1031E000BDEEC00A10EE100AADF80E0014E0029811
:1031F00090ED000A42F29800C2F20000006890EDE3
:103200000B1AB8EE411A20EE010ABDEEC00A10EE0C
:10321000100AADF80E00FFE7BDF80E0001281DDB17
:10322000FFE79DF816000146009120B1FFE70098E6
:10323000012809D011E0BDF80E0042F2E001C2F20F
:1032400000010968486308E0BDF80E0042F29801E9
:10325000C2F2000109684863FFE704E09DF8160028
:1032600000F02CF8FFE700208DF81700FFE79DF92C
:10327000170006B080BD000080B582B08DF8070051
:103280009DF807000146009120B1FFE70098012852
:1032900008D00FE042F2E000C2F2000000210DF081
:1032A000D9FE07E042F29800C2F2000000210DF0C2
:1032B000D1FEFFE7002002B080BD000080B584B0E1
:1032C0008DF80F009DF80F000146029120B1FFE735
:1032D0000298012808D00FE042F2E000C2F200009C
:1032E00000210EF099F807E042F29800C2F20000C7
:1032F00000210EF091F8FFE741F20040C4F2020015
:1033000040210022019208F037F8019804B080BDF6
:1033100083B08DF807009DF807000146009120B1A9
:10332000FFE70098012806D00BE042F24000C2F20D
:103330000000029008E041F6E870C2F2000002903E
:1033400002E000200290FFE7029803B070470000FF
:1033500082B08DF806008DF805100092009820B913
:10336000FFE7FE208DF8070010E000989DF806208A
:1033700040F24041C2F2000101EB42119DF80520EC
:1033800041F8220000208DF80700FFE79DF90700B3
:1033900002B0704783B08DF807009DF80700014622
:1033A000009140B1FFE7009801280AD0FFE700989C
:1033B00002280CD011E042F2D420C2F200000290A8
:1033C0000EE042F29020C2F20000029008E042F2C9
:1033D0001830C2F20000029002E000200290FFE7E5
:1033E000029803B07047000080B582B00190019848
:1033F00000680068C00600282AD5FFE7FFE7002024
:10340000009001980068006800900198006840688A
:1034100000900098FFE7019816F004F800EBC00157
:1034200040F2C040C2F2000000EB8100006A70B1BF
:10343000FFE7019815F0F6FF00EBC00140F2C04035
:10344000C2F2000000EB8100006A8047FFE7FFE75F
:1034500002B080BD82B08DF806008DF80510009294
:10346000009820B9FFE7FE208DF8070012E00098D1
:103470009DF8061001EBC10240F2C041C2F200010A
:1034800001EB82019DF8052041F8220000208DF813
:103490000700FFE79DF9070002B0704783B080B5D1
:1034A00085B009930892079103900020ADF80600BB
:1034B00007A80290039A029B49F20420C2F200007E
:1034C00040F2FF311EF0B0FEADF80600BDF8060078
:1034D00001280CDBFFE7BDF8061049F20420C2F218
:1034E000000000F02FF800208DF8130003E0FE200C
:1034F0008DF81300FFE79DF9130005B0BDE880408B
:1035000003B0704749F28410C2F20000007870479F
:1035100080B582B00090009820B9FFE7FE208DF8BA
:1035200007000BE0009841F2E011C2F200010860D0
:1035300000F068FC00208DF80700FFE79DF9070008
:1035400002B080BD80B582B00190ADF802100020BD
:103550008DF80100FFE70198BDF8021000F078FC3B
:1035600048B1FFE79DF8010001308DF801000A2005
:10357000FFF766FB00E005E0FFE79DF80100032888
:10358000E9DBFFE7002002B080BD0000FFE7FEE7B7
:1035900080B541F2FC60C2F2000005F069FC80BD1C
:1035A00080B541F2FC60C2F2000005F061FC80BD14
:1035B00080B541F22470C2F2000005F059FC80BDD4
:1035C00080B541F22470C2F2000005F051FC80BDCC
:1035D00080B582B000200190FFF7EEFA019942F623
:1035E0005412C2F20002009202F11C0305F036FBF5
:1035F0000099019B41F2E410C2F200000068D0F88B
:10360000C8001A461AF01EFB02B080BD80B582B019
:1036100001200090FFF7D0FA009942F67812C2F22A
:103620000002019202F11C0305F018FB019941F21E
:10363000E410C2F200000068D0F8C80000231A4667
:103640001AF000FB02B080BD83B0029001918DEDB5
:10365000000A02990020087100980199086003B0DF
:103660007047000080B588B0079006910798006801
:1036700005909DED050A9FED181A20EE010ABDEE9A
:10368000C00A10EE100AADF8120042F69C11C2F208
:10369000000101914FF404700860002003908860DD
:1036A000C860082008619DF81320084600F8182F0C
:1036B0000290BDF8120048760698D0F8B400C078A1
:1036C000FFF77AFA0199029A069BC43305F004F8D1
:1036D000039808B080BD00BF0000C84282B00190CE
:1036E00000910098008800EE100AB8EEC00A9FED25
:1036F000151A80EE010A019880ED000A00984088B2
:1037000000EE100AB8EEC00A80EE010A019880EDC2
:10371000010A0098808800EE100AB8EEC00A80EE18
:10372000010A019880ED020A0098C08800EE100A94
:10373000B8EEC00A80EE010A019880ED030A02B0DB
:10374000704700BF0000C84283B00190009101980B
:1037500020B9FFE700208DF80B000AE0019800680F
:1037600000990840401AB0FA80F040098DF80B002B
:10377000FFE79DF80B0003B07047000083B0019095
:103780000091019820B9FFE7FE208DF80B0008E0BA
:10379000009A019908689043086000208DF80B009A
:1037A000FFE79DF90B0003B07047000082B0009066
:1037B0000098006846F60001C4F20001884204D176
:1037C000FFE701208DF8070010E00098006846F23E
:1037D0000041C4F20001884204D1FFE700208DF8C7
:1037E000070003E003208DF80700FFE79DF80700BE
:1037F00002B0704780B592B010900F91109820B928
:10380000FFE7FE208DF847007DE042F29930C2F2DA
:1038100000000078C00720B1FFE7FD208DF84700C9
:1038200071E01AF0D1FB42F6A071C2F2000108600B
:1038300020B9FFE7FE208DF8470064E02020242116
:10384000002204921AF07EF91099C1F8C8000F986E
:103850001099C1F8B40005A802902821FCF70DFDCD
:1038600004980A90059006900B90012103910C9109
:10387000079008900D910E2101910E910990FFF78C
:103880009BF9029905F04CF80498FFF795F906F0BA
:10389000F9F8049843F2D152C0F600020621FFF76E
:1038A000ABF90498FFF788F9022104F0D9FE0199D9
:1038B00003980A910990FFF77FF9029905F030F813
:1038C0000398FFF779F906F0DDF8039843F20D62EB
:1038D000C0F600020821FFF78FF90398FFF76CF993
:1038E000102104F0BDFE03990498109A41F2E413EC
:1038F000C2F200031A6042F29932C2F20002117061
:103900008DF84700FFE79DF9470012B080BD000029
:1039100080B590B08DF83E000E910D920E9820B9B2
:10392000FFE7FE208DF83F0013E19DF83E000146C1
:10393000079158B1FFE707980138022869D3FFE7DC
:10394000079803380228C0F0A980FDE00E9890ED9A
:10395000000A9FED821A20EE010ABDEEC00A10EEA9
:10396000100AADF832000E9890ED010A20EE010A1F
:10397000BDEEC00A10EE100AADF830000E9890EDC2
:10398000020A20EE010ABDEEC00A10EE100AADF8E0
:103990002E000E9890ED030A20EE010ABDEEC00A3B
:1039A00010EE100AADF82C0042F69C11C2F2000194
:1039B00005914FF40070086000208860C8600820FE
:1039C00008619DF83320084600F8182F0690BDF8CE
:1039D000320048769DF831008876BDF83000C87610
:1039E0009DF82F000877BDF82E0048779DF82D0030
:1039F0008877BDF82C00C8770D98D0F8B40000780F
:103A0000FFF7DAF80599069A0D9BB83304F064FEC7
:103A10009BE00E9890ED040A9FED521A20EE010AE9
:103A2000BDEEC00A10EE100AADF82A000E9890ED17
:103A3000050A20EE010ABDEEC00A10EE100AADF82C
:103A4000280042F69C11C2F20001039140F2FF20CF
:103A5000086000208860C86008220A619DF82B3049
:103A60000A4602F8183F0492BDF82A204A769DF8CB
:103A700029208A76BDF82820CA7608774877887783
:103A8000C8770D98D0F8B4004078FFF795F80399FF
:103A9000049A0D9BBC3304F01FFE56E00E9890ED87
:103AA000070A9FED2E1A20EE010ABDEEC00A10EEA5
:103AB000100AADF826000E9890ED080A20EE010AD3
:103AC000BDEEC00A10EE100AADF824000E9890ED7D
:103AD000090A9FED231A20EE010ABDEEC00A10EE7E
:103AE000100AADF8220042F69C11C2F200010191C9
:103AF00040F2FF10086000208860C86008220A6158
:103B00009DF827300A4602F8183F0292BDF8262099
:103B10004A769DF825208A76BDF82420CA769DF83D
:103B200023200A77BDF822204A778877C8770D9836
:103B3000D0F8B4008078FFF73FF80199029A0D9B06
:103B4000C03304F0C9FD00E0FFE700208DF83F001E
:103B5000FFE79DF93F0010B080BD00BF0000804628
:103B600000401C460060EA4683B002900191019833
:103B70000178407840EA0120ADF80200019801790F
:103B8000407940EA0120ADF80000BDF8020000EEE7
:103B9000100AB8EEC00A9FED191A80EE010A9FEDD7
:103BA000181A20EE010A029880ED000A0198817827
:103BB000C07840EA012000B200EE100AB8EEC00A58
:103BC000029880ED010ABDF9000000EB8000800042
:103BD00000EE100AB8EEC00A9FED0A1A80EE010A44
:103BE000029880ED020A0198807900EE100AB8EE82
:103BF000400A029880ED030A03B0704700000046B7
:103C0000DB0FC9400000804680B586B00490039168
:103C1000049820B9FFE7FE208DF8170089E003988B
:103C200020B9FFE7FE208DF8170082E003980068B6
:103C30000190A0F20120042817D3FFE70198A0F219
:103C40000520032828D3FFE70198A0F209200228C5
:103C50003AD3FFE7019840F2112188424CD0FFE7A8
:103C60000198B0F5207F53D05EE003980068A0F281
:103C7000012002900498029900EB0110043003998E
:103C80001C31FFF771FF0299012000FA01F204993B
:103C900008681043086048E003980068A0F2052017
:103CA00002900298811D012000FA01F2049908682F
:103CB000104308600498029900EB011064300399E6
:103CC0001C31FFF751FF30E003980068A0F2092093
:103CD00002900298011D012000FA01F2049908687F
:103CE000104308600498029900EB011044300399D6
:103CF0001C31FFF739FF18E00499086840F40070A0
:103D0000086004989C3003991C31FFF7E7FC0CE035
:103D10000499086840F4806008600498AC30039906
:103D20001C3100F00BF800E0FFE700208DF81700D1
:103D3000FFE79DF9170006B080BD000082B001903A
:103D400000910098017842788078000440EA0220CF
:103D5000084400EE100AB8EEC00A9FED0A1A80EE81
:103D6000010A019880ED000A0098C0780199087155
:103D700000990879497940EA01200199C88002B088
:103D8000704700BF00007A4484B08DF80F000291A4
:103D9000ADF806209DF80F000146009123281DD89C
:103DA0000099DFE801F012131415161B1B1B1B1BD7
:103DB0001B1B1B1B1B1B1B1B1B1B1B1B1B1B1B1B53
:103DC0001B1B1B1B1B1B1718191A08E007E006E03A
:103DD00005E004E003E002E001E000E0FFE700208E
:103DE00004B070470020704780B541F29C30C2F2A9
:103DF000000049F28411C2F2000116F041FC0020DB
:103E000080BD000080B541F29C30C2F2000016F087
:103E1000F1FB002080BD000080B582B001900091D0
:103E200041F2E010C2F200000068012119F0ECFF3D
:103E3000002002B080BD000083B0029001918DF897
:103E4000032000208DF802009DF9020003B07047A6
:103E500080B586B00490ADF80E1000208DF80D00EE
:103E600041F29C30C2F20000D0F8BC0202900298ED
:103E7000D0F8140220B1FFE701208DF8170013E0FD
:103E80000499BDF80E2041F29C30C2F2000001906E
:103E900016F010FC019816F0FBFC8DF80D009DF853
:103EA0000D008DF81700FFE79DF8170006B080BDE4
:103EB00080B588B0069005918DF8132005989DF87F
:103EC000131000F08DF88DF8120005989DF813106E
:103ED00000F078F88DF811009DF8120010280DD12F
:103EE000FFE70698007F00F001008DF810000598AC
:103EF000807A00F001008DF80F0025E09DF8120097
:103F000011280DD1FFE70698407F00F001008DF8E1
:103F100010000598C07A00F001008DF80F0012E043
:103F20000698C08B9DF81210C84000F001008DF873
:103F30001000059840889DF81210C84000F001005C
:103F40008DF80F00FFE7FFE79DF811000146029191
:103F500040B1FFE70298012817D0FFE70298022836
:103F600024D02AE09DF810100020C907019031B13B
:103F7000FFE79DF80F0080F001000190FFE7019836
:103F800000F001008DF81F0017E09DF810100020D0
:103F9000C907009021B9FFE79DF80F000090FFE7E7
:103FA000009800F001008DF81F0006E09DF8100059
:103FB00000F001008DF81F00FFE79DF81F0008B01A
:103FC00080BD000082B001908DF803100198006957
:103FD0009DF8031000EB4100007A02B0704700002A
:103FE00082B001908DF80310019800699DF80310CC
:103FF00000EB4100407A02B07047000081B00090B1
:104000000098407800F0010001B0704783B0019043
:104010000091019820B9FFE7FF208DF80B000FE019
:10402000009820B9FFE7FF208DF80B0008E0019908
:10403000002008700099019A11618DF80B00FFE7CC
:104040009DF90B0003B0704783B001908DF8031009
:104050009DF80300102807D1FFE70198007F00F0CA
:1040600001008DF80B0015E09DF80300112807D121
:10407000FFE70198407F00F001008DF80B0009E098
:104080000198C08B9DF80310C84000F001008DF826
:104090000B00FFE79DF80B0003B0704784B002905F
:1040A00001918DED000A029820B9FFE7FF208DF8FD
:1040B0000F0025E0019820B9FFE7FF208DF80F00E1
:1040C0001EE0029800680199886202984068019990
:1040D000C8620298007EC00748B1FFE7019902203C
:1040E00081F834000199012081F8360004E001993B
:1040F000012081F83400FFE700208DF80F00FFE772
:104100009DF90F0004B0704780B584B00290019112
:104110008DED000A029820B9FFE7FF208DF80F000F
:1041200056E0019820B9FFE7FF208DF80F004FE01F
:1041300002980421FFF788FF80B1FFE7029805216C
:10414000FFF782FF50B1FFE702980621FFF77CFFDF
:1041500020B1FFE7019901200870FFE702980421D0
:10416000FFF772FF80B1FFE702980521FFF76CFFB0
:1041700050B1FFE702980721FFF766FF20B1FFE784
:10418000019900200870FFE70298407D20B1FFE709
:104190000298007D20B9FFE7019800F023FA13E0B0
:1041A00001980078C00738B1FFE7029801999DEDAA
:1041B000000A00F011F806E0029801999DED000A4E
:1041C00000F08CF9FFE7FFE700208DF80F00FFE714
:1041D0009DF90F0004B080BD80B584B003900291BA
:1041E0008DED010A0299012081F824000398B0F9AD
:1041F000160000EE100AB8EEC00A9DED011A20EE7E
:10420000010A0298016991ED001A20EE010A80ED81
:104210000A0A0398B0F91800404200EE100AB8EEFE
:10422000C00A9DED011A20EE010A0298016991ED84
:10423000001A20EE010A80ED0B0A02980022C261EA
:1042400002988261029880F8382003980299FFF75B
:104250002FFE58B1FFE70298016991ED091A90ED20
:10426000070A30EE010A80ED070AFFE7039802997A
:104270000122FFF71DFE58B1FFE70298016991ED99
:10428000091A90ED070A30EE410A80ED070AFFE7B0
:10429000039802990222FFF70BFE58B1FFE702983C
:1042A000016991ED091A90ED060A30EE410A80EDA0
:1042B000060AFFE7039802990322FFF7F9FD58B1B8
:1042C000FFE70298016991ED091A90ED060A30EEB8
:1042D000010A80ED060AFFE7039802990422FFF71E
:1042E000E7FDA8B1FFE70298016991ED0A1A90ED88
:1042F000060A20EE010A80ED060A0298016991ED96
:104300000A1A90ED070A20EE010A80ED070AFFE77E
:10431000039802990522FFF7CBFDA8B1FFE70298A9
:10432000016991ED0B1A90ED060A20EE010A80ED6D
:10433000060A0298016991ED0B1A90ED070A20EE2A
:10434000010A80ED070AFFE7039802990622FFF7AA
:10435000AFFD48B1FFE70299022081F834000299CD
:10436000012081F8360008E00299022081F834002B
:104370000299002081F83600FFE70398029907228E
:10438000FFF796FDB0B1FFE7029991F835000130D3
:1043900081F83500029991F835004AF6AB22CAF649
:1043A000AA22A0FB0232520802EB4202801A81F8D4
:1043B0003500FFE7039802990B22FFF779FD38B12A
:1043C000FFE7029904200875029902204875FFE76B
:1043D000039802990A22FFF76BFD40B1FFE70299AB
:1043E00091F837200120904381F83700FFE70398C8
:1043F00002990822FFF75CFD20B3FFE70298007BDB
:1044000002280BD1FFE702983930042100F0F8F8B8
:104410000299002048700299087312E00298007B0C
:10442000012801D1FFE70BE002983930032100F0A9
:10443000E7F8029902200873029901204870FFE70B
:10444000FFE7FFE7039802990922FFF731FDD8B192
:10445000FFE70298007B01280BD1FFE702990020BB
:1044600048700299087302983930022100F0C8F8A8
:1044700009E00298012101730298417002983930D5
:1044800000F0BEF8FFE703E0029900204870FFE764
:10449000039802990C22FFF70BFD28B1FFE7029960
:1044A000012081F83800FFE7039802990D22FFF7F9
:1044B000FFFC20B1FFE7029902200875FFE703988F
:1044C000C08B029948800299039AD2F81600D2F85C
:1044D0001A208A60486004B080BD000085B0049056
:1044E00003918DED020A0498407D01460191032855
:1044F00017D80199DFE801F011020A06039901209B
:1045000008750EE00399022008750AE0039904205B
:10451000087503990020487503E003990020087589
:10452000FFE70498007D01460091032831D80099E7
:10453000DFE801F02702170A0399012081F824001F
:10454000039981F8340024E00399012081F82400C4
:104550000399002081F836000399022081F8340085
:1045600017E00399012081F82400039A022182F8C0
:104570003410039A002182F83510039981F836002F
:1045800007E00399002081F82400039981F83400A2
:10459000FFE70498006803998861049840680399CC
:1045A000C861049890ED020A9DED021A20EE010AFE
:1045B0000398016991ED011A20EE010A80ED0A0AC3
:1045C000049890ED030A9DED021A20EE010A03986B
:1045D000016991ED011A20EE010A80ED0B0A05B088
:1045E0007047000081B00090009900200875009984
:1045F00081F82400009981F8340001B07047000070
:1046000083B001908DF80310019820B9FFE7FF20D7
:104610008DF80B001BE00198C078022806DCFFE74C
:104620000198C078B0F1FF3F04DCFFE7FF208DF870
:104630000B000CE09DF803000199CA788854019999
:10464000C8780130C87000208DF80B00FFE79DF995
:104650000B0003B07047000081B0ADF802008DF888
:104660000110BDF802109DF801004840C2B244F6A6
:10467000B010C0F6020030F8120080EA112001B03C
:104680007047000080B584B003900291ADF8062019
:10469000FFE70298411E029158B1FFE7BDF80600FE
:1046A00003994A1C03920978FFF7D6FFADF806007C
:1046B000EFE7BDF8060004B080BD000080B584B00F
:1046C000029001910198012804D8FFE700208DF89D
:1046D0000F001BE00298019902394FF6FF72FFF7B5
:1046E000D1FFADF80200BDF80200029A019901F075
:1046F00001031A4421F00101114431F8021C401A4F
:10470000B0FA80F040098DF80F00FFE79DF80F0028
:1047100004B080BD83B0029001918DF80320FFE7C3
:104720000198411E019178B1FFE79DF803000299BD
:104730004A1C02920978414044F6B030C0F60200AB
:10474000405C8DF80300EBE79DF8030003B0704771
:1047500080B584B0029001910198012804D8FFE748
:1047600000208DF80F0015E0029801990139FF2211
:10477000FFF7D0FF8DF803009DF80300029A01991E
:10478000114411F8011C401AB0FA80F040098DF86C
:104790000F00FFE79DF80F0004B080BD85B002A9AF
:1047A00000910146009880ED010AC0ED000A8DF8E5
:1047B000071090ED010AB5EE400AF1EE10FA03D1B0
:1047C000FFE7002004906DE09DF80700C007A0B34C
:1047D000FFE7009890ED010AB2EE0E1AB4EE410A1E
:1047E000F1EE10FA06D1FFE74FF20000C4F291504B
:1047F000049057E0009890ED010AB3EE021AB4EE6F
:10480000410AF1EE10FA06D1FFE748F20000C4F2C7
:10481000A250049046E0009890ED010AB3EE0E1A03
:10482000B4EE410AF1EE10FA06D1FFE74BF20000B8
:10483000C4F2E550049035E022E0009890ED010AC2
:10484000B2EE041AB4EE410AF1EE10FA06D1FFE717
:1048500041F20000C4F28B50049023E0009890EDE8
:10486000010AB3EE001AB4EE410AF1EE10FA06D1D5
:10487000FFE744F20000C4F2B550049012E0FFE7F5
:10488000009890ED010A9FED0A1A20EE010A90EDC2
:10489000001A9FED082A21EE021A80EE010A80ED2F
:1048A000020AFFE7009890ED020A05B0704700BFCA
:1048B00000007042DB0FC94080B584B003900291C4
:1048C000019202980078012805D0FFE702988068DD
:1048D000019908600CE0029890ED010AD0ED020AFF
:1048E00090ED031A0FF03EFD019880ED000AFFE7FE
:1048F0000399012008710398D0ED020A90ED030A94
:10490000B2EE081A00F0BAF8039880ED000A04B07D
:1049100080BD000082B0019000910198006800996C
:104920000860019800790099087102B07047000092
:1049300084B08DED030A9DED030A20EE000A8DED93
:10494000010A9DED010A9DED031A20EE010A8DED8D
:10495000000A9DED030A9FED3E1AB4EE410AF1EE06
:1049600010FA03DAFFE70020029053E09DED030AFE
:104970009FED381AB4EE410AF1EE10FA1DDAFFE7A6
:104980009DED000A9FED391A20EE010A9DED011AF6
:104990009FED372A21EE021A30EE010A9DED031A2F
:1049A0009FED342A21EE021A30EE010A9FED321AF1
:1049B00030EE010A8DED020A2BE09DED030A9FED1A
:1049C000261AB4EE410AF1EE10FA1DDAFFE79DED6A
:1049D000000A9FED221A20EE010A9DED011A9FEDBB
:1049E000202A21EE021A30EE010A9DED031A9FEDF6
:1049F0001D2A21EE021A30EE010A9FED1B1A30EE3D
:104A0000010A8DED020A03E04FF07E500290FFE7AD
:104A1000FFE7FFE79DED020AB5EE400AF1EE10FA5E
:104A200003DAFFE7002002900EE09DED020AB7EEE8
:104A3000001AB4EE410AF1EE10FA04DDFFE74FF080
:104A40007E500290FFE7FFE79DED020A04B0704739
:104A500000009C413333AF410000CC4161E0B93CE0
:104A600046B6D3BF295C21423333A4C31399B93B63
:104A7000FB5CADBEE17AD84014AE34C284B08DED9B
:104A8000030ACDED020A8DED011A9DED030A9DED9D
:104A9000012A30EE420A9DED021A31EE421A80EEF2
:104AA000010A8DED000A9DED000AB5EE400AF1EE17
:104AB00010FA03DAFFE7002000900EE09DED000AF7
:104AC000B7EE001AB4EE410AF1EE10FA04DDFFE78A
:104AD0004FF07E500090FFE7FFE79DED000A04B025
:104AE000704700000000000080B588B08DED070A17
:104AF000CDED060A05909DED050AB8EE400A10EED0
:104B0000100AFBF747FD41EC100B9FED2B1B53ECFC
:104B1000112B51EC100BFBF79BFC41EC100B51ECF3
:104B2000100BFBF74AFD00EE100A1EF0C5F99FEDD1
:104B3000261A20EE010A10EE100AFBF72BFD41ECBD
:104B4000100B51EC100B9FED1E0B52EC103BD20FD3
:104B500062F3DF7141EC100B8DED020B0798FBF750
:104B600019FD9DED021B41EC100B51EC110B53ECA8
:104B7000102BFBF7C6FB41EC100B51EC100BFBF7B5
:104B80001CFD04909DED040A9FED101AB4EE410A3D
:104B9000F1EE10FA05DDFFE79DED060A8DED010A45
:104BA00004E09DED040A8DED010AFFE79DED010A89
:104BB00008B080BD00BF00BFFCA9F1D24D62503FDC
:104BC0000000000000000000CDCC4C3ECDCC4C3F9E
:104BD00080B58EB007AB05930C900B910A920C98A0
:104BE00020B9FFE7FE208DF8370067E10B9820B968
:104BF000FFE7FE208DF8370060E10A990C98026803
:104C0000891A00EE101AB8EE400A9FEDAE1A80EE37
:104C1000010A80ED010A0A980C9908600C980B991A
:104C200009780A9A00F02EFB0C98007C014604914A
:104C300000B3FFE7049801280DD0FFE7049802387D
:104C4000032817D3FFE7049805280AD0FFE7049844
:104C500006280FD04CE00C99002048610C9988611F
:104C600046E00B9840680C9948610B9840680C9995
:104C700088613DE005980C9991ED080AC96891EDAD
:104C8000001A30EE410A80ED020A90ED020A1DF092
:104C9000CFFF059880ED010A90ED020A1EF00CF995
:104CA000059880ED000A90ED010A0B9991ED011A2B
:104CB00091ED022A20EE010A90ED001A21EE021A6F
:104CC00030EE410A0C9981ED050A90ED000A0B992E
:104CD00091ED011A91ED022A20EE010A90ED011AE0
:104CE00021EE021A30EE010A0C9880ED060AFFE769
:104CF0000C98007C01460391062848D80399DFE808
:104D000001F00404081A300408000C990020C8615E
:104D10003DE00C9901F13800CA6892ED000AD1ED2E
:104D2000011AD1ED080A9FED6B1A0FF07FF80C986D
:104D300080ED070A2BE00C9901F13800CA6892ED6A
:104D4000000A9FED631A30EE010AD1ED011AD1ED90
:104D5000080A9FED601A0FF069F80C9880ED070AB9
:104D600015E00C9890ED0B0A8DED020A0A989FED64
:104D7000560ADFED560AFFF7B7FEB0EE401A9DED7A
:104D8000020A20EE010A0C9880ED070AFFE70C9B4F
:104D900003F1120003F114011A6B93F911309FED26
:104DA0004E0A0EF0C7FC00208DF81B00FFE79DF8AF
:104DB0001B000C9991F9111088427BDAFFE70C98DF
:104DC000416A406F9DF81B2000EB421001EB82010D
:104DD00091ED000A0DF01AFC0C98406A9DF81B102A
:104DE00000EB810080ED000A0C98007C01460191E7
:104DF000E0B3FFE701980138052804D3FFE70198E5
:104E0000062821D03AE00C99486B9DF81B30C3EB83
:104E1000031200EB82000A6B02EB830292ED000AA0
:104E20004A6A02EB8302D2ED000AD1ED011A9FED2E
:104E3000291A0EF0FBFF0C98C06F9DF81B1000EBB9
:104E4000810080ED000A19E00C989DF81B10026BA0
:104E5000C06F02EB810292ED000A9FED201A80EEF6
:104E6000010A00EB810080ED000A07E00C98C16F99
:104E70009DF81B20002041F82200FFE70C999DF8C7
:104E80001B20886FC96F00EB421001EB820191ED8E
:104E9000000A0DF0BBFB0C98C06F9DF81B1000EBD7
:104EA000810080ED000AFFE79DF81B0001308DF8BE
:104EB0001B007CE700208DF83700FFE79DF93700E5
:104EC0000EB080BD00007A449A99193FCDCC4C3F7A
:104ED000AB611C3F0000000000C0DA4500A00C469A
:104EE00083B00290019100208DF80300FFE79DF848
:104EF0000300029991F91110884210DAFFE7029835
:104F0000C06F9DF8032050F82200019941F822005B
:104F1000FFE79DF8030001308DF80300E7E703B0D9
:104F20007047000082B0019000910198007C0099C8
:104F30000870019890ED080AC06890ED001A30EEF4
:104F4000410A009880ED010A02B0704780B58AB02E
:104F500005AB03930346039808930791069280EDEF
:104F6000000A089820B9FFE7FE208DF827001CE111
:104F7000079808998860089900200874069808998D
:104F8000C860079890F84C00C00728B1FFE7089860
:104F9000C06800F0DBFAFFE70898806800780146F7
:104FA0000291062832D80299DFE801F0040B1218AA
:104FB0001F2C250008990420487400208DF8130048
:104FC00024E008990420487401208DF813001DE0A6
:104FD0000899022048748DF8130017E008990420FE
:104FE000487403208DF8130010E0089904204874D9
:104FF0008DF813000AE008990120487405208DF807
:10500000130003E0FC208DF82700CEE0089890F90B
:1050100011008000FEF7A0F8089948620898406ADD
:1050200008B9FFE7A5E0089890F911008000FEF7A5
:1050300093F8089988620898806A08B9FFE798E0B1
:10504000089890F911008000FEF786F80899086327
:105050000898006B08B9FFE78BE0089890F91100F9
:10506000C0EB00108000FEF777F8089948630898B5
:10507000406B08B9FFE77CE0089890F911008000C8
:10508000FEF76AF80899C8670898C06F08B9FFE783
:105090006FE0089890F911004001FEF75DF808995B
:1050A00048670898406F08B9FFE762E0089890F9F0
:1050B00011004001FEF750F8089988670898806F42
:1050C00008B9FFE755E000208DF81200FFE79DF8D2
:1050D0001200089991F91110884233DAFFE7039A18
:1050E00008988168406B9DF81230C3EB031300EB06
:1050F000830092ED000A0A1D00210FF00FF8039AB9
:1051000008988168406F9DF8123000EB431092EDD3
:10511000000AD1ED110A0DF0D5FA039A08988168BA
:10512000806F9DF8123000EB431092ED000AD1ED34
:10513000120A0DF0C7FAFFE79DF8120001308DF852
:105140001200C4E7039A089901F1380092ED000AB1
:10515000896801F12402002101910EF0DFFF089817
:1051600012309DF813100EF037FC01988DF82700CF
:105170001BE00898406AFDF703FE0898006BFDF7F6
:10518000FFFD0898406BFDF7FBFD0898C06FFDF729
:10519000F7FD0898406FFDF7F3FD0898806FFDF765
:1051A000EFFDFE208DF82700FFE79DF927000AB0EC
:1051B00080BD000080B584B0039002910192002070
:1051C000009001980078012805D0FFE70020C4F284
:1051D000FA40009042E002980079012833D1FFE7BD
:1051E000029890ED000A9FED231AB4EE410AF1EE09
:1051F00010FA28DDFFE7029890ED000AB7EE001ADA
:10520000B4EE410AF1EE10FA05DDFFE70020CBF61F
:105210008070009016E0019890ED010A029890EDE0
:10522000001A9FED152A31EE021A9FED142A81EE25
:10523000021A9FED132A21EE021A30EE010A8DEDBB
:10524000000AFFE709E0019890ED010AD0ED020A9B
:105250000FF038F98DED000AFFE7FFE79DED000A3A
:10526000039A516AD06F92F911200FF0B7F800201D
:1052700004B080BD9A99993E9A9999BE3333333FD1
:105280000000C84280B586B004908DF80F100292DD
:10529000049820B9FFE7FE208DF8170066E09DF81E
:1052A0000F000499097C884204D1FFE700208DF8A3
:1052B00017005BE09DF80F0004281CD1FFE704985D
:1052C000007C042817D0FFE70298FAF7B5FFFAF739
:1052D000A9FF00EBD07121F00101411A0120002942
:1052E00018BF4FF0FF3000EE100AB8EEC00A049865
:1052F00080ED0B0AFFE700208DF80700FFE79DF81F
:105300000700049991F91110884227DAFFE7049801
:10531000406B9DF80710C1EB011100EB81000EF00E
:10532000C9FF0498406F9DF8071000EB41109FEDF6
:10533000110A8DED000A0DF063FA9DED000A049844
:10534000806F9DF8071000EB41100DF059FAFFE750
:105350009DF8070001308DF80700D0E79DF80F0099
:105360000499087400208DF81700FFE79DF91700D5
:1053700006B080BD0000000084B002900191029848
:1053800020B9FFE7FE208DF80F0048E0019820B912
:10539000FFE7FE208DF80F0041E00298806890F84A
:1053A0004C00C00758B1FFE7019890ED111A9FED2E
:1053B0001E0A30EE410A029880ED080A04E00198C6
:1053C000406C02990862FFE700208DF80300FFE7B8
:1053D0009DF80300029991F9111088421BDAFFE74A
:1053E00001989DF8032000EB021080680299496A39
:1053F00041F8220001989DF8032000EB0210C068DC
:105400000299896A41F82200FFE79DF80300013004
:105410008DF80300DCE700208DF80F00FFE79DF911
:105420000F0004B0704700BFDB0FC94084B0039089
:105430008DED020ACDED010A039890ED000A9DED75
:10544000021A30EE010A8DED000A9DED010AB5EE5B
:10545000400AF1EE10FA26DDFFE79DED000A9DED12
:10546000011AB4EE410AF1EE10FA09DBFFE79DEDF7
:10547000011A9DED000A30EE410A8DED000A11E09F
:105480009DED000AB5EE400AF1EE10FA09DAFFE7E9
:105490009DED011A9DED000A30EE010A8DED000A26
:1054A000FFE7FFE7FFE700980399086004B0704743
:1054B00085B08DED040ACDED030A8DED021A9DED48
:1054C000040A9DED031A30EE410A8DED010A9DEDAF
:1054D000020AB5EE400AF1EE10FA32DDFFE79DED6B
:1054E000020AB0EE001A80EE010A8DED000A9DED71
:1054F000010A9DED001AB4EE410AF1EE10FA09DD41
:10550000FFE79DED021A9DED010A30EE410A8DED97
:10551000010A15E09DED010A9DED001AB1EE411A58
:10552000B4EE410AF1EE10FA09DAFFE79DED021A36
:105530009DED010A30EE010A8DED010AFFE7FFE75C
:10554000FFE79DED010A05B07047000081B00090B3
:10555000009890ED001A9FED040A30EE410A80EDAC
:10556000000A01B0704700BFDB0FC94083B0029052
:105570008DED010ACDED000A029890ED000A9DED37
:10558000001AB4EE410AF1EE10FA04DDFFE70098CC
:1055900002990860FFE7029890ED000A9DED011A5C
:1055A000B4EE410AF1EE10FA04DAFFE7019802992D
:1055B0000860FFE703B0704780B5B4B03290319116
:1055C0003092329818B9FFE700203390FDE131980E
:1055D000013831900020ADF84E0040F26030C2F248
:1055E0000000007801461291072800F2C881129944
:1055F000DFE811F008001A002C0097003601610165
:10560000A301B4013298319945F60432C0F6020282
:105610001CF0DCFD40F26031C2F20001087801307C
:10562000087001203390D0E13298319945F632224A
:10563000C0F602021CF0CAFD40F26031C2F2000165
:1056400008780130087001203390BEE142F6E45042
:10565000C2F200001190C06818F0A6FD1198806B8E
:1056600014A90022052318F00DFAC0B1FFE7329803
:10567000319945F60422C0F602021CF0A7FD40F263
:105680006031C2F200010720087042F6E450C2F215
:105690000000C06818F068FD0120339095E142F6E3
:1056A000E450C2F20000C06818F05EFD14A8FCF7D8
:1056B00025FF90B1FFE73298319945F6DA22C0F61E
:1056C00002021CF083FD40F26031C2F20001087852
:1056D000013008700120339077E140F26130C2F26E
:1056E0000000017801310170007802280FDCFFE72B
:1056F0003298319945F65022C0F602021CF066FD40
:1057000040F26031C2F200010120087006E040F270
:105710006031C2F2000107200870FFE701203390DA
:1057200053E13298319945F62532C0F602021CF059
:105730004DFD17A8109000F01BFF10980021299133
:105740002A912B9100F0D2FFFFE7BDF84E00B0F593
:105750007A7F4BDAFFE742F6E450C2F20000806B3A
:1057600014A90F910022052318F08CF901460F9817
:10577000B1FA81F149098DF84D10FCF7BFFE8DF8A3
:105780004C009DF84D00C00778B3FFE79DF84C0032
:10579000C00750B3FFE79DED141A40F26430C2F227
:1057A000000090ED000A30EE010A80ED000A9DED48
:1057B000151A40F26830C2F2000090ED000A30EE97
:1057C000010A80ED000A9DED161A40F26C30C2F21B
:1057D000000090ED000A30EE010A80ED000ABDF8ED
:1057E0004E000130ADF84E00FFE7AEE7BDF84E00C9
:1057F00000EE100AB8EE401A40F26430C2F2000027
:1058000090ED000A80EE010A80ED000ABDF84E001E
:1058100000EE100AB8EE401A40F26830C2F2000002
:1058200090ED000A80EE010A80ED000ABDF84E00FE
:1058300000EE100AB8EE401A40F26C30C2F20000DE
:1058400090ED000A80EE010A80ED000A40F260311E
:10585000C2F2000108780130087001203390B4E0F2
:105860003298319945F6AC22C0F602021CF0AEFC2B
:1058700017A80E9000F07CFE0E9840F26431C2F240
:1058800000010968299140F26831C2F200010968FB
:105890002A9140F26C31C2F2000109682B9100F0AC
:1058A00025FF40F26031C2F2000108780130087033
:1058B0000120339089E032980C9031980D9040F29D
:1058C0006430C2F200000068FAF764FE41EC100B8D
:1058D0008DED0A0B40F26830C2F200000068FAF762
:1058E00059FE41EC100B8DED080B40F26C30C2F20A
:1058F00000000068FAF74EFE9DED081B9DED0A0BB7
:1059000002460C980B460D9943EC122B6A4682ED29
:10591000042B82ED021B82ED000B45F66832C0F6C7
:1059200002021CF053FC40F26031C2F20001087820
:10593000013008700120339047E03298319945F6E4
:105940009922C0F602021CF041FC40F26031C2F222
:105950000001082008700120339036E03298319918
:1059600045F61D22C0F602021CF030FC40F2603108
:10597000C2F20001082008700120339025E040F2B7
:105980006431C2F2000100200790086040F26831E3
:10599000C2F20001086040F26C31C2F200010860FE
:1059A00040F26131C2F2000108703298319945F637
:1059B0003842C0F602021CF009FC079840F2603140
:1059C000C2F2000108703390FFE7339834B080BD15
:1059D00080B5B0B02E902D912C922E9818B9FFE77B
:1059E00000202F9060E22D9801382D902C980121F5
:1059F0002BAA01F081FC28902C9802212AAA01F000
:105A00007BFC27902C98032129AA01F075FC269095
:105A100028982B9A45F25B31C0F60201FAF762FC36
:105A2000A0B9FFE72E982D9945F68452C0F60202E0
:105A300045F20B63C0F602031CF0C8FB40F2703164
:105A4000C2F20001002008702F902DE228982B9AB6
:105A500045F6A251C0F60201FAF744FC00285BD1DA
:105A6000FFE7279818B9FFE7269808B1FFE70BE290
:105A700040F27030C2F20000007801460A9120B175
:105A8000FFE70A98012810D045E02E982D9945F699
:105A9000B742C0F602021CF099FB40F27031C2F22C
:105AA0000001012008702F90FEE10DA809906421EB
:105AB000FAF7E3FB45F2F730C0F60200089000F079
:105AC0009DFD189045F2FA30C0F60200069000F0F5
:105AD000D7FD069A014609981791142107911CF0E9
:105AE00075FB0799089A099814301CF06FFB099808
:105AF00000F0FCFD2E982D9945F67342C0F6020287
:105B00001CF064FB40F27031C2F200010220087008
:105B100001202F90C8E19DE128982B9A45F6B351BA
:105B2000C0F60201FAF7DEFB002840F0CF80FFE765
:105B3000279818B1FFE7269808B1FFE7A4E1279856
:105B40002A9A45F6AD51C0F60201FAF7CBFB0028C0
:105B500057D1FFE700F088FD0C9040F27030C2F2A0
:105B6000000000780146059120B1FFE70598012863
:105B700010D045E02E982D9945F62252C0F602022B
:105B80001CF024FB40F27031C2F2000101200870C9
:105B90002F9089E10C9840F27131C2F2000109782E
:105BA00050F83100E0B1FFE72E982D990C9A40F2A1
:105BB0007133C2F2000304931B7852F8333045F678
:105BC0008052C0F602021CF001FB049908780130F3
:105BD000087040F27031C2F20001012008700CE040
:105BE00040F27131C2F200010020087040F27031C1
:105BF000C2F2000102200870FFE701202F9053E15C
:105C000063E027982A9A45F6A751C0F60201FAF7F1
:105C100069FB002857D1FFE700F02CFD0B9040F204
:105C20007030C2F2000000780146039120B1FFE716
:105C30000398012810D045E02E982D9945F6395249
:105C4000C0F602021CF0C2FA40F27031C2F200014A
:105C5000012008702F9027E10B9840F27131C2F2B9
:105C60000001097850F83100E0B1FFE72E982D9936
:105C70000B9A40F27133C2F2000302931B7852F880
:105C8000333045F68052C0F602021CF09FFA0299AA
:105C900008780130087040F27031C2F20001012032
:105CA00008700CE040F27131C2F20001002008706F
:105CB00040F27031C2F2000102200870FFE70120BB
:105CC0002F90F1E000E0DFE0FFE7C2E028982B9A98
:105CD00045F68D51C0F60201FAF704FB002840F0AA
:105CE000B780FFE7279818B1FFE7269808B9FFE7C4
:105CF000CAE027982A9A45F6A751C0F60201FAF79A
:105D0000F1FA00283ED1FFE740F27030C2F2000005
:105D10000078B0BBFFE70DA800F02AFC269800F041
:105D2000AFFC88B9FFE72E982D9945F67B42C0F667
:105D300002021CF04BFA40F27031C2F20001022064
:105D4000087001202F90AFE02E982D9945F63B4228
:105D5000C0F602021CF03AFA269B45F68452C0F6C1
:105D600002020DA8019014211CF030FA019800F0F5
:105D7000BDFC40F27031C2F20001012008702F908A
:105D800092E04BE027982A9A45F6AD51C0F6020101
:105D9000FAF7A8FA00283FD1FFE740F27030C2F2CC
:105DA00000000078B8BBFFE70DA800F0E1FB2698E3
:105DB00000F024FC88B9FFE72E982D9945F60A5289
:105DC000C0F602021CF002FA40F27031C2F2000189
:105DD0000220087001202F9066E02E982D9945F63C
:105DE0003B42C0F602021CF0F1F90DA800901430FD
:105DF000269B45F68452C0F6020214211CF0E6F9F7
:105E0000009800F073FC40F27031C2F200010120F2
:105E100008702F9048E000E036E0FFE740F2703075
:105E2000C2F200000078012811D1FFE72E982D99C9
:105E300045F6DD42C0F602021CF0C8F940F27031AE
:105E4000C2F200010220087001202F902CE0FFE731
:105E5000FFE7FFE7FFE740F27030C2F20000007892
:105E6000022810D1FFE72E982D9945F25632C0F640
:105E700002021CF0ABF940F27031C2F200010020C6
:105E800008702F9010E0FFE72E982D9945F6A51287
:105E9000C0F602021CF09AF940F27031C2F2000121
:105EA000002008702F90FFE72F9830B080BD0000D1
:105EB00080B588B0069005910492069818B9FFE75E
:105EC000002007908DE005980138059042F21120DE
:105ED000ADF80E00BDF80E00ADF80C009DF80E00F8
:105EE0009DF80F1040EA0120ADF80A0040F2723030
:105EF000C2F20000007801460191032861D801999F
:105F0000DFE801F00214283C0698059945F6254281
:105F1000C0F602021CF05AF940F27231C2F20001DE
:105F2000087801300870012007905AE0069805991A
:105F3000BDF80C3045F6F832C0F602021CF046F906
:105F400040F27231C2F2000108780130087001207D
:105F5000079046E006980599BDF80A3045F6CB3221
:105F6000C0F602021CF032F940F27231C2F20001B6
:105F70000878013008700120079032E0BDF80C006D
:105F8000BDF80A10884209D1FFE70698059945F641
:105F9000B332C0F602021CF019F908E00698059920
:105FA00045F6A632C0F602021CF010F9FFE740F2F7
:105FB0007231C2F2000108780130087001200790A8
:105FC0000FE00698059945F63842C0F602021CF02B
:105FD000FDF840F27231C2F2000100200870079013
:105FE000FFE7079808B080BD80B5DAB058905791A8
:105FF0005692589818B9FFE700205990C9E0579871
:106000000138579040F27330C2F200000078014628
:106010000991042800F2AD800999DFE801F003241A
:10602000778899000AA800F0A3FA58980790579823
:1060300008902298FAF7AEFA024607980B4608999C
:1060400043EC102B6A4682ED000B45F69632C0F603
:1060500002021CF0BBF840F27331C2F200010120D1
:106060000870599095E042F6E450C2F200000690A4
:10607000C06818F099F80698006F23A900220A2337
:1060800017F000FD80B1FFE742F6E450C2F20000D5
:10609000C06818F069F840F27331C2F200010320C1
:1060A00008700120599074E00AA8039000F060FA8B
:1060B00042F6E450C2F20000C06818F055F80398A8
:1060C0003899229100F012FB039800F051FA589889
:1060D0000490579805902298FAF75CFA02460498C3
:1060E0000B46059943EC102B6A4682ED000B45F6F2
:1060F0006642C0F602021CF069F840F27331C2F247
:106100000001022008700120599042E058985799E8
:1061100045F6DD42C0F602021CF058F840F2733139
:10612000C2F20001052008700120599031E0589812
:10613000579945F6D512C0F602021CF047F840F216
:106140007331C2F20001052008700120599020E04F
:106150005898579945F69342C0F602021CF036F85B
:1061600040F27331C2F200010520087001205990FD
:106170000FE05898579945F63842C0F602021CF0D5
:1061800025F840F27331C2F20001002008705990E6
:10619000FFE759985AB080BD80B5E2B060905F913A
:1061A0005E92609818B9FFE700206190C2E05F98A6
:1061B00001385F9040F27430C2F20000007801466E
:1061C000119148B1FFE71198012817D0FFE7119806
:1061D000022800F08E809DE060985F9945F63F327E
:1061E000C0F602021BF0F2FF40F27431C2F200016D
:1061F000087801300870012061909BE012A800F03F
:10620000B7F942F6E450C2F200001090C06817F0EF
:10621000CBFF1098006F2BA90022052317F032FC4A
:10622000C0B1FFE760985F9945F6E912C0F6020237
:106230001BF0CCFF40F27431C2F200010220087062
:1062400042F6E450C2F20000C06817F08DFF012052
:1062500061906FE042F6E450C2F20000C06817F0AF
:1062600083FF3C9827904098289012A800F03EFAAF
:1062700060980E905F980F90279828990691299919
:106280000891FAF787F90246069807920A46079995
:1062900042EC101B8DED0C0BFAF77CF902460898C6
:1062A00009920A46099942EC101B8DED0A0BFAF788
:1062B00071F99DED0A1B9DED0C0B02460E980B46E5
:1062C0000F9943EC122B6A4682ED042B82ED021BE0
:1062D00082ED000B45F64642C0F602021BF076FF47
:1062E00040F27431C2F20001032008700120619075
:1062F00020E060985F9945F61D22C0F602021BF06F
:1063000065FF40F27431C2F20001032008700120E1
:1063100061900FE060985F9945F63842C0F602023E
:106320001BF054FF40F27431C2F2000100200870EB
:106330006190FFE7619862B080BD000080B596B0C3
:10634000149013911292149818B9FFE70020159039
:106350000AE113980138139040F27530C2F2000040
:10636000007801460A91092800F2EE800A99DFE8D8
:1063700001F00517243643557385BCCE1498139A43
:1063800045F20871C0F60201F9F782FF40F275315B
:10639000C2F2000108780130087001201590E3E096
:1063A000149819F0D5FF40F27531C2F20001087857
:1063B0000130087001201590D6E01498139A45F624
:1063C0009701C0F60201F9F763FF40F27531C2F29E
:1063D000000108780130087001201590C4E014987D
:1063E00019F024FF40F27531C2F200010878013043
:1063F000087001201590B7E01498139A45F2977130
:10640000C0F60201F9F744FF40F27531C2F2000113
:1064100008780130087001201590A5E00BA819F04C
:1064200021FC149813990B9AC2F5C04C6B46C3F823
:1064300004C01A6045F68232C0F602024FF4C0432F
:106440001BF0C4FE40F27531C2F200010878013041
:1064500008700120159087E01498139A45F61801EA
:10646000C0F60201F9F714FF40F27531C2F20001E3
:106470000878013008700120159075E01498089094
:106480001398099042F6E450C2F20000D0F8AC1024
:106490000491D0F8B400FAF77DF80246049805920A
:1064A0000A46059942EC101B8DED060BFAF772F8BF
:1064B0009DED060B024608980B46099943EC112BFB
:1064C0006A4682ED021B82ED000B45F68E32C0F665
:1064D00002021BF07BFE40F27531C2F20001087827
:1064E00001300870012015903EE01498139A45F68B
:1064F0002411C0F60201F9F7CBFE40F27531C2F269
:106500000001087801300870012015902CE01498E3
:10651000139942F6E452C2F2000202F1CC03EC46B7
:10652000CCF8003002F1B80345F6C232C0F60202E0
:106530001BF04CFE40F27531C2F2000108780130C8
:106540000870012015900FE01498139945F6384211
:10655000C0F602021BF03AFE40F27531C2F20001B1
:10656000002008701590FFE7159816B080BD000058
:1065700080B582B0019001990020C0F60E0064221F
:10658000FCF7CAFB0198143000F038F80199C86292
:10659000019800F075F8019988620198806A38B90D
:1065A000FFE7019940F28810C2F200008862FFE71D
:1065B0000198C06A38B9FFE7019944F6E800C0F6CF
:1065C0000200C862FFE70198806A013038B9FFE72E
:1065D000019940F28810C2F200008862FFE701983A
:1065E000C06A013038B9FFE7019944F6E800C0F607
:1065F0000200C862FFE702B080BD000080B584B031
:106600000290029818B9FFE70020039029E00020CB
:106610000190FFE7019944F64C60C0F6020050F883
:106620003100D8B1FFE7019944F64C60C0F6020092
:1066300050F831000299F9F73EFE50B9FFE7019991
:1066400044F64C60C0F6020000EBC10040680390C5
:1066500007E0FFE7019801300190DBE7002003909D
:10666000FFE7039804B080BD44F64C60C0F602001A
:106670007047000044F66460C0F6020070470000F6
:1066800080B584B00290029818B9FFE7002003900B
:1066900029E000200190FFE7019944F66460C0F60C
:1066A000020050F83100D8B1FFE7019944F6646068
:1066B000C0F6020050F831000299F9F7FCFD50B91C
:1066C000FFE7019944F66460C0F6020000EBC100E8
:1066D0004068039007E0FFE7019801300190DBE795
:1066E00000200390FFE7039804B080BD80B582B01E
:1066F000019017F039F90B20FCF7EAFA0199002014
:10670000C0F60E006422FCF713FB17F083F902B009
:1067100080BD000080B541F69410C2F2000003F085
:10672000F7FB80BD80B541F2B470C2F2000003F007
:10673000EFFB80BD80B541F25470C2F2000003F05F
:10674000E7FB80BD80B541F6F410C2F2000003F013
:10675000DFFB80BD80B541F61400C2F2000003F0FB
:10676000D7FB80BD80B541F67400C2F2000003F093
:10677000CFFB80BD80B541F6D400C2F2000003F02B
:10678000C7FB80BD80B541F65420C2F2000003F083
:10679000BFFB80BD80B541F63410C2F2000003F0AB
:1067A000B7FB80BD82B001900198007810384AF69E
:1067B000AB21CAF6AA21A0FB0110000900900099A4
:1067C00044F2E860C0F60200405C0199C865009898
:1067D000042807D3FFE701990868042262F309003F
:1067E000886506E00199086840F2FF3290438865A9
:1067F000FFE70198806D02B07047000086B00590F9
:1068000000208DF813000598806A03900598806930
:1068100010BBFFE70398029003281BD80299DFE81A
:1068200001F0020D0218059890F82F00C00720B162
:10683000FFE701208DF81300FFE70CE00598C06A20
:10684000B0F1C07F04D1FFE701208DF81300FFE70E
:1068500001E000E0FFE745E005988069B0F5005FE2
:1068600025D1FFE70398019003281ED80199DFE89E
:1068700001F00206021101208DF8130016E00598C0
:1068800090F82F00C00720B1FFE701208DF813001A
:10689000FFE70BE00598C06AB0F1C07F04D1FFE7C5
:1068A00001208DF81300FFE700E0FFE719E00398EF
:1068B0000090032804D3FFE70098032804D00EE0DB
:1068C00001208DF813000BE0059890F82F00C00709
:1068D00020B1FFE701208DF81300FFE700E0FFE79C
:1068E000FFE7FFE79DF8130006B0704784B0039000
:1068F00002910192009303980168086820F48020B7
:1069000008600098039909684860039880684028E7
:1069100009D1FFE7019803990968886002980399F3
:106920000968C86008E002980399096888600198BE
:1069300003990968C860FFE704B0704782B000900F
:10694000009820B9FFE701208DF8070074E0009857
:1069500000886FF3DF20B0F5B67F09D3FFE700981A
:1069600000886FF3DF2040F29561884204D3FFE78F
:1069700001208DF807005FE000980068C0F3CA208E
:10698000B0F5B67F09D3FFE700980068C0F3CA20CE
:1069900040F29561884204D3FFE701208DF807009B
:1069A0004AE0009881880068800D40EA81206FF3FA
:1069B000DF20B0F5B67F0DD3FFE70098818800682F
:1069C000800D40EA81206FF3DF2040F2956188421C
:1069D00004D3FFE701208DF807002DE000988088A0
:1069E000C0F34A00B0F5B67F09D3FFE7009880886E
:1069F000C0F34A0040F29561884204D3FFE70120CA
:106A00008DF8070018E0009881880020B0EB913FD6
:106A100004D1FFE701208DF807000DE00098808881
:106A2000000B800720B9FFE701208DF8070003E085
:106A300000208DF80700FFE79DF8070002B07047BF
:106A400080B584B002900191029820B9FFE7FE2042
:106A50008DF80F000EE0019820B9FFE7FE208DF8B9
:106A60000F0007E001982421F9F707FC00208DF8BA
:106A70000F00FFE79DF90F0004B080BD80B584B022
:106A80000290029820B9FFE7FE208DF80F002BE05E
:106A900042F29A30C2F200000078C00720B1FFE74E
:106AA000FD208DF80F001FE017F08EFA42F6A4715A
:106AB000C2F20001086020B9FFE7FE208DF80F0048
:106AC00012E046F65542C0F6000200200190032174
:106AD000FCF7C0FC019842F29A32C2F20002012196
:106AE00011708DF80F00FFE79DF90F0004B080BD15
:106AF00080B584B002900191029820B9FFE7FE2092
:106B00008DF80F009FE00298FFF718FF20B1FFE714
:106B1000FF208DF80F0096E001982421F9F7ADFBD6
:106B2000FFE70020C4F2A5400090029800886FF3B0
:106B3000DF2000EE100AB8EE400A9FED451A30EE55
:106B4000410A30EE000A9DED002A80EE020A01980B
:106B500080ED020A02980068C0F3CA2000EE100A15
:106B6000B8EE400A30EE410A30EE000A9DED002AF0
:106B700080EE020A019880ED030A0298818800687D
:106B8000800D40EA81206FF3DF2000EE100AB8EE9E
:106B9000400A30EE410A30EE000A9DED002A80EEF8
:106BA000020A019880ED000A02988088C0F34A002A
:106BB00000EE100AB8EE400A30EE410A30EE000A4C
:106BC0009DED002A80EE020A019880ED010A0298EC
:106BD0008088800B0199487502988088C0F3013045
:106BE000019908750298C0880199C88202980089A5
:106BF0000199088302984089019948830298007B93
:106C0000002818BF0120019908770298407B0028CE
:106C100018BF0120019948770298C0890199C8835B
:106C20000298008A00EE100AB8EE400A30EE410ADF
:106C30009DED001A80EE010A019880ED040A002003
:106C40008DF80F00FFE79DF90F0004B080BD00BF75
:106C50000000804480B542F6A470C2F200000068D3
:106C6000802117F0D1F880BD80B582B0009000205F
:106C7000FCF790FB009912220BF0A8FA20B9FFE76D
:106C800000208DF8070003E0FF208DF80700FFE7E4
:106C90009DF9070002B080BD80B582B00190019AD5
:106CA0008020012117F002F98038B0FA80F0400905
:106CB00002B080BD7047000080B5012003F086FF60
:106CC00080BD000080B5082003F080FF80BD00007B
:106CD00080B5102003F07AFF80BD000080B5202031
:106CE00003F074FF80BD0000FFE700BFFDE7000078
:106CF00080B584B003908DF80B10002001900398AC
:106D000060B3FFE70398012828D0FFE70398022823
:106D100024D0FFE70398032820D0FFE70398042836
:106D20001CD0FFE70398052818D0FFE70398062832
:106D300014D0FFE70398072810D0FFE7039808282E
:106D40000CD0FFE70398092808D0FFE703980A282A
:106D500004D0FFE703980B2801D1FFE708E044F6D1
:106D60006570C0F6020040F2DB3116F06DFCFFE703
:106D70009DF80B0078B1FFE79DF80B0001280AD0C1
:106D8000FFE79DF80B00022805D0FFE79DF80B00F8
:106D9000032801D1FFE708E044F66570C0F6020061
:106DA0004FF4777116F050FCFFE79DF80B0018B90F
:106DB000FFE70020019017E09DF80B00012804D1A7
:106DC000FFE74FF4807001900DE09DF80B00022862
:106DD00004D1FFE74FF40070019003E04FF44070DE
:106DE0000190FFE7FFE7FFE743F61041C4F202011D
:106DF000086820F440700860019A08681043086031
:106E0000086820F0F8000860039A086840EAC200A9
:106E100040F002000860086840F48030086004B068
:106E200080BD000043F60040C4F202000068800507
:106E300000281FD5FFE743F60041C4F202010868AD
:106E400020F400700860FFE743F60041C4F202013D
:106E5000086840F400600860086820F4006008607A
:106E6000FFE743F60041C4F20201086840F40070F5
:106E70000860FFE743F60040C4F2020000684005E6
:106E800000281FD5FFE743F60041C4F2020108685D
:106E900020F480600860FFE743F60041C4F202017D
:106EA000086840F480500860086820F4805008604A
:106EB000FFE743F60041C4F20201086840F4806035
:106EC0000860FFE77047000080B582B08DF80700CA
:106ED00000919DF8070078B1FFE79DF807000128B1
:106EE0000AD0FFE79DF80700022805D0FFE79DF8CC
:106EF0000700032801D1FFE708E044F66570C0F6FB
:106F000002004FF46F7116F09FFBFFE70098012815
:106F100001D1FFE708E044F66570C0F6020040F2D8
:106F2000BD3116F091FBFFE743F61041C4F20201B8
:106F3000086820F440700860086840F004000860A9
:106F40009DF80720086840EA022040F4803008607D
:106F500002B080BD80B582B001908DF80310019819
:106F6000B0F1006F05D3FFE70198B0F1016F10D3C6
:106F7000FFE7019847F60001C1F6FF71884209D387
:106F8000FFE7019847F60F21C1F6FF71884201D84B
:106F9000FFE708E044F62B70C0F6020040F2BB2188
:106FA00016F052FBFFE743F61041C4F202010868F5
:106FB00020F44070086008680860086840F001002C
:106FC00008609DF803000199087002B080BD0000C0
:106FD00080B584B00390019300920398B0F1006FE4
:106FE00005D3FFE70398B0F1016F10D3FFE70398D3
:106FF00047F60001C1F6FF71884209D3FFE7039805
:1070000047F60F21C1F6FF71884201D8FFE708E07B
:1070100044F62B70C0F6020040F2672116F014FB14
:10702000FFE743F61041C4F20201086820F4407003
:107030000860086840F440700860086840F001008B
:107040000860009803990860BFF36F8F0198039957
:10705000486004B080BD000080B582B00190ADF8FA
:1070600002100198B0F1006F05D3FFE70198B0F16D
:10707000016F10D3FFE7019847F60001C1F6FF71D9
:10708000884209D3FFE7019847F60F21C1F6FF7147
:10709000884201D8FFE708E044F62B70C0F60200F2
:1070A00040F2A22116F0D0FAFFE743F61041C4F2F5
:1070B0000201086820F440700860086840F480709D
:1070C0000860086840F001000860BDF802000199FE
:1070D000088002B080BD000080B582B001900091B0
:1070E0000198B0F1006F05D3FFE70198B0F1016F8F
:1070F00010D3FFE7019847F60001C1F6FF718842FF
:1071000009D3FFE7019847F60F21C1F6FF718842C6
:1071100001D8FFE708E044F62B70C0F6020040F209
:10712000892116F091FAFFE743F61041C4F20201FB
:10713000086820F440700860086840F40070086037
:10714000086840F00100086000980199086002B0EA
:1071500080BD000043F60C40C4F202000068C00687
:1071600000280FD5FFE742F2B431C2F20001C8692E
:1071700040F01000C86143F60C41C4F20201102037
:107180000860FFE743F60C40C4F202000068800686
:1071900000280FD5FFE742F2B431C2F20001C869FE
:1071A00040F00800C86143F60C41C4F202012020FF
:1071B0000860FFE743F60C40C4F202000068400696
:1071C00000280FD5FFE742F2B431C2F20001C869CE
:1071D00040F00400C86143F60C41C4F202014020B3
:1071E0000860FFE743F60C40C4F2020000680006A6
:1071F00000280FD5FFE742F2B431C2F20001C8699E
:1072000040F00200C86143F60C41C4F20201802044
:107210000860FFE743F60C40C4F2020000688007F4
:1072200000280FD5FFE742F2B431C2F20001C8696D
:1072300040F02000C86143F60C41C4F20201022074
:107240000860FFE77047000080B584B0029000201E
:10725000019042F2B431C2F20001C86104F0C8F8F2
:107260000190FFE743F60C40C4F202000068C0033F
:10727000002815D5FFE70298013080B1FFE702989A
:1072800040B1FFE704F0B4F80199401A029988422E
:1072900004D9FFE703208DF80F0023E0FFE7E1E7C3
:1072A00043F60C40C4F202000068C00738B1FFE7A3
:1072B00043F60C41C4F2020101200860FFE743F6E7
:1072C0000C40C4F20200006810F0F20F06D0FFE795
:1072D000FFF740FF01208DF80F0003E000208DF83C
:1072E0000F00FFE79DF80F0004B080BD40F6D110FD
:1072F000C2F200007047000088B007900691059226
:1073000000200490039005990860FFE7049806990F
:10731000884260D2FFE7FFE70798017800200290DB
:1073200039B1FFE707980078203818BF0120029094
:10733000FFE70298C00720B1FFE7079801300790E8
:10734000EAE7FFE7079801780020019041B1FFE7E5
:10735000079800782038B0FA80F040090190FFE7E4
:107360000198C00720B1FFE7079801300790E9E7CF
:107370000798007868B3FFE70498013004900498F8
:107380000699884224D1FFE707980390FFE7079802
:1073900001780020009039B1FFE707980078203885
:1073A00018BF01200090FFE70098C00740B1FFE739
:1073B0000599086801300860079801300790E6E7F2
:1073C0000598006818B9FFE700200390FFE702E086
:1073D00000E000E09AE7039808B0704780B586B0F7
:1073E0000590049103920120029040F27830C2F29D
:1073F00000000068002859D1FFE740F27831C2F25E
:10740000000140F2F020C2F200000860FFE740F205
:107410007830C2F200000068002846D0FFE740F252
:107420007830C2F20000006800680068019001989E
:10743000F8F73AFF009005980099405C202805D0A5
:10744000FFE705980099405C30BBFFE7059801997C
:10745000009AF8F747FFF0B9FFE740F27830C2F240
:1074600000000068006890F90C00002812D4FFE7C3
:10747000059817F001FA40F27831C2F2000109686C
:10748000096891F90C10884203D0FFE700200290B0
:10749000FFE7FFE709E0FFE7FFE740F27831C2F2DC
:1074A0000001086840680860B1E7FFE740F2783003
:1074B000C2F20000006890B1FFE7029878B9FFE7D8
:1074C0000498039A45F28321C0F60201F8F7E0FE22
:1074D00040F27831C2F200010020086029E040F259
:1074E0007830C2F200000068B8B1FFE740F27830AF
:1074F000C2F2000000680068836804980399059A46
:1075000098470290029838B9FFE740F27831C2F20A
:10751000000100200860FFE70AE00498039A45F2A2
:10752000DB21C0F60201F8F7B3FE00200290FFE76E
:10753000FFE7029806B080BD80B586B003900020BA
:107540000190039858B9FFE74FF0500080F311887D
:10755000BFF36F8FBFF34F8F0490FFE7FEE7082064
:1075600017F0F4FF0290029858B9FFE74FF050006F
:1075700080F31188BFF36F8FBFF34F8F0590FFE744
:10758000FEE70298B0B1FFE718F0B2FA039802994B
:107590000860029900204860029840F22401C2F27B
:1075A00000010A6850600298086018F0CDFA0120C6
:1075B0000190FFE7019806B080BD000080B584B05F
:1075C00047F61020C1F6FF700068039047F61420BC
:1075D000C1F6FF700068029047F61820C1F6FF70F0
:1075E000006801900199039808440390039888B1BA
:1075F000FFE7039840F26811C2F2000100910231E6
:1076000008220AF08BFF00990298123104220AF036
:1076100085FFFFE704B080BD80B58EB006AB049354
:107620000C900B910A920C9820B9FFE7FF208DF87F
:10763000370054E10B9820B9FFE7FF208DF83700A1
:107640004DE10A990C980268891A00EE101AB8EEFA
:10765000400A9FEDA51A80EE010A80ED010A0A9802
:107660000C9908600C980B99097800F0EDF90B98CB
:1076700090ED020AB1EE400A80ED020A0B9890EDFF
:10768000010AB1EE400A80ED010A0C9810300B9906
:1076900091ED010ADFED950ACDED020AFDF7C6FE78
:1076A0009DED021A0C9890ED054A90ED430A90ED7D
:1076B0005B3A90ED5E2A32EE042A72EE430AFDF741
:1076C000F7FE9DED021A049880ED030A0C9890EDE8
:1076D000054A90ED440A90ED5B3A90ED5E2A32EE59
:1076E000042A72EE430AFDF7E3FE049981ED020AD3
:1076F0000B98083091ED020AD1ED030AFDF736FF31
:107700000B9890ED021A0C9890ED050A30EE010AE4
:1077100080ED050A0B980430F9F712FC0C98007BF9
:107720000146039140B1FFE7039801281DD0FFE710
:10773000039802285CD074E000208DF81700FFE762
:107740009DF8170001280FDCFFE70C989DF8171033
:1077500000EB81010020C1F85401FFE79DF81700FC
:1077600001308DF81700EBE75BE00C9901F1580050
:10777000D1ED011A91ED040AD1ED5A0A9FED5C1A80
:107780008DED011A0CF052FB049A9DED011A82ED69
:10779000010A0C9901F11C0092ED010AD1ED011AC8
:1077A000D1ED590A0CF042FB9DED011A0C9880EDC9
:1077B000550A0C9901F1D000D1ED011A91ED050A9D
:1077C000D1ED5B0A0CF032FB049A9DED011A82EDBB
:1077D000000A0C9901F1940092ED000AD1ED011A12
:1077E000D1ED570A0CF022FB0C9880ED560A18E0F8
:1077F00000208DF81600FFE79DF8160001280FDC29
:10780000FFE70C989DF8161000EB81010020C1F8ED
:107810005401FFE79DF8160001308DF81600EBE7E4
:10782000FFE700208DF81500FFE79DF815000128FF
:107830001BDCFFE70C999DF8152001EB421000F5C9
:107840008A7001EB820191ED550A0AF0DFFE0C9877
:107850009DF8151000EB810080ED550AFFE79DF8BB
:10786000150001308DF81500DFE70C98806890F85E
:107870008C00C00740B1FFE70C9890ED550AB1EEBF
:10788000400A80ED550AFFE70C98806890F88D005B
:10789000C00740B1FFE70C9890ED560AB1EE400AE0
:1078A00080ED560AFFE70C9890ED550AB5EE400AB8
:1078B000F1EE10FA02DAFFE700BFFFE70C9890ED57
:1078C000560AB6EE001AB4EE410AF1EE10FA02DDE5
:1078D000FFE700BFFFE700208DF83700FFE79DF9C5
:1078E00037000EB080BD00BF00007A44DB0FC940F6
:1078F0000000000082B0019000910198D0F854017E
:10790000009908600198D0F858010099486002B0C9
:107910007047000082B0019000910198007B0099AF
:10792000087002B07047000080B58AB005AA0392C3
:10793000024603980892079180ED010AC0ED000A03
:10794000089820B9FFE7FF208DF8270076E0079818
:10795000089988600899002008730898806890F852
:107960008D00C00720B1FFE706A8FDF7EFFDFFE798
:10797000039890ED010A089880ED430A089880ED7D
:10798000440A089901F58870896891ED220AB1EEE0
:10799000400ADFED2C0AFDF749FD039A089901F131
:1079A000580092ED000A896801F12002002102913D
:1079B0000CF0B4FB039A089901F11C0092ED000A47
:1079C0008A68012101910CF0A9FB039B0299089A96
:1079D00002F1D00093ED000A926860320CF09EFB39
:1079E000039B0199089A02F1940093ED000A9268B2
:1079F00040320CF093FB02988DF81300FFE79DF8DE
:107A00001300012816DCFFE7039A08999DF813007C
:107A100001EB401000F58A7092ED000A8968D1ED03
:107A2000200A0AF04FFEFFE79DF8130001308DF8A1
:107A30001300E4E700208DF82700FFE79DF92700F9
:107A40000AB080BDDB0FC94080B584B002908DF8CC
:107A50000710029820B9FFE7FF208DF80F0065E0BE
:107A60009DF807000299097B884204D1FFE70020B6
:107A70008DF80F005AE000208DF80600FFE79DF812
:107A80000600032811DCFFE702989DF80610C1EB01
:107A9000011100EB81001C300CF00CFCFFE79DF89D
:107AA000060001308DF80600E9E700208DF805009A
:107AB000FFE79DF80500012812DCFFE702989DF81A
:107AC000051000EB411000F58A709FED1A0A0AF0CC
:107AD00097FEFFE79DF8050001308DF80500E8E707
:107AE00002981030F9F72CFA0298007BB0B9FFE742
:107AF0009DF80700012805D1FFE70299D1F8680138
:107B000008610AE09DF80700022805D1FFE7029905
:107B1000D1F874010861FFE7FFE7FFE79DF8070070
:107B20000299087300208DF80F00FFE79DF90F0000
:107B300004B080BD0000000080B584B002900191C7
:107B4000029820B9FFE7FF208DF80F002EE0019882
:107B500020B9FFE7FF208DF80F0027E00198406C67
:107B60000299C1F874010198406D0299C1F8780139
:107B70000298806890F88C00C00730B1FFE7029847
:107B800000F5BA70FDF7E2FCFFE70298806890F814
:107B90008D00C00730B1FFE7029800F5BC70FDF71B
:107BA000D5FCFFE700208DF80F00FFE79DF90F00DF
:107BB00004B080BD80B586B004900391002002908F
:107BC00003980068122801D8FFE708E045F24E004C
:107BD000C0F6020040F2896115F036FDFFE7039818
:107BE000406830B1FFE703984068102801D8FFE7EC
:107BF00008E045F24E00C0F6020040F28A6115F03E
:107C000023FDFFE70398806818B3FFE703988068B7
:107C100001281ED0FFE703988068022819D0FFE7EB
:107C200003988068032814D0FFE70398806804282D
:107C30000FD0FFE70398806805280AD0FFE7039874
:107C40008068062805D0FFE703988068072801D1DF
:107C5000FFE708E045F24E00C0F6020040F28B61FB
:107C600015F0F2FCFFE7FFE7049890F83C000128CC
:107C700004D1FFE702208DF81700F7E004990120F6
:107C800081F83C00FFE7FFE7039800680A281CD34F
:107C9000FFE70398008800EB4000A0F11E010720D9
:107CA00000FA01F204980168C8689043C86003991B
:107CB0008868098801EB41011E3900FA01F2049835
:107CC0000168C8681043C86018E00398008800EB9A
:107CD0004001072000FA01F2049801680869904306
:107CE000086103998868098801EB410100FA01F2F3
:107CF00004980168086910430861FFE70398406829
:107D000006281BD8FFE70398406800EB8000411F5E
:107D10001F2000FA01F204980168486B9043486301
:107D200003990888496801EB8101053900FA01F2DD
:107D300004980168486B104348633DE0039840682D
:107D40000C281CD8FFE70398406800EB8000A0F1E6
:107D500023011F2000FA01F204980168086B904388
:107D6000086303990888496801EB8101233900FA07
:107D700001F204980168086B104308631BE0039844
:107D8000406800EB8000A0F141011F2000FA01F2E1
:107D900004980168C86A9043C862039908884968D2
:107DA00001EB8101413900FA01F204980168C86AC7
:107DB0001043C862FFE7FFE742F20030C4F201005F
:107DC00001900498006842F20001C4F20101884267
:107DD0000BD1FFE703980068122806D1FFE701994D
:107DE000486840F480004860FFE70498006842F269
:107DF0000001C4F2010188422ED1FFE70398006818
:107E0000102805D0FFE703980068112824D1FFE768
:107E10000199486840F40000486003980068102801
:107E200019D1FFE740F22800C2F2000000684DF6C9
:107E30008361C4F21B31A0FB0110800C00EB8000B9
:107E400040000290FFE7029820B1FFE70298013856
:107E50000290F8E7FFE7FFE7FFE70499002081F8C9
:107E60003C00FFE700208DF81700FFE79DF81700A2
:107E700006B080BD81B0009000980068C06C01B071
:107E80007047000080B584B0029000208DF8070094
:107E9000029820B9FFE701208DF80F00C7E1029892
:107EA000006842F20001C4F20101884212D0FFE7EB
:107EB0000298006842F20011C4F20101884209D020
:107EC000FFE70298006842F20021C4F201018842F3
:107ED00001D1FFE708E045F24E00C0F6020040F293
:107EE000431115F0B1FBFFE70298406890B1FFE73E
:107EF00002984068B0F5803F0CD0FFE702984068D8
:107F0000B0F5003F06D0FFE702984068B0F5403F6B
:107F100001D1FFE708E045F24E00C0F602004FF441
:107F2000A27115F091FBFFE70298806890B1FFE71E
:107F300002988068B0F1807F0CD0FFE702988068DB
:107F4000B0F1007F06D0FFE702988068B0F1407F73
:107F500001D1FFE708E045F24E00C0F6020040F212
:107F6000451115F071FBFFE70298006928B1FFE7A2
:107F700002980069012801D1FFE708E045F24E00B0
:107F8000C0F602004FF4A37115F05EFBFFE7029804
:107F9000007E28B1FFE70298007E012801D1FFE7AB
:107FA00008E045F24E00C0F6020040F2471115F01D
:107FB0004BFBFFE70298806A002862D0FFE7029837
:107FC000806AB0F1807F5CD0FFE70298806AB0F1F0
:107FD000007F56D0FFE70298806AB0F1407F50D012
:107FE000FFE70298806AB0F1806F4AD0FFE70298FD
:107FF000806AB0F1A06F44D0FFE70298806AB0F1C8
:10800000C06F3ED0FFE70298806AB0F1E06F38D0D1
:10801000FFE70298806AB0F1006F32D0FFE7029864
:10802000806AB0F1106F2CD0FFE70298806AB0F13F
:10803000206F26D0FFE70298806AB0F1306F20D021
:10804000FFE70298806AB0F1406F1AD0FFE702980C
:10805000806AB0F1506F14D0FFE70298806AB0F1E7
:10806000606F0ED0FFE70298806AB0F1706F08D0A1
:10807000FFE70298806A0121C0F60071884201D1B1
:10808000FFE708E045F24E00C0F602004FF4A4718D
:1080900015F0DAFAFFE70298C06830B1FFE70298FE
:1080A000C068B0F5006F01D1FFE708E045F24E006F
:1080B000C0F6020040F2491115F0C6FAFFE7029837
:1080C000C06930B1FFE70298C069102801D8FFE706
:1080D00008E045F24E00C0F602004FF4A57115F01D
:1080E000B3FAFFE7029890F8300030B1FFE702984A
:1080F00090F83000012801D1FFE708E045F24E007A
:10810000C0F6020040F24B1115F09EFAFFE702980C
:108110004069012809D0FFE70298406928B1FFE7CC
:1081200002984069022801D1FFE708E045F24E00BD
:10813000C0F602004FF4A67115F086FAFFE7029828
:1081400090F8200030B1FFE7029890F82000012855
:1081500001D1FFE708E045F24E00C0F6020040F210
:108160004D1115F071FAFFE70298806A0121C0F6FF
:108170000071884221D0FFE70298C06A90B1FFE702
:108180000298C06AB0F1805F0CD0FFE70298C06A25
:10819000B0F1005F06D0FFE70298C06AB0F1405F1F
:1081A00001D1FFE708E045F24E00C0F6020040F2C0
:1081B000511115F049FAFFE7FFE70298006C50B93A
:1081C000FFE7029800F038F802990020486402990D
:1081D00081F83C00FFE70298006CC006002817D425
:1081E000FFE70298006C40F0020020F488500299EA
:1081F00008640298F8F7DAFB0299002048640298B4
:10820000006C40F0010020F002000299086403E0D5
:1082100001208DF80700FFE7FFE70299002081F8B1
:108220003C00FFE79DF807008DF80F00FFE79DF881
:108230000F0004B080BD000080B58AB00990002016
:10824000089007900690059004900998006842F203
:108250000001C4F20101884212D1FFE7FFE70020CC
:10826000039043F64400C4F20200016841F48071B7
:108270000160006800F4807003900398FFE73AE023
:108280000998006842F20021C4F20101884231D10C
:10829000FFE7FFE70020029043F64400C4F202002B
:1082A000016841F480610160006800F48060029020
:1082B0000298FFE7FFE70020019043F63000C4F288
:1082C0000200016841F020010160006800F0200018
:1082D00001900198FFE74FF480600490032005901F
:1082E0000020069041F20040C4F2020004A902F00E
:1082F00089FCFFE7FFE70AB080BD000080B584B0CD
:10830000029001910020009002980068806840056A
:10831000002816D5FFE7029800688068C00500288D
:108320000FD5FFE70299086C40F020000864FFE7D2
:108330000299002081F83C00FFE701208DF80F0032
:108340006DE003F055F80090FFE7029800680068C0
:1083500000F00200022829D0FFE70198013020B385
:10836000FFE7019840B1FFE703F042F80099401A97
:108370000199884218D9FFE702980068006800F068
:10838000020002280FD0FFE70299086C40F00400B9
:108390000864FFE70299002081F83C00FFE7032012
:1083A0008DF80F003BE0FFE7FFE7CEE7029801689A
:1083B0006FF0120008600299086C40F400700864C5
:1083C00002980068806810F0405F24D1FFE70298AF
:1083D000007E00BBFFE702980068C06A10F4700FCF
:1083E00007D0FFE70298006880684005002812D493
:1083F000FFE70299086C20F4807008640298006C12
:10840000C004002806D4FFE70299086C40F0010080
:108410000864FFE7FFE700208DF80F00FFE79DF8F5
:108420000F0004B080BD000080B584B00290002031
:1084300001900298007E28B1FFE70298007E012893
:1084400001D1FFE708E045F24E00C0F6020040F21D
:10845000D32115F0F9F8FFE70298C06A90B1FFE761
:108460000298C06AB0F1805F0CD0FFE70298C06A42
:10847000B0F1005F06D0FFE70298C06AB0F1405F3C
:1084800001D1FFE708E045F24E00C0F602004FF4CC
:10849000357115F0D9F8FFE7FFE7029890F83C0036
:1084A000012804D1FFE702208DF80F00D4E00299E3
:1084B000012081F83C00FFE7FFE702980068806830
:1084C000C007F0B9FFE702980168886840F0010032
:1084D000886040F22800C2F2000000684DF6836117
:1084E000C4F21B31A0FB0110800C00EB4000019096
:1084F000FFE7019820B1FFE7019801380190F8E704
:10850000FFE7029800688068C007002800F09580A7
:10851000FFE70298006C40F4807040F201618843EC
:10852000029908640298006840684005002809D54F
:10853000FFE70298006C40F4805020F4005002994C
:108540000864FFE70298006CC004002806D5FFE726
:108550000299486C20F00600486403E0029900206C
:108560004864FFE7FFE70299002081F83C00FFE73D
:1085700042F20030C4F201000090029801686FF0EE
:108580002200086000984068C006E8BBFFE7029838
:10859000006842F20001C4F20101884224D0FFE7E2
:1085A0000298006842F20011C4F20101884208D129
:1085B000FFE742F20430C4F201000068C00698B13F
:1085C000FFE70298006842F20021C4F201018842EC
:1085D00019D1FFE742F20430C4F20100006800F054
:1085E0001F000F280FD8FFE702980068806810F07E
:1085F000405F07D1FFE702980168886840F080403B
:108600008860FFE7FFE717E00298006842F2000188
:10861000C4F2010188420ED1FFE702980068806829
:1086200010F0405F07D1FFE702980168886840F0CA
:1086300080408860FFE7FFE70AE00299086C40F09D
:10864000100008640299486C40F001004864FFE79C
:1086500000208DF80F00FFE79DF80F0004B080BDEB
:1086600080B584B002900191029890F820008DF8B6
:108670000300019848F67F71C0F20301884201D8D7
:10868000FFE708E045F28600C0F602004FF4D06133
:1086900014F0DAFFFFE79DF80300012805D0FFE79B
:1086A0009DF8030002280AD1FFE7019A02980168A9
:1086B00048691043486100208DF80F0008E00299D6
:1086C000486A40F48020486201208DF80F00FFE7DF
:1086D0009DF80F0004B080BD80B588B0069005916C
:1086E00004920393069890F820008DF807000698EE
:1086F0000068806800900598806828B1FFE70598B9
:108700008068042801D1FFE708E045F28600C0F642
:10871000020040F2E94114F097FFFFE70598C068B6
:1087200028B1FFE70598C068022801D1FFE708E0FB
:1087300045F28600C0F6020040F2EA4114F084FFE0
:10874000FFE705980069082801D8FFE708E045F22F
:108750008600C0F6020040F2EB4114F075FFFFE71F
:108760000598806890B9FFE7059801680020B0EB94
:10877000D12F01D1FFE708E045F28600C0F60200E4
:1087800040F2EE4114F060FFFFE711E00598416808
:108790000020B0EB517F01D1FFE708E045F28600F1
:1087A000C0F6020040F2F24114F04EFFFFE7FFE78F
:1087B0000598007D28B1FFE70598007D012801D1CB
:1087C000FFE708E045F28600C0F6020040F2F441FF
:1087D00014F03AFFFFE79DF80700012806D0FFE7F5
:1087E0009DF80700022840F08D80FFE79DF8030008
:1087F000400700280CD4FFE79DF80300000700287D
:1088000006D4FFE79DF80300C006002871D5FFE7F6
:108810000098C0F3016002900298032809D3FFE793
:108820000699486A40F40000486201208DF81F0054
:1088300071E00299012088400399086005988068DA
:1088400068B9FFE705980168C06840EA4150069999
:108850000968029A01EB0211C1F880010EE0059946
:108860004A688868C96840EAC200084306990968EE
:10887000029A01EB0211C1F88001FFE70598006937
:1088800006990968029A01EB0211C1F88401059862
:10889000007D01280CD1FFE706980068029900EBE3
:1088A0000111D1F8840140F48070C1F88401FFE720
:1088B0000498406806990968029A01EB0211C1F810
:1088C0008C010498006806990968029A01EB02116C
:1088D000C1F8880106980068029900EB0111D1F8EF
:1088E000800140F00100C1F8800100208DF81F00D8
:1088F00011E00699486A40F40010486201208DF8A2
:108900001F0008E00699486A40F480204862012070
:108910008DF81F00FFE79DF81F0008B080BD000024
:1089200080B586B004900391049800680190049883
:1089300090F820008DF803009DF80300012806D070
:10894000FFE79DF80300022840F05281FFE70398FB
:10895000408808B9FFE708E045F28600C0F602004B
:108960004FF4547114F070FEFFE70398C08808B903
:10897000FFE708E045F28600C0F6020040F2513100
:1089800014F062FEFFE70398408908B9FFE708E0AA
:1089900045F28600C0F6020040F2523114F054FE57
:1089A000FFE70398C08908B9FFE708E045F28600B1
:1089B000C0F6020040F2533114F046FEFFE7039880
:1089C000806928B1FFE703988069012801D1FFE79A
:1089D00008E045F28600C0F602004FF4557114F02D
:1089E00033FEFFE70398C06928B1FFE70398C06929
:1089F000012801D1FFE708E045F28600C0F6020039
:108A000040F2553114F020FEFFE70398006928B1C9
:108A1000FFE703980069012801D1FFE708E045F26C
:108A20008600C0F6020040F2563114F00DFEFFE75A
:108A30000398006A28B1FFE70398006A012801D172
:108A4000FFE708E045F28600C0F6020040F2573129
:108A500014F0FAFDFFE746F20040C4F20000019076
:108A6000039840691B2801D8FFE708E045F286001B
:108A7000C0F6020040F2723114F0E6FDFFE7039801
:108A8000406A1B2801D8FFE708E045F28600C0F6DF
:108A9000020040F2733114F0D7FDFFE70199D1F8DD
:108AA000000240F00100C1F800020199D1F8000273
:108AB00020F47C50C1F800020398426A0199D1F871
:108AC000000240EA0220C1F800020398406900F069
:108AD0001F01012088400290029A0199D1F81C02DE
:108AE0009043C1F81C020398C069F0B9FFE7029AED
:108AF0000199D1F80C029043C1F80C02039A9088B6
:108B0000D168526940EA0140019901EBC201C1F804
:108B10004002039A10889168526940EA0140019925
:108B200001EBC201C1F84402FFE70398C0690128C4
:108B30001ED1FFE7029A0199D1F80C021043C1F847
:108B40000C02039A90881168526940EA0140019929
:108B500001EBC201C1F84002039A90899168526901
:108B600040EA0140019901EBC201C1F84402FFE76C
:108B70000398806940B9FFE7029A0199D1F804028D
:108B80009043C1F8040207E0029A0199D1F8040267
:108B90001043C1F80402FFE70398006940B9FFE7FA
:108BA000029A0199D1F814029043C1F8140207E027
:108BB000029A0199D1F814021043C1F81402FFE798
:108BC0000398006A012808D1FFE7029A0199D1F8B9
:108BD0001C021043C1F81C02FFE70199D1F8000202
:108BE00020F00100C1F8000200208DF8170008E015
:108BF0000499486A40F48020486201208DF81700EB
:108C0000FFE79DF8170006B080BD000080B582B078
:108C100001900198FAF7CAFD8DF803009DF8030052
:108C2000032819D0FFE79DF8030040F2F822C2F2B2
:108C30000002342110FB0120006B60B1FFE79DF8BA
:108C4000030040F2F822C2F20002342110FB01209E
:108C5000006B8047FFE7FFE702B080BD80B586B0BC
:108C60000490039102920193049890F820008DF8EB
:108C70000300039820B1FFE70398012801D1FFE723
:108C800008E045F28600C0F602004FF4BE6114F021
:108C9000DBFCFFE79DF80300012806D0FFE79DF805
:108CA0000300022840F0D780FFE7039880B9FFE770
:108CB00004980068C068800748B9FFE70499486ACB
:108CC00040F40010486201208DF81700CCE00FE05E
:108CD000049800680069800748B9FFE70499486A6A
:108CE00040F40010486201208DF81700BCE0FFE757
:108CF00004980068039900EB0110D0F8B00100F06F
:108D00000400029988600298806858B9FFE70498C7
:108D10000068039900EB0110D0F8B001400D0299F2
:108D200008600AE004980068039900EB0110D0F88D
:108D3000B001C00802994860FFE7049800680399F1
:108D400000EB0110D0F8B00100F002000299C860F9
:108D500004980068039900EB0110D0F8B40100F00A
:108D60000F000299086104980068039900EB011054
:108D7000D0F8B40180B2000A0299886104980068B2
:108D8000039900EB0110D0F8B401000C029948617E
:108D900004980068039900EB0110D0F8B80101991C
:108DA000087004980068039900EB0110D0F8B8012E
:108DB000000A0199487004980068039900EB0110BB
:108DC000D0F8B801000C01998870049800680399E4
:108DD00000EB0110D0F8B801000E0199C87004989A
:108DE0000068039900EB0110D0F8BC0101990871EB
:108DF00004980068039900EB0110D0F8BC01000A48
:108E00000199487104980068039900EB0110D0F8AB
:108E1000BC01000C0199887104980068039900EB6B
:108E20000110D0F8BC01000E0199C871039838B93F
:108E3000FFE704980168C86840F02000C86006E0B9
:108E400004980168086940F020000861FFE70020ED
:108E50008DF8170008E00499486A40F480204862C1
:108E600001208DF81700FFE79DF8170006B080BDC0
:108E700080B58AB009900020089009980068406980
:108E80000790099800684068069009980068806813
:108E9000059009980068C068049009980068006906
:108EA000039009980068806902909DF81C00C00733
:108EB000002800F09480FFE79DF81400C00758B325
:108EC000FFE709980168012088609DF81400800779
:108ED000002804D5FFE7099800F042FE1BE09DF84A
:108EE00014004007002805D5FFE7089840F400600B
:108EF00008900FE09DF814000007002805D5FFE753
:108F0000089840F48050089003E0099800F000FEB3
:108F1000FFE7FFE7FFE7FFE79DF81500C00760B335
:108F2000FFE7099801684FF4807088609DF815008C
:108F30008007002804D5FFE7099800F05FFE1BE0DA
:108F40009DF815004007002805D5FFE7089840F474
:108F5000005008900FE09DF815000007002805D587
:108F6000FFE7089840F48040089003E0099800F07B
:108F70001DFEFFE7FFE7FFE7FFE79DF81600C007CC
:108F800060B3FFE7099801684FF4803088609DF86E
:108F900016008007002804D5FFE7099800F07EFE40
:108FA0001BE09DF816004007002805D5FFE708984C
:108FB00040F4004008900FE09DF8160000070028DC
:108FC00005D5FFE7089840F48030089003E0099841
:108FD00000F03CFEFFE7FFE7FFE7FFE7FFE79DF854
:108FE0001C000007002810D5FFE79DF81000C00600
:108FF000002809D5FFE7089840F400700890099808
:1090000001681020C860FFE7FFE79DF81C004007DB
:1090100000280FD5FFE79DF810000007002808D5AD
:10902000FFE7099801680820C860099800F062FC11
:10903000FFE7FFE79DF81C00800700280BD5FFE73E
:1090400009980068C068800720B1FFE7099800F020
:1090500079FCFFE7FFE79DF81C004006002810D5CB
:10906000FFE79DF80C00C006002809D5FFE7089827
:1090700040F4806008900998016810200861FFE7BB
:10908000FFE79DF81C00800600280FD5FFE79DF83C
:109090000C000007002808D5FFE7099801680820A0
:1090A0000861099800F076FCFFE7FFE79DF81C00D7
:1090B000C00600280BD5FFE7099800680069800703
:1090C00020B1FFE7099800F08DFCFFE7FFE79DF86E
:1090D0001E00800700280FD5FFE79DF81800C00686
:1090E000002808D5FFE70998016810204860099812
:1090F00000F0A0FCFFE7FFE79DF81E00C00778B175
:10910000FFE79DF818000007002808D5FFE7099839
:10911000016808204860099800F0E8FDFFE7FFE7D4
:109120009DF81D000006002840F18D80FFE79DF8A6
:1091300018004007002840F18180FFE79DF81D00DE
:10914000C00750B1FFE79DF80800C00728B1FFE74E
:10915000089840F001000890FFE79DF81D00800787
:1091600000280BD5FFE79DF808008007002805D5EB
:10917000FFE7089840F002000890FFE79DF81D0007
:10918000400700280BD5FFE79DF80800400700289E
:1091900005D5FFE7089840F004000890FFE79DF828
:1091A0001D000007002848D5FFE79DF8080010F0D3
:1091B000700F42D0FFE7029800F070000146019165
:1091C000102814D0FFE70198202815D0FFE7019858
:1091D000302816D0FFE70198402817D0FFE7019804
:1091E000502818D0FFE70198602819D01DE0089892
:1091F00040F00800089019E0089840F0100008902E
:1092000014E0089840F0200008900FE0089840F023
:10921000400008900AE0089840F08000089005E0BF
:10922000089840F48070089000E0FFE70998016812
:10923000886920F070008861FFE7FFE709980168FE
:1092400004204860FFE7089848B1FFE7089A0999A9
:10925000486A104348620998FFF7D8FCFFE70AB054
:1092600080BD000080B584B00290029820B9FFE76D
:1092700001208DF80F0063E20298006846F2004179
:10928000C4F20001884209D0FFE70298006846F660
:109290000001C4F20001884201D1FFE708E045F275
:1092A0008600C0F6020040F21D1114F0CDF9FFE770
:1092B0000298007E28B1FFE70298007E012801D1C4
:1092C000FFE708E045F28600C0F602004FF48F7118
:1092D00014F0BAF9FFE70298407E28B1FFE7029840
:1092E000407E012801D1FFE708E045F28600C0F684
:1092F000020040F21F1114F0A7F9FFE70298807EE8
:1093000028B1FFE70298807E012801D1FFE708E03D
:1093100045F28600C0F602004FF4907114F094F903
:10932000FFE70298C07E28B1FFE70298C07E0128BF
:1093300001D1FFE708E045F28600C0F6020040F2E6
:10934000211114F081F9FFE70298007F28B1FFE7AF
:109350000298007F012801D1FFE708E045F286006E
:10936000C0F602004FF4917114F06EF9FFE7029815
:10937000407F28B1FFE70298407F012801D1FFE735
:1093800008E045F28600C0F6020040F2231114F016
:109390005BF9FFE70298806890B1FFE70298806868
:1093A000B0F1804F0CD0FFE702988068B0F1004F19
:1093B00006D0FFE702988068B0F1404F01D1FFE787
:1093C00008E045F28600C0F602004FF4927114F0F6
:1093D0003BF9FFE70298C06890B1FFE70298C068C8
:1093E000B0F1807F0CD0FFE70298C068B0F1007F39
:1093F00006D0FFE70298C068B0F1407F01D1FFE7D7
:1094000008E045F28600C0F6020040F2251114F093
:109410001BF9FFE70298006900285AD0FFE702987D
:109420000069B0F5803F54D0FFE702980069B0F5BD
:10943000003F4ED0FFE702980069B0F5403F48D0AA
:10944000FFE702980069B0F5802F42D0FFE702984D
:109450000069B0F5A02F3CD0FFE702980069B0F595
:10946000C02F36D0FFE702980069B0F5E02F30D06A
:10947000FFE702980069B0F5002F2AD0FFE70298B5
:109480000069B0F5102F24D0FFE702980069B0F50D
:10949000202F1ED0FFE702980069B0F5302F18D0BA
:1094A000FFE702980069B0F5402F12D0FFE702985D
:1094B0000069B0F5502F0CD0FFE702980069B0F5B5
:1094C000602F06D0FFE702980069B0F5702F01D138
:1094D000FFE708E045F28600C0F602004FF4937102
:1094E00014F0B2F8FFE70298406950B3FFE7029822
:1094F0004069B0F5801F24D0FFE702984069B0F5BD
:10950000001F1ED0FFE702984069B0F5401F18D039
:10951000FFE702984069B0F5800F12D0FFE702988C
:109520004069B0F5A00F0CD0FFE702984069B0F594
:10953000C00F06D0FFE702984069B0F5E00F01D1F7
:10954000FFE708E045F28600C0F6020040F227116E
:1095500014F07AF8FFE70298406838B1FFE7029804
:109560004068B0F5806F01D8FFE708E045F286005B
:10957000C0F602004FF4947114F066F8FFE7029809
:1095800090F8200020B9FFE7029800F0DDF8FFE72F
:1095900002980168086820F00200086001F028FFC6
:1095A0000190FFE70298006840688007002815D501
:1095B000FFE701F01DFF0199401A0B280DD3FFE7CB
:1095C0000299486A40F4003048620299052081F807
:1095D000200001208DF80F00B2E0E3E70298016857
:1095E000086840F00100086001F002FF0190FFE709
:1095F000029800684068C007A8B9FFE701F0F8FECC
:109600000199401A0B280DD3FFE70299486A40F4EC
:10961000003048620299052081F8200001208DF871
:109620000F008DE0E4E70298007E012807D1FFE7F4
:1096300002980168086840F08000086006E002981F
:109640000168086820F080000860FFE70298407E0B
:10965000012807D1FFE702980168086840F0400040
:10966000086006E002980168086820F04000086081
:10967000FFE70298807E012807D1FFE70298016882
:10968000086840F02000086006E002980168086859
:1096900020F020000860FFE70298C07E012807D173
:1096A000FFE702980168086820F01000086006E0F3
:1096B00002980168086840F010000860FFE702980F
:1096C000007F012807D1FFE702980168086840F091
:1096D0000800086006E002980168086820F00800A9
:1096E0000860FFE70298407F012807D1FFE7029852
:1096F0000168086840F00400086006E0029801680C
:10970000086820F004000860FFE7029B19685A68A7
:109710009868D3F80CC040EA0C00D3F810C040EAB7
:109720000C005B691843013A1043C861029900209C
:109730004862029A012182F820108DF80F00FFE79D
:109740009DF80F0004B080BD80B594B01390002048
:109750001290119010900F900E901398006846F29E
:109760000041C4F20001884253D1FFE740F2BC300F
:10977000C2F200000168013101600068012812D1C5
:10978000FFE7FFE700200D9043F64000C4F202001F
:10979000016841F000710160006800F000700D90F8
:1097A0000D98FFE7FFE7FFE700200C9043F630003D
:1097B000C4F20200016841F008010160006800F095
:1097C00008000C900C98FFE703200E9002210F91E7
:1097D00000210791109111900920129040F600404D
:1097E000C4F202000EA901F00DFA079A14200590A8
:1097F0000521069102F018FA059802F0FDF9069984
:10980000079A1520089002F00FFA089802F0F4F970
:109810006EE01398006846F60001C4F20001884229
:1098200065D1FFE7FFE700200B9043F64000C4F24C
:109830000200016841F080610160006800F0806012
:109840000B900B98FFE740F2BC30C2F200000168B9
:10985000013101600068012812D1FFE7FFE7002015
:109860000A9043F64000C4F20200016841F0007122
:109870000160006800F000700A900A98FFE7FFE7B7
:10988000FFE70020099043F63000C4F202000168AF
:1098900041F002010160006800F00200099009989F
:1098A000FFE760200E9002200F90002003901090A0
:1098B000032011900920129040F20040C4F20200EF
:1098C0000EA901F09FF9039A402001900521029111
:1098D00002F0AAF9019802F08FF90299039A412047
:1098E000049002F0A1F9049802F086F9FFE7FFE77F
:1098F00014B080BD80B582B001900198F9F756FF91
:109900008DF803009DF80300032819D0FFE79DF8A8
:10991000030040F2F822C2F20002342110FB0120C1
:10992000C06960B1FFE79DF8030040F2F822C2F27F
:109930000002342110FB0120C0698047FFE7FFE7E8
:1099400002B080BD80B582B001900198F9F72EFF7A
:109950008DF803009DF80300032819D0FFE79DF858
:10996000030040F2F822C2F20002342110FB012071
:10997000806960B1FFE79DF8030040F2F822C2F26F
:109980000002342110FB012080698047FFE7FFE7D8
:1099900002B080BD80B582B001900198F9F706FF52
:1099A0008DF803009DF80300032819D0FFE79DF808
:1099B000030040F2F822C2F20002342110FB012021
:1099C000406A60B1FFE79DF8030040F2F822C2F25E
:1099D0000002342110FB0120406A8047FFE7FFE7C7
:1099E00002B080BD80B582B001900198F9F7DEFE2B
:1099F0008DF803009DF80300032819D0FFE79DF8B8
:109A0000030040F2F822C2F20002342110FB0120D0
:109A1000006A60B1FFE79DF8030040F2F822C2F24D
:109A20000002342110FB0120006A8047FFE7FFE7B6
:109A300002B080BD80B582B001900198F9F7B6FE02
:109A40008DF803009DF80300032819D0FFE79DF867
:109A5000030040F2F822C2F20002342110FB012080
:109A6000806A60B1FFE79DF8030040F2F822C2F27D
:109A70000002342110FB0120806A8047FFE7FFE7E6
:109A800002B080BD80B584B00290029890F82000AA
:109A900001282FD1FFE70299022081F820000298C7
:109AA0000168086820F00100086001F0A1FC019045
:109AB000FFE7029800684068C007A8B1FFE701F01F
:109AC00097FC0199401A0B280DD3FFE70299486AC9
:109AD00040F4003048620299052081F820000120FE
:109AE0008DF80F000FE0E4E70299002048628DF83E
:109AF0000F0008E00299486A40F400204862012003
:109B00008DF80F00FFE79DF80F0004B080BD000046
:109B100080B582B001900198F9F748FE8DF80300F6
:109B20009DF80300032819D0FFE79DF8030040F2D9
:109B3000F822C2F20002342110FB0120C06860B19B
:109B4000FFE79DF8030040F2F822C2F20002342140
:109B500010FB0120C0688047FFE7FFE702B080BD2F
:109B600080B582B001900198F9F720FE8DF80300CE
:109B70009DF80300032817D0FFE79DF80300342168
:109B8000414340F2F820C2F20000405858B1FFE7CC
:109B90009DF803003421414340F2F820C2F2000056
:109BA00040588047FFE7FFE702B080BD80B582B034
:109BB00001900198F9F7FAFD8DF803009DF8030074
:109BC000032819D0FFE79DF8030040F2F822C2F203
:109BD0000002342110FB0120006960B1FFE79DF80D
:109BE000030040F2F822C2F20002342110FB0120EF
:109BF00000698047FFE7FFE702B080BD80B582B013
:109C000001900198F9F7D2FD8DF803009DF803004B
:109C1000032819D0FFE79DF8030040F2F822C2F2B2
:109C20000002342110FB0120406860B1FFE79DF87D
:109C3000030040F2F822C2F20002342110FB01209E
:109C400040688047FFE7FFE702B080BD80B582B083
:109C500001900198F9F7AAFD8DF803009DF8030023
:109C6000032819D0FFE79DF8030040F2F822C2F262
:109C70000002342110FB0120406960B1FFE79DF82C
:109C8000030040F2F822C2F20002342110FB01204E
:109C900040698047FFE7FFE702B080BD80B582B032
:109CA00001900198F9F782FD8DF803009DF80300FB
:109CB000032819D0FFE79DF8030040F2F822C2F212
:109CC0000002342110FB0120806860B1FFE79DF89D
:109CD000030040F2F822C2F20002342110FB0120FE
:109CE00080688047FFE7FFE702B080BD80B582B0A3
:109CF00001900198F9F75AFD8DF803009DF80300D3
:109D0000032819D0FFE79DF8030040F2F822C2F2C1
:109D10000002342110FB0120C06A60B1FFE79DF80A
:109D2000030040F2F822C2F20002342110FB0120AD
:109D3000C06A8047FFE7FFE702B080BD80B582B010
:109D40000090009820B9FFE701208DF8070023E07C
:109D50000098006843F20001C4F20201884201D178
:109D6000FFE707E045F2BE00C0F60200682113F0ED
:109D70006BFCFFE70098407938B9FFE700990020B5
:109D80000871009800F00CF8FFE700990120487175
:109D900000208DF80700FFE79DF8070002B080BDA6
:109DA00082B001900198006843F20001C4F2020100
:109DB000884212D1FFE7FFE70020009043F6300011
:109DC000C4F20200016841F480510160006800F4AF
:109DD000805000900098FFE7FFE702B07047000056
:109DE00080B584B002900298806D019001F000FB74
:109DF0000090029890F8350002280DD0FFE70299F4
:109E000080204865FFE70299002081F83400FFE7D1
:109E100001208DF80F0054E002980168086820F0D6
:109E20001600086002980168486920F080004861C7
:109E30000298006C20B9FFE70298806C38B1FFE708
:109E400002980168086820F008000860FFE702989F
:109E50000168086820F001000860FFE702980068C8
:109E60000068C007C0B1FFE701F0C2FA0099401ACC
:109E7000062810D3FFE7029920204865FFE70299E2
:109E8000002081F83400FFE70299032081F83500B3
:109E90008DF80F0015E0E1E70298C16D3F20884082
:109EA00001998860FFE70299002081F83400FFE7FC
:109EB0000299012081F83500FFE700208DF80F009E
:109EC000FFE79DF80F0004B080BD000082B0009055
:109ED000009890F83500022807D0FFE7009980200D
:109EE000486501208DF807000EE00099052081F8F3
:109EF000350000980168086820F001000860FFE75D
:109F000000208DF80700FFE79DF8070002B07047BA
:109F100080B586B005900020039040F22800C2F280
:109F20000000006848F2B511C1F64E31A0FB0110E7
:109F3000800A02900598806D019001980068049055
:109F400004980599C96DC840000700281AD5FFE795
:109F50000598006800684007002812D5FFE70598BB
:109F60000168086820F0040008600598C16D0820A9
:109F70008840019988600599486D40F00100486566
:109F8000FFE7FFE704980599C96DC840C007A0B175
:109F9000FFE7059800684069000600280CD5FFE738
:109FA0000598C16D01208840019988600599486D28
:109FB00040F002004865FFE7FFE704980599C96D86
:109FC000C8404007002814D5FFE7059800680068DE
:109FD000800700280CD5FFE70598C16D0420884054
:109FE000019988600599486D40F004004865FFE7D5
:109FF000FFE704980599C96DC840C006002847D5F9
:10A00000FFE7059800680068000700283FD5FFE7D4
:10A010000598C16D102088400199886005980068F6
:10A020000068400300281AD5FFE70598006800681B
:10A030000003002809D4FFE70598006C20B1FFE772
:10A040000598016C8847FFE708E00598806C20B10F
:10A05000FFE70598816C8847FFE7FFE716E0059862
:10A0600000680068C005002807D4FFE7059801686C
:10A07000086820F008000860FFE70598006C20B130
:10A08000FFE70598016C8847FFE7FFE7FFE7FFE779
:10A0900004980599C96DC8408006002840F18D805C
:10A0A000FFE7059800680068C006002840F184803A
:10A0B000FFE70598C16D20208840019988600598C8
:10A0C00090F83500052834D1FFE705980168086845
:10A0D00020F01600086005980168486920F08000AB
:10A0E00048610598006C20B9FFE70598806C38B18D
:10A0F000FFE705980168086820F008000860FFE79E
:10A100000598C16D3F20884001998860FFE7059957
:10A11000002081F83400FFE70599012081F835001F
:10A120000598006D20B1FFE70598016D8847FFE7AE
:10A130007BE0059800680068400300281AD5FFE717
:10A140000598006800680003002809D4FFE7059817
:10A15000406C20B1FFE70598416C8847FFE708E0B5
:10A160000598C06B20B1FFE70598C16B8847FFE7F2
:10A17000FFE720E0059800680068C005002811D4BA
:10A18000FFE705980168086820F010000860FFE705
:10A190000599002081F83400FFE70599012081F836
:10A1A0003500FFE70598C06B20B1FFE70598C16B4C
:10A1B0008847FFE7FFE7FFE7FFE70598406DA0B39B
:10A1C000FFE70598406DC00730B3FFE7059905200C
:10A1D00081F8350005980168086820F001000860E2
:10A1E000FFE70398013003900299884201D9FFE705
:10A1F00007E0FFE7059800680068C0070028F0D175
:10A20000FFE7FFE70599002081F83400FFE7059993
:10A21000012081F83500FFE70598C06C20B1FFE709
:10A220000598C16C8847FFE7FFE706B080BD0000D6
:10A2300080B586B004900020039001F0D9F8029018
:10A24000049820B9FFE701208DF8170087E20498F1
:10A25000006846F21001C4F20201884200F08880D2
:10A26000FFE70498006846F22801C4F20201884220
:10A270007ED0FFE70498006846F24001C4F2020174
:10A28000884275D0FFE70498006846F25801C4F28E
:10A29000020188426CD0FFE70498006846F2700122
:10A2A000C4F20201884263D0FFE70498006846F2D6
:10A2B0008801C4F2020188425AD0FFE7049800687E
:10A2C00046F2A001C4F20201884251D0FFE704988F
:10A2D000006846F2B801C4F20201884248D0FFE7A4
:10A2E0000498006846F21041C4F2020188423FD04F
:10A2F000FFE70498006846F22841C4F20201884250
:10A3000036D0FFE70498006846F24041C4F20201EB
:10A3100088422DD0FFE70498006846F25841C4F205
:10A320000201884224D0FFE70498006846F2704199
:10A33000C4F2020188421BD0FFE70498006846F28D
:10A340008841C4F20201884212D0FFE704980068F5
:10A3500046F2A041C4F20201884209D0FFE7049806
:10A36000006846F2B841C4F20201884201D1FFE719
:10A3700007E044F6DB70C0F60200B82113F064F980
:10A38000FFE70498406850B3FFE704984068B0F1D5
:10A39000007F24D0FFE704984068B0F1806F1ED0A2
:10A3A000FFE704984068B0F1C06F18D0FFE7049849
:10A3B0004068B0F1006F12D0FFE704984068B0F138
:10A3C000206F0CD0FFE704984068B0F1406F06D0D2
:10A3D000FFE704984068B0F1606F01D1FFE707E044
:10A3E00044F6DB70C0F60200B92113F02DF9FFE747
:10A3F0000498806850B1FFE704988068402805D031
:10A40000FFE704988068802801D1FFE707E044F661
:10A41000DB70C0F60200BA2113F016F9FFE70498CA
:10A42000C068B0F5007F04D0FFE70498C06808B9A1
:10A43000FFE707E044F6DB70C0F60200BB2113F033
:10A4400003F9FFE704980069B0F5806F04D0FFE7D7
:10A450000498006908B9FFE707E044F6DB70C0F62E
:10A460000200BC2113F0F0F8FFE70498406960B1E6
:10A47000FFE704984069B0F5006F06D0FFE7049845
:10A480004069B0F5805F01D1FFE707E044F6DB707B
:10A49000C0F60200BD2113F0D7F8FFE704988069E9
:10A4A00060B1FFE704988069B0F5005F06D0FFE770
:10A4B00004988069B0F5804F01D1FFE707E044F6CA
:10A4C000DB70C0F60200BE2113F0BEF8FFE704986F
:10A4D000C06958B1FFE70498C069B0F5807F05D026
:10A4E000FFE70498C069202801D1FFE707E044F6A0
:10A4F000DB70C0F60200BF2113F0A6F8FFE7049856
:10A50000006A90B1FFE70498006AB0F5803F0CD074
:10A51000FFE70498006AB0F5003F06D0FFE7049813
:10A52000006AB0F5403F01D1FFE707E044F6DB7079
:10A53000C0F60200C02113F087F8FFE70498406AD4
:10A5400028B1FFE70498406A042801D1FFE707E03B
:10A5500044F6DB70C0F60200C12113F075F8FFE786
:10A560000498406A00285BD0FFE70498806A78B1BD
:10A57000FFE70498806A01280AD0FFE70498806A00
:10A58000022805D0FFE70498806A032801D1FFE77D
:10A5900007E044F6DB70C0F60200C62113F054F861
:10A5A000FFE70498C06A90B1FFE70498C06AB0F56D
:10A5B000000F0CD0FFE70498C06AB0F1807F06D08E
:10A5C000FFE70498C06AB0F1C07F01D1FFE707E060
:10A5D00044F6DB70C0F60200C72113F035F8FFE740
:10A5E0000498006B90B1FFE70498006BB0F5001F72
:10A5F0000CD0FFE70498006BB0F5800F06D0FFE7A2
:10A600000498006BB0F5C00F01D1FFE707E044F6F6
:10A61000DB70C0F60200C82113F016F8FFE7FFE771
:10A62000FFE70499002081F83400FFE70499022035
:10A6300081F8350004980168086820F0010008607E
:10A64000FFE7049800680068C00790B1FFE700F0DA
:10A65000CFFE0299401A06280AD3FFE7049920206A
:10A6600048650499032081F835008DF8170076E0DD
:10A67000E7E70498006800680390039848F23F01F8
:10A68000CFF2100108400390049900914868D1F876
:10A6900008C0CB680A6940EA0C00184310434A69B5
:10A6A00010438A691043CA691043096A0143039839
:10A6B000084303900498406A042808D1FFE70499EE
:10A6C000C86A096B0143039808430390FFE70398A6
:10A6D0000499096808600498006840690390039829
:10A6E00020F0070003900498416A03980843039000
:10A6F0000498406A04281AD1FFE70498816A0398F5
:10A70000084303900498C06A80B1FFE70498FCF7FF
:10A7100075F850B1FFE7049940204865049901207D
:10A7200081F835008DF8170019E0FFE7FFE703987F
:10A730000499096848610498FCF734F8019004987A
:10A74000C16D3F20884001998860049900204865C8
:10A75000049A012182F835108DF81700FFE79DF863
:10A76000170006B080BD000080B588B00690059146
:10A770000492039300208DF80B000698806D0190E1
:10A78000039828B1FFE7BDF80E0008B9FFE708E01D
:10A7900044F6DB70C0F602004FF4E67112F054FF8D
:10A7A000FFE7FFE7069890F83400012804D1FFE79F
:10A7B00002208DF81F0045E00699012081F8340041
:10A7C000FFE7FFE7069890F8350001282BD1FFE757
:10A7D0000699022081F83500069900204865069800
:10A7E0000599049A039BFCF781F80698C16D3F20F8
:10A7F00088400199886006980168086840F0160052
:10A8000008600698006C38B1FFE706980168086890
:10A8100040F008000860FFE706980168086840F00B
:10A820000100086009E0FFE70699002081F8340084
:10A83000FFE702208DF80B00FFE79DF80B008DF875
:10A840001F00FFE79DF81F0008B080BD80B584B0F1
:10A85000039000F0CDFD0290039801900198013023
:10A8600048B1FFE740F2E020C2F200000178019811
:10A8700008440190FFE7FFE700F0BAFD0299401A93
:10A880000199884201D2FFE7F6E704B080BD0000DD
:10A8900080B586B00490039101208DF80B00002054
:10A8A0000190FFE742F2B430C2F20000007E0128BE
:10A8B00004D1FFE702208DF8170094E042F2B43192
:10A8C000C2F2000101200876FFE7FFE70498006864
:10A8D00028B1FFE704980068012801D1FFE707E0ED
:10A8E00044F66570C0F60200AB2112F0ADFEFFE742
:10A8F0004CF25030FCF7A8FC8DF80B009DF80B00D3
:10A90000002863D1FFE703994FF0FF3008600498F7
:10A910000068012814D1FFE70499087C4968FCF716
:10A92000D3FA4CF25030FCF78FFC8DF80B0043F655
:10A930001041C4F20201086820F00400086042E0FF
:10A9400004988168C068084440B1FFE704988168B2
:10A95000C06808440C2801D8FFE707E044F665709A
:10A96000C0F60200C32112F06FFEFFE70498806872
:10A970000190FFE7019804998A68C96811448842E8
:10A9800020D2FFE701980499097CFCF7B1F94CF259
:10A990005030FCF759FC8DF80B0043F61041C4F21F
:10A9A0000201086820F0FA0008609DF80B0020B151
:10A9B000FFE701980399086004E0FFE70198013080
:10A9C0000190D7E7FFE7FCF72DFAFFE7FFE742F238
:10A9D000B431C2F2000100200876FFE79DF80B00B9
:10A9E0008DF81700FFE79DF8170006B080BD000046
:10A9F00043F61041C4F20201086840F000400860CC
:10AA00000020704780B588B00690059103930292AC
:10AA100001208DF80700FFE742F2B430C2F20000D7
:10AA2000007E012804D1FFE702208DF81F0069E0B5
:10AA300042F2B431C2F2000101200876FFE7FFE7DD
:10AA4000069860B1FFE70698012808D0FFE706984E
:10AA5000022804D0FFE70698032801D1FFE707E0AA
:10AA600044F62B70C0F60200A42112F0EDFDFFE7C2
:10AA70004CF25030FCF7E8FB8DF807009DF807001A
:10AA800098BBFFE7069830B9FFE705989DF80810D6
:10AA9000FCF760FA1AE00698012806D1FFE705984E
:10AAA000BDF80810FCF7D8FA0FE00698022805D187
:10AAB000FFE705980299FCF70FFB05E00598029A5D
:10AAC000039BFCF785FAFFE7FFE7FFE74CF2503006
:10AAD000FCF7BAFB8DF8070043F61041C4F20201FF
:10AAE000086820F001000860FFE7FFE742F2B43198
:10AAF000C2F2000100200876FFE79DF807008DF8FC
:10AB00001F00FFE79DF81F0008B080BD81B0002046
:10AB10008DF8030043F61040C4F202000068C00F35
:10AB2000D8B1FFE743F60441C4F2020140F223101A
:10AB3000C4F26750086048F6AB10CCF6EF500860DE
:10AB400043F61040C4F202000068C00F20B1FFE7D6
:10AB500001208DF80300FFE7FFE79DF8030001B037
:10AB60007047000080B582B0ADF8060000208DF877
:10AB70000500FFE79DF805000F2824DCFFE7BDF87E
:10AB800006009DF80510C840C007A8B1FFE79DF872
:10AB9000051040F27C30C2F2000050F8210050B1A4
:10ABA000FFE79DF8051040F27C30C2F2000050F83B
:10ABB00021008047FFE7FFE7FFE79DF80500013030
:10ABC0008DF80500D6E702B080BD000080B582B0E8
:10ABD000ADF8060043F61440C4F201000068BDF869
:10ABE000061008420CD0FFE7BDF8060043F61441FA
:10ABF000C4F201010860BDF80600FFF7B3FFFFE7EC
:10AC000002B080BD80B58EB00D900C9100200A90EE
:10AC1000099008900D980021C4F20201884240D0AA
:10AC2000FFE70D9840F20041C4F20201884238D09B
:10AC3000FFE70D9840F60001C4F20201884230D0CF
:10AC4000FFE70D9840F60041C4F20201884228D087
:10AC5000FFE70D9841F20001C4F20201884220D0C2
:10AC6000FFE70D9841F20041C4F20201884218D07A
:10AC7000FFE70D9841F60001C4F20201884210D0AE
:10AC8000FFE70D9841F60041C4F20201884208D066
:10AC9000FFE70D9842F20001C4F20201884201D19F
:10ACA000FFE707E044F6A270C0F60200AC2112F004
:10ACB000CBFCFFE70C98008828B1FFE70C98408890
:10ACC00008B9FFE707E044F6A270C0F60200AD2124
:10ACD00012F0BAFCFFE70C984068002849D0FFE763
:10ACE0000C984068012844D0FFE70C984068112870
:10ACF0003FD0FFE70C98406802283AD0FFE70C9855
:10AD00004068122835D0FFE70C9840680021C1F256
:10AD1000110188422DD0FFE70C9840680021C1F254
:10AD20002101884225D0FFE70C9840680021C1F23C
:10AD3000310188421DD0FFE70C9840680021C1F224
:10AD40001201884215D0FFE70C9840680021C1F23B
:10AD5000220188420DD0FFE70C9840680021C1F223
:10AD60003201884205D0FFE70C984068032801D1E2
:10AD7000FFE707E044F6A270C0F60200AE2112F031
:10AD800063FCFFE70C98806850B1FFE70C9880687F
:10AD9000012805D0FFE70C988068022801D1FFE761
:10ADA00007E044F6A270C0F60200AF2112F04CFC9E
:10ADB000FFE700200B90FFE70B980F2800F2B0820E
:10ADC000FFE70B99012088400A900C9800680A99C7
:10ADD0000840099009980A99884240F09C82FFE750
:10ADE0000C98406800F00300012807D0FFE70C989A
:10ADF000406800F0030002284BD1FFE70C98C068C0
:10AE000078B1FFE70C98C06801280AD0FFE70C98DA
:10AE1000C068022805D0FFE70C98C068032801D15C
:10AE2000FFE707E044F6A270C0F60200C12112F06D
:10AE30000BFCFFE70D98806808900B9841000320F9
:10AE400000FA01F10898884308900C98C0680B99A3
:10AE5000490000FA01F108980843089008980D99F4
:10AE600088600D98406808900B99012000FA01F164
:10AE70000898884308900C984068C0F300100B991C
:10AE800000FA01F108980843089008980D99486065
:10AE9000FFE70C98406800F00300032818D0FFE794
:10AEA0000D98C06808900B984100032000FA01F14A
:10AEB0000898884308900C9880680B99490000FA1C
:10AEC00001F108980843089008980D99C860FFE7B9
:10AED0000C98406800F00300022840F0EE80FFE785
:10AEE0000C980069002800F0B980FFE70C98006911
:10AEF000092800F0B380FFE70C980069002800F0F3
:10AF0000AD80FFE70C980069002800F0A780FFE7FC
:10AF10000C980069002800F0A180FFE70C980069F8
:10AF2000002800F09B80FFE70C980069012800F0E2
:10AF30009580FFE70C980069012800F08F80FFE7FB
:10AF40000C980069022800F08980FFE70C980069DE
:10AF5000022800F08380FFE70C98006902287DD06A
:10AF6000FFE70C980069032878D0FFE70C98006988
:10AF7000042873D0FFE70C98006904286ED0FFE71F
:10AF80000C980069042869D0FFE70C98006905282F
:10AF900064D0FFE70C98006905285FD0FFE70C98A4
:10AFA000006909285AD0FFE70C980069062855D097
:10AFB000FFE70C980069092850D0FFE70C9800695A
:10AFC00007284BD0FFE70C980069072846D0FFE719
:10AFD0000C980069072841D0FFE70C980069082801
:10AFE0003CD0FFE70C980069082837D0FFE70C98A1
:10AFF0000069082832D0FFE70C98006909282DD095
:10B00000FFE70C980069092828D0FFE70C98006931
:10B010000A2823D0FFE70C9800690A281ED0FFE712
:10B020000C9800690B2819D0FFE70C9800690C28D0
:10B0300014D0FFE70C9800690C280FD0FFE70C989C
:10B0400000690D280AD0FFE70C9800690C2805D08C
:10B05000FFE70C9800690F2801D1FFE707E044F6ED
:10B06000A270C0F60200DC2112F0EEFAFFE70D98A4
:10B070000B996FF0030202EA51010844006A08903C
:10B080000B9800F0070081000F2000FA01F10898EA
:10B09000884308900C9800690B9901F0070189001A
:10B0A00000FA01F108980843089008980D990B9B45
:10B0B00002EA530211440862FFE70D980068089005
:10B0C0000B984100032000FA01F10898884308908A
:10B0D0000C98406800F003000B99490000FA01F158
:10B0E00008980843089008980D9908600C98C07952
:10B0F000C006002840F10E81FFE7FFE7002007901F
:10B1000043F64400C4F20200016841F4804101604A
:10B11000006800F4804007900798FFE70B9820F044
:10B12000030043F60801C4F20101405808900B984F
:10B1300000F0030081000F2000FA01F10898884315
:10B1400008900D980021C4F20201884203D1FFE764
:10B15000002006905EE00D9840F20041C4F202012A
:10B16000884203D1FFE70120059050E00D9840F69A
:10B170000001C4F20201884203D1FFE702200490DB
:10B1800042E00D9840F60041C4F20201884203D12A
:10B19000FFE70320039034E00D9841F20001C4F270
:10B1A0000201884203D1FFE70420029026E00D98B7
:10B1B00041F20041C4F20201884203D1FFE70520B9
:10B1C000019018E00D9841F60001C4F20201884296
:10B1D00003D1FFE7062000900AE00D9941F60042F6
:10B1E000C4F202020820914208BF07200090FFE746
:10B1F00000980190FFE701980290FFE70298039002
:10B20000FFE703980490FFE704980590FFE705988F
:10B210000690FFE70698C0B20B9901F00301890080
:10B2200000FA01F108980843089008980B9921F05A
:10B23000030143F60802C4F20102885043F60040BD
:10B24000C4F20100006808900999089888430890A2
:10B250000C988079C00728B1FFE70999089808433E
:10B260000890FFE7089843F60041C4F20101086026
:10B2700043F60440C4F20100006808900999089858
:10B28000884308900C9880798007002805D5FFE74F
:10B290000999089808430890FFE7089843F6044185
:10B2A000C4F20101086043F60840C4F201000068DE
:10B2B000089009990898884308900C988079C006EE
:10B2C000002805D5FFE70999089808430890FFE78B
:10B2D000089843F60841C4F20101086043F60C40A7
:10B2E000C4F2010000680890099908988843089002
:10B2F0000C9880798006002805D5FFE70999089801
:10B3000008430890FFE7089843F60C41C4F2010196
:10B310000860FFE7FFE7FFE70B9801300B904BE574
:10B320000EB080BD80B582B00190ADF80210BDF8BE
:10B33000020020B1FFE7002008B9FFE708E044F66B
:10B34000A270C0F602004FF4BD7112F07DF9FFE764
:10B3500001980069BDF80210084204D0FFE70120FF
:10B360008DF8010003E000208DF80100FFE79DF853
:10B37000010002B080BD000080B582B00190ADF840
:10B3800002108DF80120BDF8020020B1FFE7002077
:10B3900008B9FFE708E044F6A270C0F6020040F2E8
:10B3A0009B1112F051F9FFE79DF8010028B1FFE76A
:10B3B0009DF80100012801D1FFE708E044F6A270E2
:10B3C000C0F602004FF4CE7112F03EF9FFE79DF88F
:10B3D000010028B1FFE7BDF802000199886105E08E
:10B3E000BDF80200000401998861FFE702B080BD4A
:10B3F00049F20460C2F200000068704780B58EB068
:10B400000C900C9820B9FFE701208DF8370002E27C
:10B410000C98006845F20041C4F20001884212D045
:10B42000FFE70C98006845F60001C4F2000188426D
:10B4300009D0FFE70C98006845F60041C4F200010E
:10B44000884201D1FFE708E045F2F600C0F60200AD
:10B4500040F2BF1112F0F8F8FFE70C98406850B1C5
:10B46000FFE70C98406841F68021C0F2060188424F
:10B4700001D8FFE708E045F2F600C0F602004FF4FD
:10B48000E07112F0E1F8FFE70C98806830B1FFE757
:10B490000C988068B0F5804F01D1FFE708E045F2D5
:10B4A000F600C0F6020040F2C11112F0CDF8FFE73D
:10B4B0000C98C068800A08B9FFE708E045F2F6007A
:10B4C000C0F602004FF4E17112F0BEF8FFE70C98ED
:10B4D0000069B0F5804F06D0FFE70C980069B0F521
:10B4E000404F01D1FFE708E045F2F600C0F6020048
:10B4F00040F2C31112F0A8F8FFE70C98406928B198
:10B50000FFE70C984069012801D1FFE708E045F208
:10B51000F600C0F602004FF4E27112F095F8FFE772
:10B520000C9880696FF0FE01084201D1FFE708E046
:10B5300045F2F600C0F6020040F2C51112F084F8A0
:10B54000FFE70C98C06928B1FFE70C98C069402854
:10B5500001D1FFE708E045F2F600C0F602004FF423
:10B56000E37112F071F8FFE70C98006A28B1FFE769
:10B570000C98006A802801D1FFE708E045F2F60048
:10B58000C0F6020040F2C71112F05EF8FFE70C9817
:10B5900090F83D0040B9FFE70C99002081F83C008D
:10B5A0000C9800F03DF9FFE70C99242081F83D004C
:10B5B0000C980168086820F0010008600C98016888
:10B5C000086840F4004008600C980168086820F49E
:10B5D0000040086001F054FE0A900C98406848F260
:10B5E000A061C0F2010188420BD8FFE70A9948F236
:10B5F0008042C0F21E020020914238BF0120099013
:10B600000AE00A9940F60012C0F23D020020914281
:10B6100038BF01200990FFE70998012804D1FFE70E
:10B6200001208DF83700F6E00A984DF68361C4F2E8
:10B630001B31A0FB0110800C0B900C980068406837
:10B6400020F03F000B9908430C99096848600C985A
:10B650000068006A20F03F0008900C98406848F2AB
:10B66000A061C0F20101884204D8FFE70B980130C5
:10B6700007900EE00B984FF49671484344F6D3516F
:10B68000C1F26201A0FB0101012000EB91100790C3
:10B69000FFE70898079908430C99096808620C9815
:10B6A0000068C0694CF6FF71884306900C984068AA
:10B6B00048F2A061C0F2010188421FD8FFE70A9852
:10B6C00001380C9949684900B0FBF1F001306FF383
:10B6D0001F30032803D8FFE7042005900BE00A98E9
:10B6E00001380C9949684900B0FBF1F001306FF363
:10B6F0001F300590FFE7059804904CE00C98806897
:10B7000068B9FFE70A9801380C99496801EB4101D3
:10B71000B0FBF1F001306FF31F3003900DE00A9899
:10B7200001380C99496819225143B0FBF1F00130FE
:10B73000042161F31F300390FFE70398000518B957
:10B74000FFE70120029023E00C98806868B9FFE7CA
:10B750000A9801380C99496801EB4101B0FBF1F0FE
:10B7600001306FF31F3001900DE00A9801380C99F9
:10B77000496819225143B0FBF1F00130042161F313
:10B780001F300190FFE7019840F400400290FFE76E
:10B7900002980490FFE70698049908430C990968F9
:10B7A000C8610C980068006820F0C0000C9B196804
:10B7B000DA691B6A1A43104308600C9800688068B5
:10B7C00048F2FF3188430C9A1168D36812691A4312
:10B7D000104388600C980068C06820F0FF000C9B44
:10B7E00019685A699B691A431043C8600C9801682C
:10B7F000086840F0010008600C99002008640C9A69
:10B80000202182F83D100C9908630C9981F83E00C4
:10B810008DF83700FFE79DF837000EB080BD0000BF
:10B8200080B594B0139000201290119010900F905A
:10B830000E901398006845F20041C4F2000188425E
:10B8400035D1FFE7FFE700200D9043F63000C4F24A
:10B850000200016841F002010160006800F002008E
:10B860000D900D98FFE74FF440700E9012200F904E
:10B8700001201090032011900420129040F200400B
:10B88000C4F202000EA9FFF7BDF9FFE700200C90FB
:10B8900043F64000C4F20200016841F40011016067
:10B8A000006800F400100C900C98FFE7FBE0139880
:10B8B000006845F60001C4F2000188425FD1FFE74D
:10B8C000FFE700200B9043F63000C4F2020001684D
:10B8D00041F020010160006800F020000B900B98FF
:10B8E000FFE703200E9012210F910121109111907A
:10B8F0000420129041F20040C4F202000EA9FFF7AA
:10B9000081F9FFE700200A9043F64000C4F20200EC
:10B91000016841F480010160006800F480000A9031
:10B920000A98FFE741F25470C2F20000069046F216
:10B93000B801C4F2020101604FF060614160402132
:10B9400081600021C1604FF48062026141618161C8
:10B95000C1614FF4003202624162FEF769FC18B126
:10B96000FFE7FBF7C1F9FFE7FFE7139841F25471D6
:10B97000C2F20001416313988863FFE792E01398D5
:10B98000006845F60041C4F20001884240F0898019
:10B99000FFE7FFE70020099043F63000C4F2020001
:10B9A000016841F004010160006800F004000990A2
:10B9B0000998FFE7FFE70020089043F63000C4F243
:10B9C0000200016841F001010160006800F001001F
:10B9D00008900898FFE74FF400700E901220019035
:10B9E0000F900120029010900320039011900420EA
:10B9F0000490129040F60000C4F202000EA90591D6
:10BA0000FFF700F9DDF804C0029B039A049805993A
:10BA10004FF4807ECDF838E0CDF83CC01093119201
:10BA200012900020C4F20200FFF7ECF8FFE70020BC
:10BA3000079043F64000C4F20200016841F400019F
:10BA40000160006800F4000007900798FFE741F2EA
:10BA5000B470C2F20000009046F24001C4F202014C
:10BA600001604FF0C061416000218160C1604FF40E
:10BA70008062026141618161C16101624162FEF7E0
:10BA8000D7FB18B1FFE7FBF72FF9FFE7FFE71398A4
:10BA900041F2B471C2F20001816313988863FFE739
:10BAA000FFE7FFE7FFE714B080BD000040F2E020B1
:10BAB000C2F20000027849F20461C2F20001086893
:10BAC000104408607047000080B543F60041C4F29E
:10BAD0000201086840F400700860086840F4806063
:10BAE0000860086840F480700860032000F0D0F817
:10BAF0000F2000F005F800F03BF8002080BD0000AA
:10BB000080B582B0009040F22800C2F200000068C8
:10BB100040F2E021C2F200010A784FF47A71B1FBE1
:10BB2000F2F1B0FBF1F003F005FB20B1FFE70120DB
:10BB30008DF8070018E000980F280DD8FFE700994E
:10BB40004FF0FF30002200F06FF8009840F2E4213F
:10BB5000C2F20001086003E001208DF8070003E055
:10BB600000208DF80700FFE79DF8070002B080BDB8
:10BB700080B582B0FFE70020019043F64400C4F294
:10BB80000200016841F480410160006800F48040D7
:10BB900001900198FFE7FFE70020009043F6400086
:10BBA000C4F20200016841F080510160006800F0B9
:10BBB000805000900098FFE76FF001000F210022F5
:10BBC00000F032F802B080BD80B582B08DF8070079
:10BBD0009DF90700002801D4FFE707E045F21300B4
:10BBE000C0F60200CE2111F02FFDFFE79DF90700FE
:10BBF00011F08CFC02B080BD80B582B08DF80700DA
:10BC00009DF90700002801D4FFE707E045F2130083
:10BC1000C0F60200BE2111F017FDFFE79DF90700F5
:10BC200011F090FC02B080BD80B586B08DF8170091
:10BC3000049103920020029003980F2801D8FFE797
:10BC400007E045F21300C0F60200AA2111F0FCFC47
:10BC5000FFE704980F2801D8FFE707E045F213003B
:10BC6000C0F60200AB2111F0EFFCFFE711F082FCFF
:10BC700002909DF91700019002980499039A07F029
:10BC8000C5FE0146019811F07DFC06B080BD0000A4
:10BC900080B582B001900198072810D0FFE7019885
:10BCA00006280CD0FFE70198052808D0FFE7019887
:10BCB000042804D0FFE70198032801D1FFE707E03B
:10BCC00045F21300C0F60200922111F0BDFCFFE71F
:10BCD000019811F09BFC02B080BD000082B0019081
:10BCE0008DF8031002B0704782B00190ADF80210D9
:10BCF000BDF80200019909684862002002B070474F
:10BD000084B003908DF80B10ADF8082003980068FC
:10BD1000406A00909DF80B0048B9FFE7BDF8081095
:10BD2000009840EA014003990968886233E003986B
:10BD30000068816A009800EB1140009000208DF8A7
:10BD40000700FFE79DF807009DF80B1001398842B6
:10BD500013D2FFE7039800689DF8071000EB8100FD
:10BD6000D0F80411009800EB11400090FFE79DF817
:10BD7000070001308DF80700E4E7BDF808100098CF
:10BD800040EA0140039909689DF80B2001EB82010C
:10BD9000C1F80001FFE7002004B0704780B582B011
:10BDA00001900198D0F804040FF014FB02B080BD9C
:10BDB00080B582B001908DF80310019AD2F8040486
:10BDC0009DF80310C1EBC10302EB8302926C0FF0EC
:10BDD000DFF902B080BD000080B582B001908DF81F
:10BDE0000310019AD2F804049DF80310C1EBC103BB
:10BDF00002EB8302D2F808220FF070FA02B080BD85
:10BE000080B582B001900198D0F804040FF0E8FAF0
:10BE100002B080BD80B584B002908DF807109DF807
:10BE20000700000600280FD5FFE702989DF80710CD
:10BE300001F00F01C1EBC10100EB81003C3000902B
:10BE40000099012048700FE002989DF8071001F05A
:10BE50000F01C1EBC10100EB810000F5FE70009005
:10BE6000009900204870FFE79DF8070000F00F00E0
:10BE700000990870FFE7029890F8BC03012804D1EC
:10BE8000FFE702208DF80F0014E00299012081F8ED
:10BE9000BC03FFE7FFE702980068009910F064FA1E
:10BEA000FFE70299002081F8BC03FFE700208DF82E
:10BEB0000F00FFE79DF80F0004B080BD80B584B08F
:10BEC00002908DF807109DF8070000F00F0002990E
:10BED0004968884204D9FFE701208DF80F004DE042
:10BEE0009DF80700000600280FD5FFE702989DF88F
:10BEF000071001F00F01C1EBC10100EB81003C30E4
:10BF000000900099012048700FE002989DF80710FA
:10BF100001F00F01C1EBC10100EB810000F5FE70E3
:10BF20000090009900204870FFE700990020887079
:10BF30009DF8070000F00F0000990870FFE70298D5
:10BF400090F8BC03012804D1FFE702208DF80F0010
:10BF500014E00299012081F8BC03FFE7FFE7029893
:10BF60000068009910F084FDFFE70299002081F835
:10BF7000BC03FFE700208DF80F00FFE79DF80F00DE
:10BF800004B080BD82B001908DF8031001989DF837
:10BF9000031001F00F01C1EBC10100EB8100D0F8EB
:10BFA000140202B07047000080B586B004908DF88E
:10BFB0000F10ADF80C208DF80B3000208DF80A0022
:10BFC0009DF80F00000600280FD5FFE704989DF8A4
:10BFD0000F1001F00F01C1EBC10100EB81003C30FB
:10BFE00001900199012048700FE004989DF80F100E
:10BFF00001F00F01C1EBC10100EB810000F5FE7003
:10C000000190019900204870FFE79DF80F0000F0B3
:10C010000F0001990870BDF80C00019988609DF827
:10C020000B000199C8700198407820B1FFE7019991
:10C030000878C880FFE79DF80B00022804D1FFE7CD
:10C04000019900200871FFE7FFE7049890F8BC030E
:10C05000012804D1FFE702208DF8170015E00499AC
:10C06000012081F8BC03FFE7FFE70498006801990D
:10C0700010F036F8FFE70499002081F8BC03FFE7D1
:10C080009DF80A008DF81700FFE79DF8170006B02D
:10C0900080BD000080B586B005908DF81310039226
:10C0A000029305989DF8131001F00F01C1EBC10137
:10C0B00000EB810000F5FE70019003980199C860C3
:10C0C000029801994861019900208861019948709E
:10C0D0009DF8130000F00F000199087005980069A1
:10C0E000012804D1FFE7039801990861FFE79DF853
:10C0F0001300000738B9FFE7059A10680199127C10
:10C1000010F06EFB06E0059A10680199127C10F0A1
:10C1100053FDFFE7002006B080BD000080B584B06D
:10C1200002908DF807109DF8070000F00F000299AB
:10C130004968884204D9FFE701208DF80F0058E0D4
:10C140009DF80700000600280FD5FFE702989DF82C
:10C15000071001F00F01C1EBC10100EB81003C3081
:10C1600000900099012048700DE002989DF807109A
:10C17000C1EBC10100EB810000F5FE700090009959
:10C1800000204870FFE70099012088709DF80700A3
:10C1900000F00F0000990870FFE7029890F8BC03C8
:10C1A000012804D1FFE702208DF80F0021E0029959
:10C1B000012081F8BC03FFE7FFE7029800680099BF
:10C1C00010F0A6FC9DF80700000740B9FFE7029AAF
:10C1D0001068117C02F5717210F0FAFBFFE7FFE7BF
:10C1E0000299002081F8BC03FFE700208DF80F00C2
:10C1F000FFE79DF80F0004B080BD000080B586B059
:10C2000005908DF813100392029305989DF8131072
:10C2100001F00F01C1EBC10100EB81003C30019046
:10C2200003980199C860029801994861019900201A
:10C2300088610199012048709DF8130000F00F00FB
:10C240000199087005980069012804D1FFE7039857
:10C2500001990861FFE79DF81300000738B9FFE76F
:10C26000059A10680199127C10F0BAFA06E0059A56
:10C2700010680199127C10F09FFCFFE7002006B0C7
:10C2800080BD000080B58CB00B900B9800680A90C0
:10C290000A9809900B98006810F0C0FE002840F042
:10C2A0001A83FFE70B98006810F024FF08B9FFE736
:10C2B00011E30B98006810F01DFF8007002807D5D8
:10C2C000FFE70B980168486900F002004861FFE74A
:10C2D0000B98006810F00EFFC006002862D5FFE73B
:10C2E0000B980168886920F0100088610A98006A3C
:10C2F00003900B98039901F00F01C1EBC10100EB12
:10C30000810000F5FE700290039800F4F011022005
:10C31000B0EB514F23D1FFE7BDF80C0047F6F071A9
:10C3200008421BD0FFE70A980299C968039AC2F332
:10C330000A1210F0EDFE039847F6F07100EA0103CF
:10C34000029AD06800EB1310D060039800EA010253
:10C350000299886900EB12108861FFE71BE00398DF
:10C3600000F4F0110620B0EB514F12D1FFE70A980C
:10C370000B9901F57171082210F0CAFE039847F677
:10C38000F07100EA01020299886900EB12108861DD
:10C3900000E0FFE7FFE70B980168886940F01000B4
:10C3A0008861FFE70B98006810F0A4FE00030028E6
:10C3B00070D5FFE7002005900B98006810F048FE4C
:10C3C0000790FFE70798002863D0FFE79DF81C005F
:10C3D000C007002856D0FFE70B9800689DF814109E
:10C3E00010F070FE06909DF81800C00760B1FFE7DE
:10C3F0000998059900EB41110120C1F8080B0B9831
:10C40000059907F087FBFFE79DF818000007002853
:10C410000CD5FFE70998059900EB41110820C1F8F8
:10C42000080B0B98059907F02FFBFFE79DF8180004
:10C43000C006002808D5FFE70998059900EB4111CF
:10C440001020C1F8080BFFE79DF8180080060028AF
:10C4500008D5FFE70998059900EB41112020C1F8A4
:10C46000080BFFE79DF819008006002809D5FFE7B3
:10C470000998059900EB41114FF40050C1F8080BE1
:10C48000FFE7FFE7059801300590079840080790FF
:10C4900098E7FFE70B98006810F02CFE4003002897
:10C4A00040F1AC80FFE70B98006810F0BFFD0790EB
:10C4B00000200590FFE70798002800F09E80FFE726
:10C4C0009DF81C00C007002800F09080FFE70B9843
:10C4D00000689DF8141010F0CDFD06909DF818002E
:10C4E000C00700283ED0FFE7059800F00F010120AB
:10C4F00000FA01F10491049B099AD2F83418994387
:10C50000C2F834180999059A01EB4211C1F80809DB
:10C510000B98006901281FD1FFE70B980599C1EB23
:10C52000C10100EB81014A6C886C10448864059855
:10C5300088B9FFE70B980599C1EBC10100EB8100B9
:10C54000006D40B9FFE70B99086801F57172012190
:10C5500010F03EFAFFE7FFE70B989DF81410FFF785
:10C5600027FCFFE79DF818000007002808D5FFE723
:10C570000998059900EB41110820C1F80809FFE767
:10C580009DF81800C006002808D5FFE7099805990E
:10C5900000EB41111020C1F80809FFE79DF81800D1
:10C5A0004006002808D5FFE70998059900EB4111DE
:10C5B0004020C1F80809FFE79DF81800800700280F
:10C5C00008D5FFE70998059900EB41110220C1F851
:10C5D0000809FFE79DF818000006002805D5FFE7C9
:10C5E0000B98059907F088FBFFE7FFE705980130F6
:10C5F00005900798400807905DE7FFE70B980068F3
:10C6000010F078FDC00F00B3FFE70999D1F80408D6
:10C6100020F00100C1F804080B9890F8F4030128F9
:10C6200008D1FFE70B98002180F8F4130B98FFF76F
:10C6300055FB03E00B9800F061FBFFE70B980168E6
:10C64000486900F000404861FFE70B98006810F06F
:10C6500051FD0005002811D5FFE70998D0F808081A
:10C66000C00720B1FFE70B9800F0D6FBFFE70B985F
:10C670000168486900F400604861FFE70B980068B2
:10C6800010F038FDC004002840F19080FFE70999C0
:10C69000D1F8040820F00100C1F804080B980068E4
:10C6A000102110F06BFC00200890FFE708980B9910
:10C6B000496888423BD2FFE70998089900EB41118D
:10C6C0004FF67F30C1F808090999089A01EB421228
:10C6D000D2F8001921F40011C2F800190999089A3A
:10C6E00001EB4212D2F8001941F00061C2F80019C2
:10C6F0000999089A01EB4211C1F8080B09980899A9
:10C7000000EB4111D1F8000B20F40010C1F8000B30
:10C710000998089900EB4111D1F8000B40F0006036
:10C72000C1F8000BFFE7089801300890BEE70999AF
:10C73000D1F81C0840F00110C1F81C080B98006BE0
:10C7400078B1FFE70999D1F8840840F00B00C1F8EF
:10C7500084080999D1F8440840F00B00C1F8440856
:10C760000FE00999D1F8140842F22B021043C1F8E6
:10C7700014080999D1F8100840F00B00C1F810080E
:10C78000FFE70999D1F8000820F4FE60C1F800081D
:10C790000B9A1068117C02F5717210F019F90B9860
:10C7A0000168486900F480504861FFE70B98006811
:10C7B00010F0A0FC800400281FD5FFE70B9800684C
:10C7C0000FF0FEFC0B98006810F002FC0B99C8609B
:10C7D0000B980068019000F04DFD014601980B9AFE
:10C7E000127B10F01BFD0B9800F05EFA0B980168AD
:10C7F000486900F400504861FFE70B98006810F0AA
:10C8000079FC000700280AD5FFE70B9800F080FAB2
:10C810000B980168486900F008004861FFE70B9831
:10C82000006810F067FCC00200280ED5FFE700206A
:10C8300005900B989DF8141000F050F80B980168C3
:10C84000486900F480104861FFE70B98006810F019
:10C8500051FC800200280ED5FFE7002005900B98C0
:10C860009DF8141000F048F80B980168486900F42E
:10C8700000104861FFE70B98006810F03BFC400097
:10C8800000280AD5FFE70B98FFF788FA0B98016894
:10C89000486900F080404861FFE70B98006810F09D
:10C8A00029FC4007002815D5FFE70B980068406871
:10C8B00003909DF80C004007002804D5FFE70B9873
:10C8C000FFF79EFAFFE7039A0B9801684868104348
:10C8D0004860FFE7FFE70CB080BD000080B582B084
:10C8E00001908DF803100198D0F804049DF803100E
:10C8F0000EF008FE02B080BD80B582B001908DF8C8
:10C9000003100198D0F804049DF803100EF026FEE1
:10C9100002B080BD2DE9F04F97B01590159820B961
:10C92000FFE701208DF85B0060E115980068B0F129
:10C93000A04F08D0FFE7159800680021C4F2040159
:10C94000884201D1FFE707E044F6BB60C0F6020071
:10C95000872110F079FEFFE715980068149015986C
:10C9600090F8BD0340B9FFE71599002081F8BC039A
:10C97000159800F041F9FFE71599032081F8BD03F0
:10C980001498C06BC005002804D4FFE71599002057
:10C990000861FFE7159800680FF018FF15981090D0
:10C9A0000168119141688268C368D0F810C0446979
:10C9B0008569C669076AD0F82480D0F82890D0F835
:10C9C0002CA0D0F830B0D0F834E068461290C0F80F
:10C9D00024E01198DDF848E0CEF820B0CEF81CA095
:10C9E000CEF81890CEF81480CEF81070CEF80C6007
:10C9F000CEF80850CEF80440CEF800C00FF0F6FB99
:10CA000040B1FFE71599022081F8BD0301208DF8A0
:10CA10005B00EBE01598006800210F9110F0A0FB7F
:10CA20000F988DF84F00FFE79DF84F001599496862
:10CA3000884245D2FFE715989DF84F10C1EBC10120
:10CA400000EB8101012081F83D009DF84F00159910
:10CA5000C0EBC00201EB820181F83C009DF84F0061
:10CA60001599C0EBC00201EB8201A1F842001598B4
:10CA70009DF84F10C1EBC10100EB8101002081F84E
:10CA80003F0015999DF84F20C2EBC20201EB8201D5
:10CA9000486415999DF84F20C2EBC20201EB820158
:10CAA000886415999DF84F20C2EBC20201EB820108
:10CAB0000865FFE79DF84F0001308DF84F00B3E7A0
:10CAC00000208DF84F00FFE79DF84F001599496849
:10CAD00088423ED2FFE715989DF84F10C1EBC10187
:10CAE00000EB8101002081F8FD019DF84F10159A9F
:10CAF000C1EBC10302EB830282F8FC1115999DF88A
:10CB00004F20C2EBC20201EB820181F8FF011599AF
:10CB10009DF84F20C2EBC20201EB8201C1F8040272
:10CB200015999DF84F20C2EBC20201EB8201C1F8BA
:10CB3000080215999DF84F20C2EBC20201EB820159
:10CB4000C1F81002FFE79DF84F0001308DF84F004B
:10CB5000BAE715980C9001680D9141688268C36826
:10CB6000D0F810C044698569C669076AD0F8248086
:10CB7000D0F82890D0F82CA0D0F830B0D0F834E01D
:10CB800068460E90C0F824E00D98DDF838E0CEF845
:10CB900020B0CEF81CA0CEF81890CEF81480CEF8B5
:10CBA0001070CEF80C60CEF80850CEF80440CEF8E5
:10CBB00000C00FF0A9FC40B1FFE71599022081F8F1
:10CBC000BD0301208DF85B0010E0159900200B904B
:10CBD00081F838001599012081F8BD031598006887
:10CBE0000FF07CFC0B988DF85B00FFE79DF85B0075
:10CBF00017B0BDE8F08F000080B58AB00990002022
:10CC00000890079006900590049009980068B0F18C
:10CC1000A04F47D1FFE7FFE70020039043F6300025
:10CC2000C4F20200016841F001010160006800F0F7
:10CC3000010003900398FFE74FF4C05004900220D6
:10CC4000059000200690032007900A2008900020FD
:10CC5000C4F2020004A9FDF7D5FFFFE743F6340153
:10CC6000C4F20201086840F080000860FFE700207D
:10CC7000029043F64400C4F20200016841F480418E
:10CC80000160006800F4804002900298FFE7FFE72F
:10CC90004320019005210022FEF7C6FF0198FEF710
:10CCA000ABFFFFE70AB080BD80B582B001900120E4
:10CCB0008DF803000198C06820B9FFE700208DF8C7
:10CCC00003000CE00198C068022804D1FFE70120AE
:10CCD0008DF8030002E0FAF707F8FFE7FFE7019895
:10CCE000D0F804049DF803100EF036FD0198D0F83A
:10CCF00004040EF0A7FC02B080BD000080B582B035
:10CD000001900198D0F804040EF0ECFC02B080BD54
:10CD100080B582B001900198D0F804040EF0F4FCC4
:10CD200002B080BD80B584B002908DF80710FFE797
:10CD3000029890F8BC03012804D1FFE702208DF887
:10CD40000F001AE00299012081F8BC03FFE7FFE71A
:10CD50009DF80700029981F83800029800689DF854
:10CD6000071010F02DFAFFE70299002081F8BC03AC
:10CD7000FFE700208DF80F00FFE79DF80F0004B0DB
:10CD800080BD000080B582B001900199D1F8040403
:10CD900001F571710EF00AFD02B080BD80B584B05E
:10CDA0000290029800680190FFE7029890F8BC0397
:10CDB000012804D1FFE702208DF80F0027E0029937
:10CDC000012081F8BC03FFE7FFE70298806A012891
:10CDD0000BD1FFE702988069012806D0FFE701998F
:10CDE000886B40F480308863FFE70298006810F099
:10CDF00095F8029800680FF05BFBFFE702990020AE
:10CE000081F8BC03FFE700208DF80F00FFE79DF8D5
:10CE10000F0004B080BD000080B582B00190019881
:10CE2000D0F804040EF044FD01980168D1F8000E1A
:10CE300040F00100C1F8000E0198006A48B1FFE718
:10CE40004EF61051CEF20001086840F0060008606E
:10CE5000FFE702B080BD000080B584B00290019170
:10CE6000029820B9FFE701208DF80F00FDE102983C
:10CE7000006830B1FFE7029800680F2801D8FFE78B
:10CE800008E044F6F360C0F602004FF4177110F0AA
:10CE9000DBFBFFE70198E0B1FFE70198012818D01C
:10CEA000FFE70198022814D0FFE70198032810D06B
:10CEB000FFE7019804280CD0FFE70198052808D067
:10CEC000FFE70198062804D0FFE70198072801D161
:10CED000FFE708E044F6F360C0F6020040F25D218F
:10CEE00010F0B2FBFFE7019843F60041C4F20201E3
:10CEF000096801F00701884212D9FFE7019943F65A
:10CF00000040C4F202000170006800F007000199BF
:10CF1000884204D0FFE701208DF80F00A5E1FFE76C
:10CF2000029800788007002860D5FFE70298007813
:10CF30004007002809D5FFE743F60801C4F20201C3
:10CF4000086840F4E0500860FFE7029800780007A6
:10CF5000002809D5FFE743F60801C4F2020108687A
:10CF600040F460400860FFE70298806840B3FFE744
:10CF700002988068802823D0FFE702988068902874
:10CF80001ED0FFE702988068A02819D0FFE702981A
:10CF90008068B02814D0FFE702988068C0280FD0BE
:10CFA000FFE702988068D0280AD0FFE702988068DF
:10CFB000E02805D0FFE702988068F02801D1FFE75C
:10CFC00008E044F6F360C0F602004FF4207110F060
:10CFD0003BFBFFE743F60801C4F20201086820F0BA
:10CFE000F000029A926810430860FFE70298007808
:10CFF000C007002800F08C80FFE70298406878B1F5
:10D00000FFE70298406801280AD0FFE702984068CD
:10D01000022805D0FFE702984068032801D1FFE706
:10D0200008E044F6F360C0F6020040F2872110F0F9
:10D030000BFBFFE702984068012811D1FFE743F698
:10D040000000C4F20200006800F400310020B0EBE0
:10D05000514F04D1FFE701208DF80F0005E12CE0CE
:10D0600002984068022805D0FFE70298406803282C
:10D0700011D1FFE743F60000C4F20200006800F09F
:10D0800000710020B0EB516F04D1FFE701208DF853
:10D090000F00EAE010E043F60000C4F2020000686E
:10D0A00000F002010020B0EB510F04D1FFE7012096
:10D0B0008DF80F00D9E0FFE7FFE743F60801C4F25F
:10D0C0000201086820F00300029A526810430860C9
:10D0D000FEF78EF90090FFE743F60800C4F2020065
:10D0E000006800F00C0002994968B0EB810F0ED087
:10D0F000FFE7FEF77DF90099401A41F28931884235
:10D1000004D3FFE703208DF80F00AEE0E4E7FFE76C
:10D11000019843F60041C4F20201096801F00701D9
:10D12000884212D2FFE7019943F60040C4F20200A0
:10D130000170006800F007000199884204D0FFE701
:10D1400001208DF80F0090E0FFE70298007840077B
:10D15000002832D5FFE70298C068C0B1FFE7029807
:10D16000C068B0F5805F12D0FFE70298C068B0F5E4
:10D17000A05F0CD0FFE70298C068B0F5C05F06D092
:10D18000FFE70298C068B0F5E05F01D1FFE708E073
:10D1900044F6F360C0F6020040F2C52110F054FAE4
:10D1A000FFE743F60801C4F20201086820F4E050EA
:10D1B000029AD26810430860FFE7029800780007DF
:10D1C000002833D5FFE702980069C0B1FFE7029855
:10D1D0000069B0F5805F12D0FFE702980069B0F5F2
:10D1E000A05F0CD0FFE702980069B0F5C05F06D0E1
:10D1F000FFE702980069B0F5E05F01D1FFE708E0C2
:10D2000044F6F360C0F602004FF4337110F01CFADC
:10D21000FFE743F60801C4F20201086820F4604009
:10D22000029A126940EAC2000860FFE700F04CF879
:10D2300043F60801C4F202010968C9B20A0944F2BE
:10D24000D061C0F60201895CC84040F22801C2F2F8
:10D250000001086040F2E420C2F200000068FEF71E
:10D260004FFC00208DF80F00FFE79DF80F0004B081
:10D2700080BD000040F22800C2F200000068704744
:10D2800080B5FFF7F7FF43F60801C4F20201096811
:10D29000C1F3822244F2E061C0F60201895CC84019
:10D2A00080BD000080B5FFF7E5FF43F60801C4F23A
:10D2B0000201096889B24A0B44F2E061C0F602013A
:10D2C000895CC84080BD000080B586B00020059014
:10D2D00004900390029043F60800C4F20200006834
:10D2E00000F00C000146019140B1FFE701980428CD
:10D2F0000AD0FFE7019808280CD04FE042F2004026
:10D30000C0F2F40002904FE041F60030C0F2B700E6
:10D31000029049E043F60400C4F20200016801F003
:10D320003F01059100684002002813D5FFE743F64E
:10D330000400C4F202000068C0F3881041F6003116
:10D34000C0F2B701A0FB0101059A0023F2F738FFF4
:10D35000049012E043F60400C4F202000068C0F337
:10D36000881042F20041C0F2F401A0FB0101059ACD
:10D370000023F2F725FF0490FFE743F60400C4F210
:10D380000200006800F44031022000EBD13003902D
:10D3900004980399B0FBF1F0029005E042F20040DE
:10D3A000C0F2F4000290FFE7029806B080BD0000D2
:10D3B00080B586B00490049828B9FFE701208DF865
:10D3C000170000F048BC049800680F2801D8FFE758
:10D3D00007E044F6F360C0F60200E82110F034F9EB
:10D3E000FFE704980078C007002800F0BE80FFE740
:10D3F0000498406860B1FFE704984068B0F5803F4A
:10D4000006D0FFE704984068B0F5A02F01D1FFE7F0
:10D4100007E044F6F360C0F60200ED2110F014F9C5
:10D42000FFE743F60800C4F20200006800F00C00B9
:10D43000042813D0FFE743F60800C4F20200006896
:10D4400000F00C0008281ED1FFE743F60400C4F2E8
:10D45000020000684002002815D5FFE743F60000EF
:10D46000C4F20200006800F400310020B0EB514F1C
:10D4700008D0FFE70498406820B9FFE701208DF845
:10D480001700E8E370E0FFE704984068B0F5803FDC
:10D4900009D1FFE743F60001C4F20201086840F435
:10D4A0008030086020E004984068B0F5A02F0DD1CE
:10D4B000FFE743F60001C4F20201086840F480204F
:10D4C0000860086840F4803008600CE043F6000112
:10D4D000C4F20201086820F480300860086820F473
:10D4E00080200860FFE7FFE7FFE704984068E8B1A5
:10D4F000FFE7FDF77DFF0390FFE743F60000C4F26E
:10D500000200006800F400310020B0EB514F0CD154
:10D51000FFE7FDF76DFF0399401A652804D3FFE785
:10D5200003208DF8170096E3E7E71CE0FDF760FFA6
:10D530000390FFE743F60000C4F20200006800F425
:10D5400000310020B0EB514F0CD0FFE7FDF750FF4A
:10D550000399401A652804D3FFE703208DF81700CC
:10D5600079E3E7E7FFE7FFE7FFE704980078800744
:10D57000002840F1B880FFE70498C06828B1FFE7B1
:10D580000498C068012801D1FFE708E044F6F36081
:10D59000C0F6020040F21F1110F056F8FFE70498A1
:10D5A00000691F2801D8FFE708E044F6F360C0F6E1
:10D5B00002004FF4907110F047F8FFE743F60800BF
:10D5C000C4F20200006810F00C0F13D0FFE743F61E
:10D5D0000800C4F20200006800F00C0008282CD1FA
:10D5E000FFE743F60400C4F202000068400200288E
:10D5F00023D4FFE743F60000C4F20200006800F005
:10D6000002010020B0EB510F09D0FFE70498C06879
:10D61000012804D0FFE701208DF817001BE343F633
:10D620000001C4F20201086820F0F800049A1269AF
:10D6300040EAC2000860FFE754E00498C06870B395
:10D64000FFE70021C4F2472101200860FDF7D0FE6A
:10D650000390FFE743F60000C4F20200006800F008
:10D6600002010020B0EB510F0CD1FFE7FDF7C0FE27
:10D670000399401A032804D3FFE703208DF817000D
:10D68000E9E2E7E743F60001C4F20201086820F08E
:10D69000F800049A126940EAC200086021E0002103
:10D6A000C4F2472100200860FDF7A2FE0390FFE7C7
:10D6B00043F60000C4F20200006800F002010020FE
:10D6C000B0EB510F0CD0FFE7FDF792FE0399401A23
:10D6D000032804D3FFE703208DF81700BBE2E7E738
:10D6E000FFE7FFE7FFE704980078000700285ED512
:10D6F000FFE70498406928B1FFE7049840690128D2
:10D7000001D1FFE708E044F6F360C0F602004FF4F1
:10D71000B0710FF099FFFFE70498406918B3FFE775
:10D7200040F68061C4F2472101200860FDF760FEE9
:10D730000390FFE743F67400C4F20200006800F0B3
:10D7400002010020B0EB510F0CD1FFE7FDF750FEB6
:10D750000399401A032804D3FFE703208DF817002C
:10D7600079E2E7E722E040F68061C4F24721002039
:10D770000860FDF73DFE0390FFE743F67400C4F236
:10D780000200006800F002010020B0EB510F0CD045
:10D79000FFE7FDF72DFE0399401A032804D3FFE7A6
:10D7A00003208DF8170056E2E7E7FFE7FFE704984C
:10D7B00000784007002840F1E680FFE700208DF860
:10D7C00007000498806850B1FFE70498806801283A
:10D7D00005D0FFE704988068052801D1FFE708E03D
:10D7E00044F6F360C0F602004FF4C6710FF02CFF50
:10D7F000FFE743F64000C4F202000068C0000028C2
:10D8000015D4FFE7FFE70020009043F64000C4F284
:10D810000200016841F080510160006800F0805012
:10D8200000900098FFE701208DF80700FFE747F21E
:10D830000000C4F200000068C005002822D4FFE701
:10D8400047F20001C4F20001086840F480700860EB
:10D85000FDF7CEFD0390FFE747F20000C4F20000A1
:10D860000068C00500280CD4FFE7FDF7C1FD03994F
:10D87000401A032804D3FFE703208DF81700EAE1DC
:10D88000EAE7FFE7FFE704988068012809D1FFE78E
:10D8900043F67001C4F20201086840F0010008601C
:10D8A0001FE00498806805280DD1FFE743F670015A
:10D8B000C4F20201086840F004000860086840F003
:10D8C000010008600CE043F67001C4F20201086830
:10D8D00020F001000860086820F004000860FFE7FD
:10D8E000FFE7FFE704988068F8B1FFE7FDF780FDE8
:10D8F0000390FFE743F67000C4F20200006800F0F6
:10D9000002010020B0EB510F0ED1FFE7FDF770FDD3
:10D910000399401A41F28931884204D3FFE703207A
:10D920008DF8170097E1E5E71EE0FDF761FD039034
:10D93000FFE743F67000C4F20200006800F0020145
:10D940000020B0EB510F0ED0FFE7FDF751FD03991A
:10D95000401A41F28931884204D3FFE703208DF851
:10D96000170078E1E5E7FFE79DF80700012809D1F6
:10D97000FFE743F64001C4F20201086820F080503E
:10D980000860FFE7FFE70498806950B1FFE704985B
:10D990008069012805D0FFE704988069022801D139
:10D9A000FFE708E044F6F360C0F6020040F2CF1152
:10D9B0000FF04AFEFFE704988069002800F04781D5
:10D9C000FFE743F60800C4F20200006800F00C0014
:10D9D000082800F0F080FFE704988069022840F0F2
:10D9E000C780FFE70498C06930B1FFE70498C069B9
:10D9F000B0F5800F01D1FFE708E044F6F360C0F610
:10DA000002004FF4EC710FF01FFEFFE70498006A6C
:10DA10003F2801D8FFE708E044F6F360C0F60200B3
:10DA200040F2D9110FF010FEFFE70498406A322847
:10DA300007D3FFE70498406AB0F5D87F01D8FFE725
:10DA400008E044F6F360C0F602004FF4ED710FF009
:10DA5000FBFDFFE70498806A02280FD0FFE70498D7
:10DA6000806A04280AD0FFE70498806A062805D057
:10DA7000FFE70498806A082801D1FFE708E044F630
:10DA8000F360C0F6020040F2DB110FF0DDFDFFE7AE
:10DA90000498C06A022806D3FFE70498C06A0F28DA
:10DAA00001D8FFE708E044F6F360C0F602004FF447
:10DAB000EE710FF0C9FDFFE76021C4F2472100209D
:10DAC0000860FDF795FC0390FFE743F60000C4F201
:10DAD0000200006800F000710020B0EB516F0CD024
:10DAE000FFE7FDF785FC0399401A032804D3FFE7FD
:10DAF00003208DF81700AEE0E7E70499C869D1F874
:10DB000020C04B6A8A6A40EA0C0040EA8310D203C4
:10DB10004FF6FF739A43A2F580321043C96A40EA78
:10DB2000016043F60401C4F2020108606021C4F2FE
:10DB3000472101200860FDF75BFC0390FFE743F6F7
:10DB40000000C4F20200006800F000710020B0EB99
:10DB5000516F0CD1FFE7FDF74BFC0399401A0328E6
:10DB600004D3FFE703208DF8170074E0E7E721E016
:10DB70006021C4F2472100200860FDF739FC0390C2
:10DB8000FFE743F60000C4F20200006800F00071F5
:10DB90000020B0EB516F0CD0FFE7FDF729FC039993
:10DBA000401A032804D3FFE703208DF8170052E042
:10DBB000E7E7FFE74AE004988069012804D1FFE71E
:10DBC00001208DF8170046E043F60400C4F202007D
:10DBD0000068029004988069012831D0FFE702981C
:10DBE00000F480000499C969884229D1FFE70298AE
:10DBF00000F03F000499096A884221D1FFE70298AA
:10DC000047F6C07108400499496AB0EB811F17D1EB
:10DC1000FFE7029800F440300499896AC9034FF67F
:10DC2000FF729143A1F58031884209D1FFE7029844
:10DC300000F070600499C96AB0EB016F04D0FFE78F
:10DC400001208DF8170006E0FFE7FFE7FFE700205F
:10DC50008DF81700FFE79DF8170006B080BD0000A3
:10DC600080B582B00090009820B9FFE701208DF8C0
:10DC700007002EE00098006840F60001C5F206019A
:10DC8000884201D1FFE707E045F22E10C0F60200FE
:10DC9000A3210FF0D9FCFFE70098407938B9FFE7DE
:10DCA000009900200871009800F018F8FFE700992B
:10DCB0000220487100980168086840F0040008607C
:10DCC0000099012048710099002088608DF80700B4
:10DCD000FFE79DF8070002B080BD000082B0019010
:10DCE0000198006840F60001C5F20601884212D191
:10DCF000FFE7FFE70020009043F63400C4F2020083
:10DD0000016841F040010160006800F040000090AF
:10DD10000098FFE7FFE702B07047000080B582B0CF
:10DD20000190019808F03CFC8DF803009DF8030079
:10DD300003281BD0FFE7019808F032FC014640F2AF
:10DD40004040C2F2000000EB4110806968B1FFE77B
:10DD5000019808F025FC014640F24040C2F2000064
:10DD600000EB411080698047FFE7FFE702B080BD0C
:10DD700080B584B00290029820B9FFE701208DF8A9
:10DD80000F00D2E10298006843F20001C4F20101E1
:10DD9000884212D0FFE70298006843F60001C4F2FF
:10DDA0000001884209D0FFE70298006843F600416D
:10DDB000C4F20001884201D1FFE708E045F2661095
:10DDC000C0F602004FF4A1710FF03EFCFFE702988D
:10DDD000406830B1FFE702984068B0F5827F01D11A
:10DDE000FFE708E045F26610C0F6020040F243117A
:10DDF0000FF02AFCFFE70298806860B1FFE7029805
:10DE00008068B0F5806F06D0FFE702988068B0F5B3
:10DE1000004F01D1FFE708E045F26610C0F60200AE
:10DE20004FF4A2710FF010FCFFE70298C068B0F544
:10DE3000006F04D0FFE70298C06808B9FFE708E068
:10DE400045F26610C0F6020040F245110FF0FCFBEF
:10DE5000FFE702988069B0F5007F0AD0FFE70298DB
:10DE6000806930B1FFE702988069B0F5802F01D159
:10DE7000FFE708E045F26610C0F602004FF4A37118
:10DE80000FF0E2FBFFE70298C06918B3FFE70298C2
:10DE9000C06908281ED0FFE70298C069102819D071
:10DEA000FFE70298C069182814D0FFE70298C069FC
:10DEB00020280FD0FFE70298C06928280AD0FFE782
:10DEC0000298C069302805D0FFE70298C069382859
:10DED00001D1FFE708E045F26610C0F6020040F20B
:10DEE00047110FF0B1FBFFE70298006A28B1FFE786
:10DEF0000298006A802801D1FFE708E045F2661029
:10DF0000C0F602004FF4A4710FF09EFBFFE70298E9
:10DF1000406A28B1FFE70298406A102801D1FFE764
:10DF200008E045F26610C0F6020040F249110FF019
:10DF30008BFBFFE70298406A002863D1FFE7029855
:10DF4000006928B1FFE702980069022801D1FFE7C4
:10DF500008E045F26610C0F602004FF4A6710FF01B
:10DF600073FBFFE70298406928B1FFE70298406918
:10DF7000012801D1FFE708E045F26610C0F6020073
:10DF800040F24D110FF060FBFFE702984068B0F5DA
:10DF9000827F32D1FFE70298C06918B3FFE7029889
:10DFA000C06908281ED0FFE70298C069102819D060
:10DFB000FFE70298C069182814D0FFE70298C069EB
:10DFC00020280FD0FFE70298C06928280AD0FFE771
:10DFD0000298C069302805D0FFE70298C069382848
:10DFE00001D1FFE708E045F26610C0F6020040F2FA
:10DFF00051110FF029FBFFE703E002990020C861EF
:10E00000FFE736E00298C06918B3FFE70298C069DD
:10E0100008281ED0FFE70298C069102819D0FFE732
:10E020000298C069182814D0FFE70298C069202818
:10E030000FD0FFE70298C06928280AD0FFE70298AE
:10E04000C069302805D0FFE70298C069382801D19F
:10E05000FFE708E045F26610C0F6020040F25B11EF
:10E060000FF0F2FAFFE70299002008610299486177
:10E07000FFE7029900208862029890F8510040B9A9
:10E08000FFE70299002081F85000029800F052F852
:10E09000FFE70299022081F85100029801680868A0
:10E0A00020F040000860029A019211685068D2F88E
:10E0B00008C0D36800F482700CF4044C604403F48C
:10E0C00000631844136903F002031844536903F012
:10E0D00001031844936903F400731844D36903F0EF
:10E0E00038031844136A03F080031843926A02F459
:10E0F000005210430860029A508B00F0040011682F
:10E10000526A02F010021044486002980168C8691F
:10E1100020F40060C861029900204865029A01213C
:10E1200082F851108DF80F00FFE79DF80F0004B042
:10E1300080BD000080B592B01190002010900F902B
:10E140000E900D900C901198006843F20001C4F2FB
:10E150000101884240F0B680FFE7FFE700200B9006
:10E1600043F64400C4F20200016841F480510160AA
:10E17000006800F480500B900B98FFE7FFE7002049
:10E180000A9043F63000C4F20200016841F0020137
:10E190000160006800F002000A900A98FFE7FFE7BC
:10E1A0000020099043F63000C4F20200016841F0FB
:10E1B00001010160006800F0010009900998FFE783
:10E1C00018200C90022001900D90012002900E90DA
:10E1D000032003900F9005200490109040F200401F
:10E1E000C4F202000CA90591FCF70CFDDDF804C097
:10E1F000029B039A049805994FF0800ECDF830E009
:10E20000CDF834C00E930F9210900020C4F202009B
:10E21000FCF7F8FC41F61400C2F20000069046F24A
:10E220004041C4F2020101604FF0C0614160002131
:10E230008160C1604FF48062026141618161C161AE
:10E240004FF4403202624162FBF7F2FF18B1FFE780
:10E25000F8F74AFDFFE7FFE7119841F61401C2F213
:10E260000001C16411988863FFE741F67400C2F2AF
:10E270000000009046F25841C4F2020101604FF0E4
:10E28000C0614160402181600021C1604FF4806223
:10E29000026141618161C1614FF4003202624162F9
:10E2A000FBF7C6FF18B1FFE7F8F71EFDFFE7FFE732
:10E2B000119841F67401C2F20001816411988863DB
:10E2C000FFE73EE01198006843F60001C4F2000148
:10E2D000884235D1FFE7FFE70020089043F6400071
:10E2E000C4F20200016841F480410160006800F45A
:10E2F000804008900898FFE7FFE70020079043F66A
:10E300003000C4F20200016841F0020101600068BF
:10E3100000F0020007900798FFE74FF460400C9070
:10E3200002200D9001200E9003200F9005201090E8
:10E3300040F20040C4F202000CA9FCF763FCFFE7C6
:10E34000FFE712B080BD000080B588B0069005914F
:10E35000ADF81220039300208DF80700069840685E
:10E36000B0F5827F16D1FFE70698806890B9FFE785
:10E370000699042081F851000698059ABDF81230DC
:10E380000399EC46CCF80010114600F089FB8DF89B
:10E390001F00EDE0FFE7069890F85000012804D137
:10E3A000FFE702208DF81F00E2E00699012081F8C6
:10E3B0005000FFE7FFE7FDF71BF80290069890F882
:10E3C0005100012804D0FFE702208DF80700C0E0CB
:10E3D000059820B1FFE7BDF8120020B9FFE7012042
:10E3E0008DF80700B5E00699042081F851000699E0
:10E3F000002048650599069A9163BDF81210069AA7
:10E400009187BDF81210069AD1870699086306997C
:10E4100088860699C886069908640699486406980D
:10E420008068B0F5004F0DD1FFE7069801680868D5
:10E4300020F04000086006980168086820F48040D9
:10E440000860FFE706980068006800F04000402878
:10E4500007D0FFE706980168086840F040000860B0
:10E46000FFE70698C06880BBFFE7FFE70698C08F0C
:10E4700050B3FFE7069800688068C00778B1FFE7EF
:10E4800006980068007B0699896B08700699886B6E
:10E49000013088630699C88F0138C88713E0FCF7FC
:10E4A000A7FF0299401A0399884204D3FFE7039813
:10E4B000013018B9FFE7039820B9FFE703208DF872
:10E4C000070046E0FFE7D1E72FE0FFE70698C08F9F
:10E4D00050B3FFE7069800688068C00778B1FFE78F
:10E4E00006980068C0680699896B08800699886B51
:10E4F000023088630699C88F0138C88713E0FCF79B
:10E5000077FF0299401A0399884204D3FFE70398E2
:10E51000013018B9FFE7039820B9FFE703208DF811
:10E52000070016E0FFE7D1E7FFE706980399029A94
:10E5300007F072FF20B1FFE7069920204865FFE74A
:10E540000698406D20B1FFE701208DF80700FFE736
:10E55000FFE70699012081F85100FFE706990020A6
:10E5600081F85000FFE79DF807008DF81F00FFE7D6
:10E570009DF81F0008B080BD80B584B00290019165
:10E58000ADF8022000208DF801000298C06C08B19F
:10E59000FFE708E045F26610C0F6020040F2CA61EB
:10E5A0000FF052F8FFE70298806810BBFFE702986F
:10E5B0004068B0F5827F1CD1FFE70299042081F802
:10E5C00051000298806C08B1FFE708E045F2661040
:10E5D000C0F6020040F2D1610FF036F8FFE7029872
:10E5E000019ABDF80230114600F01CFC8DF80F00B6
:10E5F000A8E0FFE7029890F85000012804D1FFE757
:10E6000002208DF80F009DE00299012081F8500052
:10E61000FFE7FFE7029890F85100012804D0FFE7D8
:10E6200002208DF8010082E0019820B1FFE7BDF8DB
:10E63000020020B9FFE701208DF8010077E0029980
:10E64000042081F851000299002048650199029A3E
:10E650009163BDF80210029A9187BDF80210029AE8
:10E66000D1870299086402994864029988860299C0
:10E67000C88602988068B0F5004F0DD1FFE7029878
:10E680000168086820F04000086002980168086886
:10E6900020F480400860FFE70298C16C46F2BD207C
:10E6A000C0F6010008640298C16C46F2ED20C0F685
:10E6B0000100C8630298C16C46F28920C0F60100CF
:10E6C000C8640298C16C00200865029B19689A6BA7
:10E6D000D86C0C31DB8FFCF747F860B1FFE702998B
:10E6E000486D40F01000486501208DF80100029946
:10E6F00081F851001BE002980068006800F04000BB
:10E70000402807D0FFE702980168086840F0400001
:10E710000860FFE702980168486840F02000486000
:10E7200002980168486840F001004860FFE7FFE791
:10E730000299002081F85000FFE79DF801008DF854
:10E740000F00FFE79DF80F0004B080BD80B582B0D8
:10E750000190019807F024FF8DF803009DF8030055
:10E7600003281BD0FFE7019807F01AFF014640F28B
:10E770004040C2F2000000EB4110406868B1FFE782
:10E78000019807F00DFF014640F24040C2F2000040
:10E7900000EB411040688047FFE7FFE702B080BD13
:10E7A00080B582B00190019807F0FAFE8DF8030061
:10E7B0009DF8030003281BD0FFE7019807F0F0FE47
:10E7C000014640F24040C2F2000000EB41100069F7
:10E7D00068B1FFE7019807F0E3FE014640F24040D0
:10E7E000C2F2000000EB411000698047FFE7FFE73D
:10E7F00002B080BD80B588B006900591ADF81220BA
:10E80000039300208DF807000698806830B1FFE779
:10E8100006988068B0F5004F01D1FFE708E045F2A7
:10E820006610C0F6020040F20A310EF00DFFFFE75D
:10E83000FFE7069890F85000012804D1FFE7022076
:10E840008DF81F0028E10699012081F85000FFE7AC
:10E85000FFE7FCF7CDFD0290BDF81200ADF8040013
:10E86000069890F85100012804D0FFE702208DF8A7
:10E87000070002E1059820B1FFE7BDF8120020B9BA
:10E88000FFE701208DF80700F7E00699032081F8E3
:10E8900051000699002048650599069A1163BDF854
:10E8A0001210069A9186BDF81210069AD186069922
:10E8B0008863069988870699C887069948640699E7
:10E8C000086406988068B0F5004F0DD1FFE7069800
:10E8D0000168086820F04000086006980168086830
:10E8E00040F480400860FFE706980068006800F088
:10E8F0004000402807D0FFE706980168086840F00C
:10E9000040000860FFE70698C068B0F5006F47D187
:10E91000FFE70698406828B1FFE7BDF8040001282A
:10E920000ED1FFE706980168006B0088C860069961
:10E93000086B023008630699C88E0138C886FFE765
:10E94000FFE70698C08E50B3FFE70698006880681E
:10E95000800700280ED5FFE706980168006B008845
:10E96000C8600699086B023008630699C88E0138A2
:10E97000C88613E0FCF73CFD0299401A03998842CF
:10E9800004D3FFE70398013018B9FFE7039820B9D3
:10E99000FFE703208DF807006FE0FFE7D1E746E0CF
:10E9A0000698406828B1FFE7BDF8040001280ED1A1
:10E9B000FFE706980168006B007808730699086BFA
:10E9C000013008630699C88E0138C886FFE7FFE763
:10E9D0000698C08E50B3FFE70698006880688007ED
:10E9E00000280ED5FFE706980168006B00780873D1
:10E9F0000699086B013008630699C88E0138C886ED
:10EA000013E0FCF7F5FC0299401A0399884204D3FD
:10EA1000FFE70398013018B9FFE7039820B9FFE733
:10EA200003208DF8070028E0FFE7D1E7FFE706980D
:10EA30000399029A07F062FD20B1FFE706992020B2
:10EA40004865FFE70698806870B9FFE7FFE7002098
:10EA5000009006980068C06800900698006880687A
:10EA600000900098FFE7FFE70698406D20B1FFE7B0
:10EA700001208DF80700FFE7FFE70699012081F8E4
:10EA80005100FFE70699002081F85000FFE79DF84C
:10EA900007008DF81F00FFE79DF81F0008B080BD3C
:10EAA00080B58EB0DDF840C00C900B910A92ADF8A5
:10EAB00026300120059000208DF813000C98806806
:10EAC00008B9FFE708E045F26610C0F6020040F220
:10EAD0007E410EF0B9FDFFE7FFE70C9890F850007B
:10EAE000012804D1FFE702208DF8370095E10C9949
:10EAF000012081F85000FFE7FFE7FCF779FC069062
:10EB00000C9890F851008DF81F000C984068089000
:10EB1000BDF82600ADF824009DF81F00012812D092
:10EB2000FFE70898B0F5827F09D1FFE70C9880686D
:10EB300028B9FFE79DF81F00042804D0FFE7022052
:10EB40008DF813005AE10B9838B1FFE70A9820B10D
:10EB5000FFE7BDF8260020B9FFE701208DF813007C
:10EB60004CE10C9890F85100042805D0FFE70C996F
:10EB7000052081F85100FFE70C99002048650A99AB
:10EB80000C9A9163BDF826100C9AD187BDF8261017
:10EB90000C9A91870B990C9A1163BDF826100C9A68
:10EBA000D186BDF826100C9A91860C9908640C99B0
:10EBB00048640C980068006800F04000402807D0C6
:10EBC000FFE70C980168086840F040000860FFE724
:10EBD0000C98C068B0F5006F76D1FFE70C984068DC
:10EBE00028B1FFE7BDF8240001280ED1FFE70C98FB
:10EBF0000168006B0088C8600C99086B02300863DC
:10EC00000C99C88E0138C886FFE7FFE70C98C18EC3
:10EC10000120029039B9FFE70C98C08F002818BF77
:10EC200001200290FFE70298C00700284BD0FFE7C1
:10EC30000C98006880688007002818D5FFE70C98BA
:10EC4000C08EA0B1FFE70598012810D1FFE70C980E
:10EC50000168006B0088C8600C99086B023008637B
:10EC60000C99C88E0138C88600200590FFE70C98E3
:10EC700000688068C007A8B1FFE70C98C08F88B112
:10EC8000FFE70C980068C0680C99896B08800C99A4
:10EC9000886B023088630C99C88F0138C8870120BF
:10ECA0000590FFE7FCF7A4FB0699401A10998842EB
:10ECB00008D3FFE71098013020B1FFE703208DF85B
:10ECC00013009BE0A2E778E00C98406828B1FFE7CA
:10ECD000BDF8240001280ED1FFE70C980168006BF5
:10ECE000007808730C99086B013008630C99C88E82
:10ECF0000138C886FFE7FFE70C98C18E012001901C
:10ED000039B9FFE70C98C08F002818BF0120019087
:10ED1000FFE70198C00700284ED0FFE70C98006875
:10ED200080688007002818D5FFE70C98C08EA0B136
:10ED3000FFE70598012810D1FFE70C980168006BE8
:10ED4000007808730C99086B013008630C99C88E21
:10ED50000138C88600200590FFE70C98006880689D
:10ED6000C007A8B1FFE70C98C08F88B1FFE70C98E7
:10ED70000068C0680C99896B08700C99886B013029
:10ED800088630C99C88F0138C88701200590FFE778
:10ED9000FCF72EFB0699401A1099884204D3FFE72E
:10EDA0001098013018B9FFE7109820B9FFE7032049
:10EDB0008DF8130022E09FE7FFE70C981099069A60
:10EDC00007F09CFB38B1FFE701208DF813000C9988
:10EDD0002020486512E00C98806870B9FFE7FFE7D3
:10EDE000002003900C980068C06803900C9800689D
:10EDF000806803900398FFE7FFE7FFE70C99012085
:10EE000081F85100FFE70C99002081F85000FFE7DE
:10EE10009DF813008DF83700FFE79DF837000EB01E
:10EE200080BD000080B588B0069005910492ADF8D1
:10EE30000E3000208DF806000698C06C08B1FFE780
:10EE400008E045F26610C0F602004FF4E8610EF0EB
:10EE5000FBFBFFE70698806C08B1FFE708E045F28E
:10EE60006610C0F6020040F241710EF0EDFBFFE7C4
:10EE70000698806808B9FFE708E045F26610C0F61A
:10EE8000020040F244710EF0DFFBFFE7FFE7069857
:10EE900090F85000012804D1FFE702208DF81F00F0
:10EEA000EFE00699012081F85000FFE7FFE70698A0
:10EEB00090F851008DF807000698406802909DF880
:10EEC0000700012812D0FFE70298B0F5827F09D130
:10EED000FFE70698806828B9FFE79DF80700042837
:10EEE00004D0FFE702208DF80600BFE0059838B196
:10EEF000FFE7049820B1FFE7BDF80E0020B9FFE757
:10EF000001208DF80600B1E0069890F85100042821
:10EF100005D0FFE70699052081F85100FFE7069923
:10EF2000002048650599069A1163BDF80E10069AEF
:10EF30009186BDF80E10069AD1860499069A9163BF
:10EF4000BDF80E10069A9187BDF80E10069AD1876B
:10EF50000699086406994864069890F851000428B8
:10EF60000FD1FFE70698C16C46F2BD20C0F6010044
:10EF700008640698C16C46F2ED20C0F60100C86333
:10EF80000EE00698C16C46F2D520C0F60100086478
:10EF90000698C16C46F29130C0F60100C863FFE7E5
:10EFA0000698C16C46F28920C0F60100C864069834
:10EFB000C16C00200865069B19689A6BD86C0C31EF
:10EFC000DB8FFBF7D1FB60B1FFE70699486D40F09E
:10EFD0001000486501208DF80600069981F851005F
:10EFE00044E006980168486840F0010048600698CF
:10EFF000816C002008640699896CC8630699896C45
:10F00000C8640699896C0865069B1A68196B986C28
:10F010000C32DB8EFBF7A8FB60B1FFE70699486D69
:10F0200040F01000486501208DF80600069981F82F
:10F0300051001BE006980068006800F0400040287E
:10F0400007D0FFE706980168086840F040000860B4
:10F05000FFE706980168486840F02000486006987D
:10F060000168486840F002004860FFE7FFE7069942
:10F07000002081F85000FFE79DF806008DF81F0082
:10F08000FFE79DF81F0008B080BD000080B582B08A
:10F090000190019807F084FA8DF803009DF80300B1
:10F0A00003281BD0FFE7019807F07AFA014640F2E7
:10F0B0004040C2F2000000EB4110806868B1FFE7F9
:10F0C000019807F06DFA014640F24040C2F200009C
:10F0D00000EB411080688047FFE7FFE702B080BD8A
:10F0E00080B582B00190019807F05AFA8DF80300BC
:10F0F0009DF8030003281BD0FFE7019807F050FAA2
:10F10000014640F24040C2F2000000EB411040696D
:10F1100068B1FFE7019807F043FA014640F240402A
:10F12000C2F2000000EB411040698047FFE7FFE7B3
:10F1300002B080BD80B582B00190019807F0D8FF81
:10F1400002B080BD81B0009001B0704781B00090E6
:10F1500001B0704780B584B002900191002000900A
:10F16000029800680021C4F20101884209D0FFE73B
:10F170000298006840F20041C4F20101884201D1C6
:10F18000FFE708E045F2D610C0F6020040F2B47185
:10F190000EF05AFAFFE701980068B0F5006F04D04E
:10F1A000FFE70198006808B9FFE708E045F2D610CC
:10F1B000C0F6020040F2B5710EF046FAFFE7019882
:10F1C0004068B0F5806F04D0FFE70198406808B947
:10F1D000FFE708E045F2D610C0F6020040F2B67133
:10F1E0000EF032FAFFE70198806890B1FFE70198CE
:10F1F0008068B0F5807F0CD0FFE701988068B0F59B
:10F20000007F06D0FFE701988068B0F5407F01D10C
:10F21000FFE708E045F2D610C0F6020040F2B771F1
:10F220000EF012FAFFE70198C068FF2801D8FFE747
:10F2300008E045F2D610C0F602004FF4F7610EF078
:10F2400003FAFFE701980069B0F5805F04D0FFE79B
:10F250000198006908B9FFE708E045F2D610C0F64A
:10F26000020040F2B9710EF0EFF9FFE70198406932
:10F2700030B1FFE701984069B0F5005F01D1FFE7C9
:10F2800008E045F2D610C0F6020040F2BA710EF066
:10F29000DBF9FFE70198C069B0F5804F04D0FFE7C4
:10F2A0000198C06908B9FFE708E045F2D610C0F63A
:10F2B000020040F2BB710EF0C7F9FFE7FFE70298CA
:10F2C00090F83C00012804D1FFE702208DF80F00E0
:10F2D00044E00299012081F83C00FFE7FFE7009835
:10F2E00020F0FF000199C96808430090009820F4BD
:10F2F00040700199896808430090009820F480606C
:10F300000199496808430090009820F40060019931
:10F31000096808430090009820F480500199096919
:10F3200008430090009820F400500199496908436F
:10F330000090009820F480400199C969084300902A
:10F340000098029909684864FFE70299002081F853
:10F350003C00FFE700208DF80F00FFE79DF80F004D
:10F3600004B080BD80B586B0049003910498006815
:10F370000021C4F2010188423CD0FFE704980068F4
:10F38000B0F1804F36D0FFE70498006840F20041AA
:10F39000C4F2000188422DD0FFE70498006840F6CF
:10F3A0000001C4F20001884224D0FFE704980068FD
:10F3B00040F60041C4F2000188421BD0FFE70498E8
:10F3C000006841F20001C4F20001884212D0FFE758
:10F3D0000498006841F20041C4F20001884209D05B
:10F3E000FFE70498006840F20041C4F2010188423E
:10F3F00001D1FFE708E045F2D610C0F6020040F266
:10F4000077710EF021F9FFE70398006818B3FFE762
:10F410000398006810281ED0FFE703980068202892
:10F4200019D0FFE703980068302814D0FFE703984D
:10F43000006840280FD0FFE70398006850280AD0E2
:10F44000FFE703980068602805D0FFE7039800688D
:10F45000702801D1FFE708E045F2D610C0F602009F
:10F460004FF4EF610EF0F0F8FFE703984068802852
:10F4700004D0FFE70398406808B9FFE708E045F2C9
:10F48000D610C0F6020040F279710EF0DDF8FFE709
:10F49000FFE7049890F83C00012804D1FFE7022020
:10F4A0008DF817007EE00499012081F83C00FFE709
:10F4B000FFE70499022081F83D0004980068406845
:10F4C00002900498006880680190029820F0700013
:10F4D00002900398016802980843029002980499E8
:10F4E00009684860049800680021C4F2010188425C
:10F4F0003CD0FFE704980068B0F1804F36D0FFE7BA
:10F500000498006840F20041C4F2000188422DD006
:10F51000FFE70498006840F60001C4F20001884249
:10F5200024D0FFE70498006840F60041C4F20001CF
:10F5300088421BD0FFE70498006840F20041C4F203
:10F540000101884212D0FFE70498006844F20001EC
:10F55000C4F20101884209D0FFE70498006841F62F
:10F560000001C4F2000188420ED1FFE7019820F0AB
:10F570008000019003984168019808430190019828
:10F58000049909688860FFE70499012081F83D002B
:10F59000FFE70499002081F83C00FFE700208DF888
:10F5A0001700FFE79DF8170006B080BD80B582B058
:10F5B0000090009820B9FFE701208DF8070012E1C4
:10F5C000009800680021C4F20101884272D0FFE770
:10F5D00000980068B0F1804F6CD0FFE70098006899
:10F5E00040F20041C4F20001884263D0FFE7009876
:10F5F000006840F60001C4F2000188425AD0FFE7DB
:10F600000098006840F60041C4F20001884251D0E1
:10F61000FFE70098006841F20001C4F2000188424F
:10F6200048D0FFE70098006841F20041C4F20001B1
:10F6300088423FD0FFE70098006840F20041C4F2E2
:10F640000101884236D0FFE70098006844F20001CB
:10F65000C4F2010188422DD0FFE70098006844F20F
:10F660000041C4F20101884224D0FFE700980068FD
:10F6700044F60001C4F2010188421BD0FFE7009864
:10F68000006841F60001C4F20001884212D0FFE791
:10F690000098006841F60041C4F20001884209D098
:10F6A000FFE70098006842F20001C4F200018842BE
:10F6B00001D1FFE708E045F29E10C0F6020040F2DB
:10F6C00013110DF0C1FFFFE700988068A0B1FFE7BC
:10F6D0000098806810280FD0FFE7009880682028E5
:10F6E0000AD0FFE700988068402805D0FFE700981F
:10F6F0008068602801D1FFE708E045F29E10C0F65F
:10F7000002004FF48A710DF09FFFFFE70098006937
:10F7100060B1FFE700980069B0F5807F06D0FFE791
:10F7200000980069B0F5007F01D1FFE708E045F2DD
:10F730009E10C0F6020040F215110DF085FFFFE7A4
:10F740000098806928B1FFE700988069802801D17E
:10F75000FFE708E045F29E10C0F602004FF48B71FF
:10F760000DF072FFFFE7009890F83D0040B9FFE709
:10F770000099002081F83C00009800F039F8FFE77C
:10F780000099022081F83D00009951F8040B07F020
:10F7900063FD0099012081F84600FFE700990120F0
:10F7A00081F83E00009981F83F00009981F84000FF
:10F7B000009981F84100FFE7FFE70099012081F8F7
:10F7C0004200009981F84300009981F844000099B3
:10F7D00081F84500FFE70099012081F83D000020F5
:10F7E0008DF80700FFE79DF8070002B080BD00001C
:10F7F00080B58AB00990099800680021C4F201011F
:10F8000088421BD1FFE7FFE70020089043F6440041
:10F81000C4F20200016841F001010160006800F0DB
:10F82000010008900898FFE71820019005210022A8
:10F83000FCF7FAF90198FCF7DFF9B0E009980068E5
:10F8400040F20041C4F20001884212D1FFE7FFE715
:10F850000020079043F64000C4F20200016841F026
:10F8600002010160006800F0020007900798FFE7BE
:10F8700094E00998006840F60001C4F20001884253
:10F8800012D1FFE7FFE70020069043F64000C4F2E4
:10F890000200016841F004010160006800F004000A
:10F8A00006900698FFE778E00998006840F6004166
:10F8B000C4F20001884212D1FFE7FFE70020059063
:10F8C00043F64000C4F20200016841F00801016003
:10F8D000006800F0080005900598FFE75CE00998D3
:10F8E000006841F20041C4F2000188421BD1FFE7E9
:10F8F000FFE70020049043F64000C4F202000168D4
:10F9000041F020010160006800F02000049004989C
:10F91000FFE73720009005210022FCF785F90098C9
:10F92000FCF76AF937E00998006840F20041C4F238
:10F930000101884212D1FFE7FFE70020039043F660
:10F940004400C4F20200016841F002010160006855
:10F9500000F0020003900398FFE71BE0099800689D
:10F9600044F20041C4F20101884212D1FFE7FFE7EF
:10F970000020029043F64400C4F20200016841F402
:10F9800000310160006800F4003002900298FFE747
:10F99000FFE7FFE7FFE7FFE7FFE7FFE7FFE70AB063
:10F9A00080BD000080B584B00290029800680021FC
:10F9B000C4F20101884272D0FFE702980068B0F1FA
:10F9C000804F6CD0FFE70298006840F20041C4F21B
:10F9D0000001884263D0FFE70298006840F600010A
:10F9E000C4F2000188425AD0FFE70298006840F64E
:10F9F0000041C4F20001884251D0FFE7029800683C
:10FA000041F20001C4F20001884248D0FFE70298A9
:10FA1000006841F20041C4F2000188423FD0FFE794
:10FA20000298006840F20041C4F20101884236D0D9
:10FA3000FFE70298006844F20001C4F20101884225
:10FA40002DD0FFE70298006844F20041C4F20101A2
:10FA5000884224D0FFE70298006844F60001C4F20F
:10FA6000010188421BD0FFE70298006841F60001BF
:10FA7000C4F20001884212D0FFE70298006841F604
:10FA80000041C4F20001884209D0FFE702980068F3
:10FA900042F20001C4F20001884201D1FFE708E010
:10FAA00045F29E10C0F6020040F2CF110DF0CCFDE1
:10FAB000FFE7029890F83D00012804D0FFE70120FD
:10FAC0008DF80F006AE00299022081F83D0002984B
:10FAD0000168C86840F00100C86002980068002111
:10FAE000C4F2010188423CD0FFE702980068B0F1FF
:10FAF000804F36D0FFE70298006840F20041C4F220
:10FB0000000188422DD0FFE70298006840F600010E
:10FB1000C4F20001884224D0FFE70298006840F652
:10FB20000041C4F2000188421BD0FFE70298006840
:10FB300040F20041C4F20101884212D0FFE702986E
:10FB4000006844F20001C4F20101884209D0FFE7D5
:10FB50000298006841F60001C4F20001884212D107
:10FB6000FFE702980068806800F0070001900198A4
:10FB7000062807D0FFE702980168086840F00100F6
:10FB80000860FFE706E002980168086840F001009D
:10FB90000860FFE700208DF80F00FFE79DF80F00D9
:10FBA00004B080BD80B586B004900391FFE704984F
:10FBB00090F83C00012805D1FFE702208DF81700DE
:10FBC00000F069BC0499012081F83C00FFE7FFE7E1
:10FBD0000499022081F83D0003980068B0F5805F29
:10FBE0002DD0FFE703980068B0F5005F27D0FFE74E
:10FBF0000398006818B3FFE70398006810281ED028
:10FC0000FFE703980068202819D0FFE703980068F1
:10FC1000302814D0FFE70398006840280FD0FFE792
:10FC20000398006850280AD0FFE70398006860280E
:10FC300005D0FFE703980068702801D1FFE708E0CE
:10FC400045F29E10C0F6020041F222410DF0FCFC8C
:10FC5000FFE70498006880680290029820F077001F
:10FC60000290029820F47F4002900298049909685B
:10FC70008860039800680190002800F0A883FFE7DF
:10FC80000198102800F0A383FFE70198202800F0D6
:10FC90009E83FFE70198302800F09983FFE70198E1
:10FCA000402800F00883FFE70198502800F0EB811E
:10FCB000FFE70198602800F07282FFE70198702842
:10FCC00000F09180FFE70198B0F5805F06D0FFE774
:10FCD0000198B0F5005F00F03A81CDE30498006828
:10FCE0000021C4F20101884272D0FFE70498006845
:10FCF000B0F1804F6CD0FFE70498006840F20041FB
:10FD0000C4F20001884263D0FFE70498006840F61F
:10FD10000001C4F2000188425AD0FFE7049800684D
:10FD200040F60041C4F20001884251D0FFE7049838
:10FD3000006841F20001C4F20001884248D0FFE7A8
:10FD40000498006841F20041C4F2000188423FD0AB
:10FD5000FFE70498006840F20041C4F201018842C4
:10FD600036D0FFE70498006844F20001C4F20101B4
:10FD700088422DD0FFE70498006844F20041C4F2A5
:10FD80000101884224D0FFE70498006844F600018E
:10FD9000C4F2010188421BD0FFE70498006841F6D5
:10FDA0000001C4F20001884212D0FFE70498006805
:10FDB00041F60041C4F20001884209D0FFE70498EF
:10FDC000006842F20001C4F20001884201D1FFE75D
:10FDD00008E045F29E10C0F6020041F22E410DF0FF
:10FDE00033FCFFE749E3049800680021C4F20101F5
:10FDF00088423CD0FFE704980068B0F1804F36D0CD
:10FE0000FFE70498006840F20041C4F20001884214
:10FE10002DD0FFE70498006840F60001C4F200010D
:10FE2000884224D0FFE70498006840F60041C4F2FD
:10FE3000000188421BD0FFE70498006840F20041AF
:10FE4000C4F20101884212D0FFE70498006844F22E
:10FE50000001C4F20101884209D0FFE7049800685C
:10FE600041F60001C4F20001884201D1FFE708E039
:10FE700045F29E10C0F6020041F235410DF0E4FB60
:10FE8000FFE70398806890B1FFE703988068B0F5BA
:10FE9000805F0CD0FFE703988068B0F5005F06D064
:10FEA000FFE703988068B0F5405F01D1FFE708E005
:10FEB00045F29E10C0F6020041F238410DF0C4FB3D
:10FEC000FFE703984068B0F5004F12D0FFE70398B2
:10FED000406870B1FFE70398406850B1FFE70398AE
:10FEE0004068022805D0FFE7039840680A2801D13E
:10FEF000FFE708E045F29E10C0F6020041F23941EA
:10FF00000DF0A2FBFFE70398C0680F2801D8FFE7B8
:10FF100008E045F29E10C0F6020041F23A410DF0B1
:10FF200093FBFFE704980068039B5A689968DB68B5
:10FF300007F000FB0498006880680290029840F087
:10FF400077000290029804990968886095E2049805
:10FF500000680021C4F2010188422AD0FFE704981A
:10FF60000068B0F1804F24D0FFE70498006840F2A9
:10FF70000041C4F2000188421BD0FFE704980068EA
:10FF800040F60001C4F20001884212D0FFE7049855
:10FF9000006840F60041C4F20001884209D0FFE742
:10FFA0000498006840F20041C4F20101884201D186
:10FFB000FFE708E045F29E10C0F6020041F24D4115
:10FFC0000DF042FBFFE70398806890B1FFE70398CC
:10FFD0008068B0F5805F0CD0FFE703988068B0F5CB
:10FFE000005F06D0FFE703988068B0F5405F01D15D
:10FFF000FFE708E045F29E10C0F6020041F25041D2
:020000040801F1
:100000000DF022FBFFE703984068B0F5004F12D0D7
:10001000FFE70398406870B1FFE70398406850B16C
:10002000FFE703984068022805D0FFE7039840687F
:100030000A2801D1FFE708E045F29E10C0F6020051
:1000400041F251410DF000FBFFE70398C0680F2813
:1000500001D8FFE708E045F29E10C0F6020041F229
:1000600052410DF0F1FAFFE704980068039B5A68CB
:100070009968DB6807F05EFA04980168886840F4C4
:1000800080408860F9E1049800680021C4F2010111
:1000900088423CD0FFE704980068B0F1804F36D02A
:1000A000FFE70498006840F20041C4F20001884272
:1000B0002DD0FFE70498006840F60001C4F200016B
:1000C000884224D0FFE70498006840F60041C4F25B
:1000D000000188421BD0FFE70498006840F200410D
:1000E000C4F20101884212D0FFE70498006844F28C
:1000F0000001C4F20101884209D0FFE704980068BA
:1001000041F60001C4F20001884201D1FFE708E096
:1001100045F29E10C0F6020041F261410DF094FAE2
:10012000FFE703984068B0F5004F12D0FFE703984F
:10013000406870B1FFE70398406850B1FFE703984B
:100140004068022805D0FFE7039840680A2801D1DB
:10015000FFE708E045F29E10C0F6020041F264415C
:100160000DF072FAFFE70398C0680F2801D8FFE787
:1001700008E045F29E10C0F6020041F265410DF024
:1001800063FAFFE704980068039A5168D26807F0A1
:1001900087FC04980068502107F0E6F96DE10498A7
:1001A00000680021C4F2010188423CD0FFE70498B6
:1001B0000068B0F1804F36D0FFE70498006840F245
:1001C0000041C4F2000188422DD0FFE70498006886
:1001D00040F60001C4F20001884224D0FFE70498F1
:1001E000006840F60041C4F2000188421BD0FFE7DE
:1001F0000498006840F20041C4F20101884212D024
:10020000FFE70498006844F20001C4F2010188424B
:1002100009D0FFE70498006841F60001C4F200012C
:10022000884201D1FFE708E045F29E10C0F60200C7
:1002300041F271410DF008FAFFE703984068B0F50C
:10024000004F12D0FFE70398406870B1FFE70398B2
:10025000406850B1FFE703984068022805D0FFE7E7
:10026000039840680A2801D1FFE708E045F29E1094
:10027000C0F6020041F274410DF0E6F9FFE7039881
:10028000C0680F2801D8FFE708E045F29E10C0F6CD
:10029000020041F275410DF0D7F9FFE704980068BC
:1002A000039A5168D26807F023FC04980068602123
:1002B00007F05AF9E1E0049800680021C4F2010156
:1002C00088423CD0FFE704980068B0F1804F36D0F8
:1002D000FFE70498006840F20041C4F20001884240
:1002E0002DD0FFE70498006840F60001C4F2000139
:1002F000884224D0FFE70498006840F60041C4F229
:10030000000188421BD0FFE70498006840F20041DA
:10031000C4F20101884212D0FFE70498006844F259
:100320000001C4F20101884209D0FFE70498006887
:1003300041F60001C4F20001884201D1FFE708E064
:1003400045F29E10C0F6020041F281410DF07CF9A9
:10035000FFE703984068B0F5004F12D0FFE703981D
:10036000406870B1FFE70398406850B1FFE7039819
:100370004068022805D0FFE7039840680A2801D1A9
:10038000FFE708E045F29E10C0F6020041F284410A
:100390000DF05AF9FFE70398C0680F2801D8FFE76E
:1003A00008E045F29E10C0F6020041F285410DF0D2
:1003B0004BF9FFE704980068039A5168D26807F088
:1003C0006FFB04980068402107F0CEF855E00498D0
:1003D00000680021C4F2010188423CD0FFE7049884
:1003E0000068B0F1804F36D0FFE70498006840F213
:1003F0000041C4F2000188422DD0FFE70498006854
:1004000040F60001C4F20001884224D0FFE70498BE
:10041000006840F60041C4F2000188421BD0FFE7AB
:100420000498006840F20041C4F20101884212D0F1
:10043000FFE70498006844F20001C4F20101884219
:1004400009D0FFE70498006841F60001C4F20001FA
:10045000884201D1FFE708E045F29E10C0F6020095
:1004600041F294410DF0F0F8FFE704980068039919
:10047000096807F079F800E0FFE70499012081F8A6
:100480003D00FFE70499002081F83C00FFE70020D1
:100490008DF81700FFE79DF8170006B080BD00003B
:1004A00081B0009001B0704780B582B00190019892
:1004B0000068006900F002010020B0EB510F28D065
:1004C000FFE701980068C06800F002010020B0EB6F
:1004D000510F1DD0FFE7019801686FF0020008611D
:1004E000019901200877019800688069800720B190
:1004F000FFE70198FFF7D4FF06E0019800F04CFAFF
:10050000019800F0A3FDFFE7019900200877FFE7BD
:10051000FFE701980068006900F004010020B0EBDB
:10052000910F29D0FFE701980068C06800F004012E
:100530000020B0EB910F1ED0FFE7019801686FF02B
:100540000400086101990220087701980068806919
:1005500010F4407F04D0FFE70198FFF7A1FF06E009
:10056000019800F019FA019800F070FDFFE7019979
:1005700000200877FFE7FFE701980068006900F0B6
:1005800008010020B0EBD10F28D0FFE701980068E8
:10059000C06800F008010020B0EBD10F1DD0FFE7CC
:1005A000019801686FF0080008610199042008773C
:1005B00001980068C069800720B1FFE70198FFF744
:1005C0006FFF06E0019800F0E7F9019800F03EFDAA
:1005D000FFE7019900200877FFE7FFE7019800682F
:1005E000006900F010010020B0EB111F29D0FFE7D7
:1005F00001980068C06800F010010020B0EB111FE6
:100600001ED0FFE7019801686FF0100008610199A2
:100610000820087701980068C06910F4407F04D072
:10062000FFE70198FFF73CFF06E0019800F0B4F9FE
:10063000019800F00BFDFFE7019900200877FFE724
:10064000FFE7019800680069C00780B1FFE70198E3
:100650000068C068C00748B1FFE7019801686FF003
:1006600001000861019801F057F8FFE7FFE70198E2
:1006700000680069C1B20020B0EBD11F13D0FFE7C2
:1006800001980068C068C1B20020B0EBD11F09D04A
:10069000FFE7019801686FF0800008610198FEF79C
:1006A00051FDFFE7FFE701980068006900F0400195
:1006B0000020B0EB911F14D0FFE701980068C068DC
:1006C00000F040010020B0EB911F09D0FFE7019836
:1006D00001686FF040000861019801F033F8FFE70E
:1006E000FFE701980068006900F020010020B0EBEE
:1006F000511F14D0FFE701980068C06800F0200186
:100700000020B0EB511F09D0FFE7019801686FF09E
:10071000200008610198FEF719FDFFE7FFE702B02E
:1007200080BD000080B592B01190002010900F9015
:100730000E900D900C90119800680021C4F20101F8
:10074000884222D1FFE7FFE700200B9043F63000FC
:10075000C4F20200016841F010010160006800F07D
:1007600010000B900B98FFE74FF4D4400C9002213F
:100770000D9101200E900F91109041F20000C4F2F3
:1007800002000CA9FAF73EFA03E11198006840F262
:100790000041C4F20001884222D1FFE7FFE70020B8
:1007A0000A9043F63000C4F20200016841F00401EF
:1007B0000160006800F004000A900A98FFE74FF417
:1007C00080700C9002200D9001210E910F901090DE
:1007D00040F60000C4F202000CA9FAF713FAD7E0C1
:1007E0001198006840F60001C4F20001884223D14C
:1007F000FFE7FFE70020099043F63000C4F2020053
:10080000016841F008010160006800F008000990EB
:100810000998FFE74FF480400C9002200D900121D1
:100820000E9103210F91109040F60040C4F2020097
:100830000CA9FAF7E7F9AAE01198006840F6004120
:10084000C4F20001884222D1FFE7FFE700200890B0
:1008500043F63000C4F20200016841F080010160FB
:10086000006800F0800008900898FFE74FF4E0501F
:100870000C9002200D9001210E910F90109041F6E6
:100880000040C4F202000CA9FAF7BCF97EE011980E
:10089000006840F20041C4F2010188424AD1FFE7FA
:1008A000FFE70020079043F63000C4F20200016821
:1008B00041F480710160006800F48070079007982F
:1008C000FFE7FFE70020069043F63000C4F2020085
:1008D000016841F004010160006800F00400069026
:1008E0000698FFE7402000900C90022002900D90A7
:1008F000012101910E910F9003200390109042F27C
:100900000000C4F202000CA90491FAF77BF9DDF8AB
:1009100000C0019B029A03980499CDF830C00D9253
:100920000E930F92109040F60000C4F20200FAF706
:1009300069F92AE01198006844F20041C4F201010B
:10094000884221D1FFE7FFE70020059043F6300001
:10095000C4F20200016841F020010160006800F06B
:10096000200005900598FFE740200C9002200D9094
:100970000E900F900320109041F20040C4F202004C
:100980000CA9FAF73FF9FFE7FFE7FFE7FFE7FFE70B
:10099000FFE712B080BD000081B0009001B0704749
:1009A00080B586B0049003910292029880B1FFE76F
:1009B000029804280CD0FFE70298082808D0FFE727
:1009C00002980C2804D0FFE702983C2801D1FFE7E9
:1009D00008E045F29E10C0F6020041F217010CF04B
:1009E00033FEFFE703980068602805D0FFE703980F
:1009F0000068702801D1FFE708E045F29E10C0F6BC
:100A0000020041F218010CF01FFEFFE70398806816
:100A100028B1FFE703988068022801D1FFE708E0CA
:100A200045F29E10C0F6020041F219010CF00CFED6
:100A3000FFE70398006928B1FFE7039800690428DD
:100A400001D1FFE708E045F29E10C0F6020041F236
:100A50001A010CF0F9FDFFE7FFE7049890F83C005D
:100A6000012804D1FFE702208DF81700C3E10499A3
:100A7000012081F83C00FFE7FFE7029801900C2875
:100A800000F2AE810199DFE811F00D00AB01AB017E
:100A9000AB019800AB01AB01AB010001AB01AB01B5
:100AA000AB015501049800680021C4F2010188429D
:100AB00060D0FFE704980068B0F1804F5AD0FFE79C
:100AC0000498006840F20041C4F20001884251D00D
:100AD000FFE70498006840F60001C4F20001884274
:100AE00048D0FFE70498006840F60041C4F20001D6
:100AF00088423FD0FFE70498006840F20041C4F20A
:100B00000101884236D0FFE70498006844F20001F2
:100B1000C4F2010188422DD0FFE70498006844F236
:100B20000041C4F20101884224D0FFE70498006824
:100B300044F60001C4F2010188421BD0FFE704988B
:100B4000006841F60001C4F20001884212D0FFE7BC
:100B50000498006841F60041C4F20001884209D0BF
:100B6000FFE70498006842F20001C4F200018842E5
:100B700001D1FFE708E045F29E10C0F6020041F205
:100B800024010CF061FDFFE704980068039906F06A
:100B900001FD04980168886940F0080088610498A4
:100BA0000168886920F0040088610398026904984C
:100BB000016888691043886113E104980068002186
:100BC000C4F2010188423CD0FFE704980068B0F10C
:100BD000804F36D0FFE70498006840F20041C4F22D
:100BE000000188422DD0FFE70498006840F600011C
:100BF000C4F20001884224D0FFE70498006840F660
:100C00000041C4F2000188421BD0FFE7049800684D
:100C100040F20041C4F20101884212D0FFE704987B
:100C2000006844F20001C4F20101884209D0FFE7E4
:100C30000498006841F60001C4F20001884201D125
:100C4000FFE708E045F29E10C0F6020041F23501D0
:100C50000CF0FAFCFFE704980068039906F04CFDDD
:100C600004980168886940F400608861049801680C
:100C7000886920F48060886103980269049801689B
:100C8000886940EA02208861ABE00498006800218E
:100C9000C4F2010188422AD0FFE704980068B0F14D
:100CA000804F24D0FFE70498006840F20041C4F26E
:100CB000000188421BD0FFE70498006840F600015D
:100CC000C4F20001884212D0FFE70498006840F6A1
:100CD0000041C4F20001884209D0FFE7049800688F
:100CE00040F20041C4F20101884201D1FFE708E06F
:100CF00045F29E10C0F6020041F246010CF0A4FC41
:100D0000FFE704980068039906F0ACFD04980168B9
:100D1000C86940F00800C86104980168C86920F0FB
:100D20000400C8610398026904980168C869104307
:100D3000C86156E0049800680021C4F201018842AD
:100D40002AD0FFE704980068B0F1804F24D0FFE775
:100D50000498006840F20041C4F2000188421BD0B0
:100D6000FFE70498006840F60001C4F200018842E1
:100D700012D0FFE70498006840F60041C4F2000179
:100D8000884209D0FFE70498006840F20041C4F2AD
:100D90000101884201D1FFE708E045F29E10C0F64C
:100DA000020041F257010CF04FFCFFE70498006885
:100DB000039906F00DFE04980168C86940F40060CC
:100DC000C86104980168C86920F48060C86103980C
:100DD000026904980168C86940EA0220C86100E01D
:100DE000FFE7FFE70499002081F83C00FFE70020BF
:100DF0008DF81700FFE79DF8170006B080BD0000D2
:100E000080B582B00090009820B9FFE701208DF8EE
:100E1000070012E1009800680021C4F20101884235
:100E200072D0FFE700980068B0F1804F6CD0FFE708
:100E30000098006840F20041C4F20001884263D08B
:100E4000FFE70098006840F60001C4F20001884204
:100E50005AD0FFE70098006840F60041C4F2000154
:100E6000884251D0FFE70098006841F20001C4F2C7
:100E70000001884248D0FFE70098006841F2004135
:100E8000C4F2000188423FD0FFE70098006840F2BA
:100E90000041C4F20101884236D0FFE700980068A3
:100EA00044F20001C4F2010188422DD0FFE700980E
:100EB000006844F20041C4F20101884224D0FFE7F7
:100EC0000098006844F60001C4F2010188421BD07A
:100ED000FFE70098006841F60001C4F20001884273
:100EE00012D0FFE70098006841F60041C4F200010B
:100EF000884209D0FFE70098006842F20001C4F27E
:100F00000001884201D1FFE708E045F29E10C0F6DB
:100F1000020040F20E510CF097FBFFE7009880684A
:100F2000A0B1FFE70098806810280FD0FFE7009875
:100F3000806820280AD0FFE700988068402805D004
:100F4000FFE700988068602801D1FFE708E045F2DC
:100F50009E10C0F6020040F20F510CF075FBFFE747
:100F60000098006960B1FFE700980069B0F5807FE4
:100F700006D0FFE700980069B0F5007F01D1FFE7D8
:100F800008E045F29E10C0F602004FF4A2610CF09A
:100F90005BFBFFE70098806928B1FFE70098806954
:100FA000802801D1FFE708E045F29E10C0F602005C
:100FB00040F211510CF048FBFFE7009890F83D001B
:100FC00040B9FFE70099002081F83C00009800F04C
:100FD00039F8FFE70099022081F83D00009951F8A7
:100FE000040B06F039F90099012081F84600FFE76B
:100FF0000099012081F83E00009981F83F00009996
:1010000081F84000009981F84100FFE7FFE700996F
:10101000012081F84200009981F84300009981F88D
:101020004400009981F84500FFE70099012081F80C
:101030003D0000208DF80700FFE79DF8070002B093
:1010400080BD000081B0009001B0704781B0009079
:1010500001B0704780B58CB00A9009910A98006879
:101060000021C4F20101884214D1FFE70998002849
:1010700000F0E780FFE70998042800F0E280FFE72E
:101080000998082800F0DD80FFE709980C2800F097
:10109000D880FFE70A980068B0F1804F14D1FFE7CD
:1010A0000998002800F0CD80FFE70998042800F097
:1010B000C880FFE70998082800F0C380FFE7099877
:1010C0000C2800F0BE80FFE70A98006840F200415B
:1010D000C4F20001884214D1FFE70998002800F00B
:1010E000B080FFE70998042800F0AB80FFE709987B
:1010F000082800F0A680FFE709980C2800F0A180DE
:10110000FFE70A98006840F60001C4F20001884237
:1011100014D1FFE70998002800F09380FFE70998B1
:10112000042800F08E80FFE70998082800F08980E5
:10113000FFE709980C2800F08480FFE70A98006810
:1011400040F60041C4F20001884210D1FFE709983F
:10115000002876D0FFE70998042872D0FFE70998A5
:1011600008286ED0FFE709980C286AD0FFE70A9894
:10117000006840F20041C4F20101884210D1FFE74B
:10118000099800285DD0FFE70998042859D0FFE7A7
:101190000998082855D0FFE709980C2851D0FFE797
:1011A0000A98006844F20001C4F20101884208D1A3
:1011B000FFE70998002844D0FFE70998042840D0A9
:1011C000FFE70A98006844F20041C4F20101884236
:1011D00003D1FFE70998A0B3FFE70A98006844F637
:1011E0000001C4F20101884203D1FFE7099840B32E
:1011F000FFE70A98006841F60001C4F20001884246
:1012000007D1FFE70998E0B1FFE70998042818D053
:10121000FFE70A98006841F60041C4F200018842E5
:1012200003D1FFE7099860B1FFE70A98006842F22E
:101230000001C4F20001884204D1FFE7099808B90F
:10124000FFE708E045F29E10C0F6020040F294511C
:101250000CF0FAF9FFE7099828B9FFE70A9890F827
:101260003E0007901CE00998042805D1FFE70A9882
:1012700090F83F00069010E00998082805D1FFE794
:101280000A9890F84000059004E00A9890F8410010
:101290000590FFE705980690FFE706980790FFE79F
:1012A0000798012804D0FFE701208DF82F00AFE058
:1012B000099828B9FFE70A99022081F83E001EE04C
:1012C0000998042806D1FFE70A99022081F83F0017
:1012D000049012E00998082806D1FFE70A99022035
:1012E00081F84000039005E00A99022081F841004E
:1012F0000390FFE703980490FFE70498FFE70A983C
:10130000006809990122019206F074F801980A997F
:1013100009680022C4F20102914202900CD0FFE75A
:101320000A9800684FF60041CBF6FE710844B0FA07
:1013300080F040090290FFE70298C00738B1FFE74C
:101340000A980168486C40F400404864FFE70A9836
:1013500000680021C4F2010188423CD0FFE70A98EE
:101360000068B0F1804F36D0FFE70A98006840F27D
:101370000041C4F2000188422DD0FFE70A980068BE
:1013800040F60001C4F20001884224D0FFE70A9829
:10139000006840F60041C4F2000188421BD0FFE71C
:1013A0000A98006840F20041C4F20101884212D05C
:1013B000FFE70A98006844F20001C4F20101884284
:1013C00009D0FFE70A98006841F60001C4F2000165
:1013D000884212D1FFE70A980068806800F0070091
:1013E00008900898062807D0FFE70A98016808685F
:1013F00040F001000860FFE706E00A98016808680D
:1014000040F001000860FFE700208DF82F00FFE7A3
:101410009DF82F000CB080BD80B586B0059004917A
:10142000059800680021C4F20101884214D1FFE749
:101430000498002800F0E780FFE70498042800F0F3
:10144000E280FFE70498082800F0DD80FFE70498B9
:101450000C2800F0D880FFE705980068B0F1804FB5
:1014600014D1FFE70498002800F0CD80FFE704982E
:10147000042800F0C880FFE70498082800F0C38023
:10148000FFE704980C2800F0BE80FFE7059800688D
:1014900040F20041C4F20001884214D1FFE70498F1
:1014A000002800F0B080FFE70498042800F0AB802B
:1014B000FFE70498082800F0A680FFE704980C28AE
:1014C00000F0A180FFE70598006840F60001C4F233
:1014D0000001884214D1FFE70498002800F09380AF
:1014E000FFE70498042800F08E80FFE7049808289E
:1014F00000F08980FFE704980C2800F08480FFE763
:101500000598006840F60041C4F20001884210D1FD
:10151000FFE70498002876D0FFE70498042872D0EB
:10152000FFE7049808286ED0FFE704980C286AD0DB
:10153000FFE70598006840F20041C4F201018842CB
:1015400010D1FFE7049800285DD0FFE70498042835
:1015500059D0FFE70498082855D0FFE704980C28D5
:1015600051D0FFE70598006844F20001C4F2010180
:10157000884208D1FFE70498002844D0FFE7049888
:10158000042840D0FFE70598006844F20041C4F207
:101590000101884203D1FFE70498A0B3FFE7059853
:1015A000006844F60001C4F20101884203D1FFE75C
:1015B000049840B3FFE70598006841F60001C4F2C3
:1015C0000001884207D1FFE70498E0B1FFE70498E3
:1015D000042818D0FFE70598006841F60041C4F2DE
:1015E0000001884203D1FFE7049860B1FFE7059846
:1015F000006842F20001C4F20001884204D1FFE712
:10160000049808B9FFE708E045F29E10C0F6020012
:101610004FF4B9610CF018F8FFE7059800680499D9
:10162000002205F0E7FE0598016801200022C4F2BF
:101630000102914203900CD0FFE7059800684FF635
:101640000041CBF6FE710844B0FA80F040090390E7
:10165000FFE70398C007D8B1FFE7FFE705980068E8
:10166000006A41F21111084210D1FFE705980068A5
:10167000006A40F24441084207D1FFE7059801683B
:10168000486C20F400404864FFE7FFE7FFE7FFE70E
:10169000FFE705980068006A41F21111084210D175
:1016A000FFE705980068006A40F24441084207D10C
:1016B000FFE705980168086820F001000860FFE76F
:1016C000FFE7FFE7049828B9FFE70599012081F8B3
:1016D0003E001EE00498042806D1FFE7059901208A
:1016E00081F83F00029012E00498082806D1FFE735
:1016F0000599012081F84000019005E0059901203D
:1017000081F841000190FFE701980290FFE70298FD
:10171000FFE7002006B080BD81B00090009800680F
:1017200041F20041C4F20001884208D1FFE741F6CE
:10173000B031C2F20001086801300860FFE701B073
:101740007047000081B0009001B0704782B00190F6
:10175000ADF8021002B0704780B582B001900198D8
:1017600007F060FE8DF803009DF8030004281BD0ED
:10177000FFE79DF8030000EBC00140F2C040C2F259
:10178000000000EB8100C06968B1FFE79DF803002D
:1017900000EBC00140F2C040C2F2000000EB81004B
:1017A000C0698047FFE7FFE702B080BD80B582B027
:1017B000019001980168C86820F49070C860019891
:1017C0000168486920F0010048610198006B012818
:1017D00007D1FFE701980168C86820F01000C860D1
:1017E000FFE7019800684069400600282BD5FFE715
:1017F00001980168486920F0400048610198806BB9
:1018000098B1FFE70198816B49F21130C0F60100F1
:1018100008650198806BF8F759FB28B1FFE701983C
:10182000806B016D8847FFE70CE001990020C885B7
:10183000019A202182F83E10019908630198FFF770
:101840008BFFFFE70CE001990020C885019A202159
:1018500082F83E10019908630198FFF77DFFFFE7CA
:10186000002002B080BD000080B582B001900198D8
:1018700007F0D8FD8DF803009DF8030004281BD065
:10188000FFE79DF8030000EBC00140F2C040C2F248
:10189000000000EB8100006968B1FFE79DF80300DC
:1018A00000EBC00140F2C040C2F2000000EB81003A
:1018B00000698047FFE7FFE702B080BD80B588B0D0
:1018C0000790079800680068069007980068C0684D
:1018D00005900798006840690490002003900290EA
:1018E000069800F00F000390039888B9FFE79DF871
:1018F0001800800600280AD5FFE79DF8140080062E
:10190000002804D5FFE7079807F0BEFD78E1FFE760
:101910000398002800F0B480FFE79DF81000C0078E
:1019200038B9FFE7BDF8140010F4907F00F0A880EC
:10193000FFE79DF81800C00758B1FFE79DF81500B4
:10194000C00730B1FFE70799086C40F00100086458
:10195000FFE79DF81800400700280BD5FFE79DF82A
:101960001000C00730B1FFE70799086C40F0020093
:101970000864FFE79DF81800800700280BD5FFE7F3
:101980009DF81000C00730B1FFE70799086C40F0E0
:1019900004000864FFE79DF818000007002811D52F
:1019A000FFE79DF814008006002805D4FFE79DF8A6
:1019B0001000C00730B1FFE70799086C40F008003D
:1019C0000864FFE70798006C002858D0FFE79DF8EF
:1019D0001800800600280AD5FFE79DF8140080064D
:1019E000002804D5FFE7079807F04EFDFFE70798AA
:1019F00000684069C0F3801002900798006C0007EF
:101A0000002803D4FFE7029888B3FFE7079807F0A0
:101A1000C3FC0798006840694006002822D5FFE70C
:101A200007980168486920F0400048610798806B7A
:101A300098B1FFE70798816B49F2BD10C0F601002D
:101A400008650798806BF8F741FA28B1FFE7079817
:101A5000806B016D8847FFE703E00798FFF704FFFD
:101A6000FFE703E00798FFF7FFFEFFE706E00798B0
:101A7000FFF7FAFE079900200864FFE7FFE7BFE0E1
:101A80000798006B012840F09B80FFE79DF8180045
:101A9000C006002840F19480FFE79DF81400C006BE
:101AA000002840F18D80FFE7FFE7002001900798B4
:101AB00000680068019007980068406801900198EC
:101AC000FFE7079800684069400600284AD5FFE70D
:101AD0000798806B00684068ADF80200BDF802000E
:101AE00000283ED0FFE7BDF802000799898D8842A3
:101AF00037DAFFE7BDF802000799C8850798806BC1
:101B0000C069B0F5807F24D0FFE707980168C868F6
:101B100020F48070C86007980168486920F00100CF
:101B2000486107980168486920F0400048610799BA
:101B3000202081F83E00079900200863079801687B
:101B4000C86820F01000C8600798806BF8F748F963
:101B5000FFE70798818DC28D891A89B2FFF7F6FDDC
:101B6000FFE74DE00799888DC98D401AADF8000058
:101B70000798C08D18B3FFE7BDF80000F8B1FFE784
:101B800007980168C86820F49070C86007980168D9
:101B9000486920F0010048610799202081F83E0043
:101BA00007990020086307980168C86820F01000B2
:101BB000C8600798BDF80010FFF7C8FDFFE71FE0F9
:101BC0009DF81800000600280AD5FFE79DF81400CC
:101BD0000006002804D5FFE7079807F037FE0FE05E
:101BE0009DF81800400600280AD5FFE79DF814006C
:101BF0004006002804D5FFE7079807F0F1FBFFE750
